:100000000C94131F0C94401F0C94401F0C94401F21
:100010000C94401F0C94401F0C94401F0C94401FE4
:100020000C94401F0C94401F0C94401F0C94401FD4
:100030000C94401F0D94EC110C94401F0C94401F25
:100040000C94401F0C94A8270C94401F0C94401F44
:100050000C94401F0C94401F0C9489D50D94430EB2
:100060000C94401F0C94DC2E0C94401F0C94401FE9
:100070000C94401F0C94401F0C94401F0C94401F84
:100080000C94401F0C94401F0C94401F0C94401F74
:100090000C94401F0C94401F0C94401F0D94990623
:1000A0000C94401F0C94401F0C94401F0C94401F54
:1000B0000C94401F0C94401F0C94401F0C94401F44
:1000C0000C94401F0C94401F0C94401F0C94401F34
:1000D0000C94401F0C94401F0C94401F0C94401F24
:1000E0000C94401F084AD73B3BCE016E84BCBFFD39
:1000F000C12F3D6C74319ABD56833DDA3D00C77FF8
:1001000011BED9E4BB4C3E916BAAAABE0000008090
:100110003F05A84CCDB2D44EB93836A9020C50B91F
:10012000918688083CA6AAAA2ABE000000803F4506
:10013000313A200045303A20005A3A2000593A20FE
:1001400000583A20004D53312C4D53322050696EE7
:10015000730A0024F404D9201BC40C5C0E9804C458
:10016000095F0265077101F405F900FB04B300485B
:10017000048700C10369005803550003034500BE0E
:10018000023A008402310053022A002902250004A9
:10019000022000E4011C00C8011900AF01170098FB
:1001A000011400840113007101100061011000515D
:1001B000010E0043010D0036010B002B010B002046
:1001C000010B00150109000C01090003010800FBE7
:1001D000000800F3000800EB000700E4000600DE62
:1001E000000600D8000600D2000600CC000500C7BB
:1001F000000500C2000500BD000400B9000400B500
:10020000000400B1000400AD000400A9000400A532
:10021000000300A20003009F0004009B000300985D
:100220000003009500020093000300900003008D7E
:100230000002008B00030088000200860002008498
:10024000000300810002007F0002007D0002007BAD
:1002500000020079000200770001007600020074BD
:1002600000020072000100710002006F0002006DC8
:100270000001006C0002006A0001006900020067D2
:1002800000010066000100650001006400020062D8
:1002900000010061000100600001005F0002005DDC
:1002A0000001005C0001005B0001005A00010059E0
:1002B00000010058000100570001005600010055E0
:1002C00000010054000100530000005300010052DF
:1002D00000010051000100500001004F0001004EDC
:1002E0000000004E0001004D0001004C0001004BD9
:1002F0000000004B0001004A0001004900010048D5
:1003000000000048000100470001004600000046D0
:1003100000010045000000450001004400010043C9
:1003200000000043000100420000004200010041C3
:1003300000000041000100400001003F0000003FBC
:100340000001003E0000003E0001003D0000003DB5
:100350000001003C0000003C0000003C0001003BAC
:100360000000003B0001003A0000003A00010039A3
:10037000000000390001003800000038000000389B
:100380000001003700000037000100360000003691
:100390000000003600010035000000350000003587
:1003A000000100340000003400000034000100337C
:1003B0000000003300000033000100320000003272
:1003C0000000003200010031000000310000003167
:1003D0000001003000000030000000300001002F5C
:1003E0000000002F0000002F0000002F0001002E51
:1003F0000000002E0000002E0001002D0000002D46
:100400000000002D0000002D0001002C0000002C39
:100410000000002C0000002C0001002B0000002B2D
:100420000000002B0000002B0001002A0000002A21
:100430000000002A0000002A000100290000002915
:100440000000002900000029000000290001002808
:1004500000000028000000280000002800000028FC
:1004600000010027000000270000002700000027EF
:1004700000000027000100260000002600000026E2
:1004800000000026000000260001002500000025D5
:1004900000000025000000250000002500000025C8
:1004A00000010024000000240000002400000024BB
:1004B00000000024000100230000002300000023AE
:1004C00000000023000000230000002300000023A0
:1004D0000001002200000022000000220000002293
:1004E0000000002200000022000100210000002185
:1004F0000000002100000021000000210000002178
:100500000000002100010020000000200000002069
:10051000000000200000002000000020000000205B
:10052000000000200001001F0000001F0000001F4D
:100530000000001F0000001F0000001F0000001F3F
:100540000001001E0000001E0000001E0000001E32
:1005500000000024F4D43050C38E20C2A240178281
:100560008B7011127A910D816CD90AA861E108C7CC
:10057000586607615143061E4B5D05C145A7041A25
:10058000411104093D9803713931034036DB02659E
:10059000339102D4305402802E1D02632CEE01757B
:1005A0002AC501B028A001102781018F2564012BE5
:1005B000244B01E0223401AC211F018D200D01806C
:1005C0001FFC00841EED00971DDF00B81CD200E662
:1005D0001BC600201BBC00641AB200B219A8000A96
:1005E00019A0006A189900D117910040178B00B527
:1005F00016840031167E00B31579003A157300C7D2
:10060000146F0058146A00EE136600881363002507
:10061000135E00C7125B006C12570015125400C124
:1006200011510070114F0021114B00D61049008D5F
:100630001047004610440002104200C00F400080E6
:100640000F3E00420F3C00060F3B00CB0E380093DC
:100650000E37005C0E3500270E3400F30D3200C15A
:100660000D3100900D3000600D2E00320D2D000573
:100670000D2C00D90C2B00AE0C2900850C29005C38
:100680000C2700350C27000E0C2600E80B2400C4B4
:100690000B2400A00B23007D0B23005A0B210039F3
:1006A0000B2100180B2000F80A1F00D90A1E00BBFE
:1006B0000A1E009D0A1D00800A1D00630A1C0047D7
:1006C0000A1B002C0A1B00110A1A00F7091A00DD88
:1006D000091900C4091900AB091900920917007B18
:1006E000091800630917004C091600360916002086
:1006F0000916000A091500F5081500E0081400CCD9
:10070000081400B8081400A4081400900813007D11
:100710000812006B08130058081200460812003433
:10072000081100230811001208110001081100F03F
:10073000071000E0071000D0071000C0071000B03D
:10074000070F00A107100091070E0083070F007428
:10075000070F0065070E0057070E0049070E003B04
:10076000070D002E070E0020070D0013070D0006D1
:10077000070D00F9060C00ED060D00E0060C00D494
:10078000060C00C8060C00BC060C00B0060C00A449
:10079000060B0099060C008D060B0082060B0077F5
:1007A000060B006C060B0061060A0057060B004C96
:1007B000060A0042060A0038060A002E060A00242D
:1007C000060A001A060A001006090007060A00FDBC
:1007D000050900F4050900EB050900E2050900D947
:1007E000050900D0050900C7050900BE050900B5C7
:1007F000050800AD050800A50509009C0508009442
:100800000508008C050800840508007C05080074B4
:100810000508006C050700650508005D0507005622
:100820000508004E05070047050700400508003889
:10083000050700310507002A050700230507001CEE
:10084000050600160507000F05070008050600024B
:10085000050700FB040600F5040700EE040600E8A7
:10086000040600E2040700DB040600D5040600CFFE
:10087000040600C9040600C3040600BD040600B750
:10088000040600B1040500AC040600A6040600A09E
:100890000405009B04060095040500900406008AE8
:1008A00004050085040500800406007A040500752F
:1008B000040500700405006B040500660405006172
:1008C0000405005C04050057040500520405004DB2
:1008D00004050048040500430405003E0404003AF2
:1008E00004050035040500300404002C040500272D
:1008F000040400230405001E0404001A0404001666
:10090000040500110404000D04040009040500049A
:1009100004040000040400FC030400F8030400F4D1
:10092000030400F0030400EC030400E8030400E403
:10093000030400E0030400DC030400D8030400D433
:10094000030400D0030400CC030400C8030300C563
:100950000303006563686F3A00656E6473746F70BB
:1009600073206869743A205A00205A3A00656E6410
:1009700073746F7073206869743A20590020593A73
:1009800000656E6473746F7073206869743A2058E0
:100990000020583A00656E6473746F707320686944
:1009A000743A200000060900FE06018902FE20FFBD
:1009B000FE07FE06FE00000006000701060606020E
:1009C00000808080800080030303060103A0A0A0B4
:1009D0000507070600FF5050F850F8505005090968
:1009E0000600FE2070A8A07028A87020060808063F
:1009F00000FF40A84810204854080507070600FFDC
:100A000060909060989068010303060203808080E4
:100A10000207070602FF40808080808040020707AF
:100A20000602FF804040404040800505050600006A
:100A30008850F850880505050600002020F8202081
:100A40000204040602FEC0404080050101060002C7
:100A5000F8020202060200C0C004060606010010E9
:100A6000102040808004060606010060909090905F
:100A70006003060606010040C0404040E004060650
:100A80000601006090102040F0040606060100F008
:100A900020601010E005060606000010305090F8A7
:100AA00010040606060100F080E01010E0040606BF
:100AB0000601006080E0909060040606060100F0E8
:100AC00010102040400406060601006090609090DF
:100AD0006004060606010060909070106002050533
:100AE000060200C0C000C0C00207070602FEC0C068
:100AF00000C04040800505050600001860806018B1
:100B0000050303060001F800F8050505060000C00E
:100B1000300830C0040707060100609010604000F4
:100B2000400506060600007090A8B0807005060615
:100B3000060000205088F88888050606060000F0A8
:100B400088F08888F0040606060100609080809096
:100B500060040606060100E090909090E00406060E
:100B6000060100F080E08080F0040606060100F037
:100B700080E0808080040606060100609080B090CE
:100B8000600406060601009090F09090900306061F
:100B9000060100E040404040E0050606060000383F
:100BA000101010906004060606010090A0C0A090EE
:100BB000900406060601008080808080F00506060D
:100BC00006000088D8A8A8888804060606010090B8
:100BD000D0B090909005060606000070888888883E
:100BE00070040606060100E09090E080800407078C
:100BF0000601FF609090D0B0601004060606010068
:100C0000E09090E09090040606060100609040207D
:100C10009060050606060000F8202020202004062B
:100C20000606010090909090906004060606010070
:100C3000909090F060600506060600008888A8A8DD
:100C4000D888050606060000885020205088050632
:100C500006060000888850202020040606060100B1
:100C6000F010204080F0030606060100E08080803E
:100C700080E0040606060100808040201010030674
:100C800006060100E020202020E005030306000303
:100C90002050880501010600FEF802020206020447
:100CA000804004040406010070909070040606065B
:100CB00001008080E09090E0040404060100708050
:100CC00080700406060601001010709090700404F5
:100CD0000406010060B0C070040606060100205042
:100CE00040E040400406060601FE609090701060EF
:100CF0000406060601008080E09090900306060638
:100D000001004000C04040E00308080601FE20004A
:100D100060202020A0400406060601008080A0C0BC
:100D2000A090030606060100C040404040E00504D4
:100D300004060000D0A8A888040404060100E0907E
:100D4000909004040406010060909060040606067A
:100D500001FEE09090E080800406060601FE70909F
:100D600090701010040404060100A0D080800404D8
:100D70000406010070C030E0040606060100404091
:100D8000E040502004040406010090909070040498
:100D9000040601009090606005040406000088A825
:100DA000A850040404060100906060900406060642
:100DB00001FE909090709060040404060100F02001
:100DC00040F003070706010020404080404020011A
:100DD00007070602FF808080808080800307070667
:100DE0000100804040204040800402020601035080
:100DF000A0FFFFFFFFFFFFFFFFFFFFFFFFFFFFFF62
:100E0000FFFFFFFFFFFFFFFFFFFFFFFFFFFFFFFFF2
:100E1000FFFF000000060007010606060200800032
:100E2000808080800406060601FF2070A0A070204C
:100E30000507070600FF304840F04040F80505056B
:100E4000060000A8508850A8050606060000885035
:100E5000F820F8200107070602FF808080008080CC
:100E6000800407070601FF708060906010E00301B6
:100E700001060105A0060707060000788494A494E3
:100E8000847803050506010160A06000E005050502
:100E90000600002850A05028040303060100F010AB
:100EA00010040101060102F006070706000078841D
:100EB000B4A4A48478040101060105F00403030628
:100EC00001026090600507070600FF2020F820203F
:100ED00000F803050506010140A02040E0030505D8
:100EE000060101C0204020C0020202060204408028
:100EF0000405050601FF9090B0D0800506060600A7
:100F00000078E8E868282801010106020280020250
:100F1000020602FE408003050506010140C0404074
:100F2000E003050506010140A04000E005050506B7
:100F30000000A0502850A00508080600FF40C0404F
:100F400050703078100508080600FF40C040506817
:100F50000810380508080600FFC0204030F030783F
:100F6000100407070601002000206080906005073C
:100F700007060000402020507088880507070600FB
:100F800000102020507088880507070600002050B8
:100F900020507088880507070600002850205070F0
:100FA00088880507070600005000205070888805D3
:100FB00007070600002050205070888805060606A6
:100FC000000078A0F0A0A0B80408080601FE609018
:100FD0008080906020400407070601004020F080D8
:100FE000E080F00407070601002040F080E080F078
:100FF0000407070601002050F080E080F004070796
:101000000601005000F080E080F0030707060100B1
:101010008040E0404040E00307070601002040E038
:10102000404040E003070706010040A0E040404088
:10103000E0030707060100A000E0404040E005068D
:10104000060600007048E8484870040707060100DB
:1010500050A090D0B0909004070706010040206097
:1010600090909060040707060100204060909090E7
:10107000600407070601002050609090906004070C
:101080000706010050A060909090600407070601D9
:1010900000500060909090600505050600008850A3
:1010A0002050880408080601FF1070B0B0D0D0E0CE
:1010B000800407070601004020909090906004078C
:1010C00007060100204090909090600407070601F9
:1010D0000020509090909060040707060100500097
:1010E000909090906005070706000010208850201F
:1010F000202004060606010080E09090E0800406AF
:10110000060601006090A0A090A004070706010059
:1011100040200070909070040707060100204000F6
:1011200070909070040707060100205000709090A6
:101130007004070706010050A0007090907004062C
:101140000606010050007090907004070706010029
:101150002050207090907005040406000070A8B024
:10116000780406060601FE708080702040040707A0
:1011700006010040200060B0C070040707060100AF
:1011800020400060B0C07004070706010020500036
:1011900060B0C070040606060100500060B0C07068
:1011A000030707060100804000C04040E003070736
:1011B000060100204000C04040E003070706010090
:1011C00040A000C04040E0030606060100A000C0A9
:1011D0004040E00407070601003060107090906006
:1011E00004070706010050A000E090909004070754
:1011F000060100402000609090600407070601008F
:101200002040006090906004070706010020500015
:101210006090906004070706010050A00060909065
:101220006004060606010050006090906005050508
:101230000600002000F8002004040406010070B03D
:10124000D0E0040707060100402000909090700451
:1012500007070601002040009090907004070706E1
:101260000100205000909090700406060601005086
:1012700000909090700409090601FE2040009090B3
:10128000907090600408080601FE8080E09090E075
:1012900080800408080601FE5000909090709060D5
:1012A00000060900FE070199032B20FFFE08FE0738
:1012B000FE00000006000001070706020080808093
:1012C00080800080030303060104A0A0A005070797
:1012D0000600005050F850F850500507070600006F
:1012E0002070A07028702005070706000048A8504D
:1012F0002050A89005070706000040A0A040A89035
:1013000068010303060204808080030707060100CA
:101310002040808080402003070706010080402095
:10132000202040800505050600018850F8508805FA
:1013300005050600012020F820200303030601FF15
:10134000604080050101060003F80303030601FF66
:1013500040E0400507070600000808102040808094
:1013600005070706000020508888885020050707D9
:101370000600002060A0202020F8050707060000D6
:10138000708808304080F8050707060000F808104C
:101390003008887005070706000010305090F810DC
:1013A00010050707060000F880B0C8088870050718
:1013B00007060000304080B0C888700507070600A7
:1013C00000F808101020404005070706000070884C
:1013D000887088887005070706000070889868087C
:1013E00010600307070601FF40E0400040E04003B3
:1013F00007070601FF40E040006040800407070641
:10140000010010204080402010050303060002F870
:1014100000F80407070601008040201020408005E6
:101420000707060000708810202000200507070627
:101430000000708898A8B08070050707060000209B
:10144000508888F88888050707060000F04848702B
:101450004848F00507070600007088808080887083
:10146000050707060000F04848484848F005070708
:10147000060000F88080F08080F80507070600006D
:10148000F88080F080808005070706000070888063
:1014900080988870050707060000888888F8888883
:1014A00088030707060100E04040404040E0050790
:1014B000070600003810101010906005070706009E
:1014C000008890A0C0A090880507070600008080D3
:1014D00080808080F80507070600008888D8A888E3
:1014E00088880507070600008888C8A898888805A6
:1014F0000707060000708888888888700507070637
:101500000000F08888F08080800508080600FF70E1
:1015100088888888A87008050707060000F0888872
:10152000F0A0908805070706000070888070088882
:1015300070050707060000F820202020202005075E
:1015400007060000888888888888700507070600D5
:1015500000888888505050200507070600008888BA
:1015600088A8A8D88805070706000088885020505A
:10157000888805070706000088885020202020055D
:101580000707060000F80810204080F80307070648
:101590000100E08080808080E00507070600008071
:1015A000804020100808030707060100E0202020E3
:1015B0002020E005030306000420508805010106F1
:1015C00000FFF8020202060206804005050506003B
:1015D0000070087888780507070600008080B0C88A
:1015E00088C8B0050505060000708880887005076A
:1015F0000706000008086898889868050505060031
:10160000007088F88070050707060000304840F039
:101610004040400507070600FE78888878088870F3
:101620000507070600008080B0C888888803070780
:101630000601004000C0404040E00409090601FEE8
:101640001000301010109090600507070600008011
:10165000808890E09088030707060100C040404062
:101660004040E0050505060000D0A8A8A8880505AB
:1016700005060000B0C888888805050506000070CA
:10168000888888700507070600FEB0C888C8B08043
:10169000800507070600FE68988898680808050511
:1016A00005060000B0C880808005050506000070B2
:1016B000807008F00507070600004040F0404048F1
:1016C0003005050506000088888898680505050628
:1016D000000088885050200505050600008888A86D
:1016E000A85005050506000088502050880507070A
:1016F0000600FE88889868088870050505060000C1
:10170000F8102040F8040707060100304020C020F0
:1017100040300107070602008080808080808004BE
:101720000707060100C02040304020C00503030623
:10173000000448A890000000010000000000010023
:101740000000000001000000000001000000000097
:101750000100000000000100000000000100000086
:101760000000010000000000010000000000010076
:101770000000000001000000000001000000000067
:101780000100000000000100000000000100000056
:101790000000010000000000010000000000010046
:1017A0000000000001000000000001000000000037
:1017B0000100000000000100000000000100000026
:1017C0000000010000000000010000000000010016
:1017D0000000000001000000000001000000000007
:1017E00001000000000001000000000001000000F6
:1017F00000000100000000000100000000000600E1
:1018000000010707060200800080808080800507B5
:10181000070600FF2078A0A0A07820050707060093
:1018200000304840E04048B00505050600008870DB
:101830005070880508080600FF88885020F820208E
:101840002001070706020080808000808080050854
:10185000080600FF7080E090483808700301010618
:101860000107A00507070600007088A8C8A88870AF
:101870000406060601017090B05000F0060505064A
:1018800000002448904824040202060102F01004DB
:101890000101060103F00507070600007088E8C88B
:1018A000C88870050101060007F803030306010458
:1018B00040A0400506060600002020F82020F8047D
:1018C000050506010360902040F0040505060103AC
:1018D000E0106010E00202020602064080050606E3
:1018E0000600FF888888C8B08005070706000078D2
:1018F000E8E86828282801010106020380020202A4
:101900000602FE408003050506010340C04040E09A
:101910000406060601016090906000F006050506C9
:10192000000090482448900609090600FF40C04086
:1019300040E40C143C040609090600FF40C0404086
:10194000E81404081C0509090600FFC0204020C84F
:101950001828780805070706000020002020408886
:10196000700508080600004020708888F8888805FF
:1019700008080600001020708888F8888805080884
:101980000600002050708888F8888805080806003E
:101990000048B0708888F88888050808060000505C
:1019A00000708888F88888050808060000205070B4
:1019B0008888F888880607070600003C50909CF04D
:1019C000909C0509090600FE708880808088702040
:1019D0004005080806000040F88080F08080F80587
:1019E000080806000010F88080F08080F8050808DC
:1019F00006000020F88080F08080F80508080600C6
:101A00000050F88080F08080F8030808060100800C
:101A100040E040404040E00308080601002040E06C
:101A200040404040E003080806010040A0E040407C
:101A30004040E0030808060100A000E040404040AC
:101A4000E0050707060000F04848E84848F00508A8
:101A500008060000285088C8A89888880508080645
:101A600000004020708888888870050808060000FB
:101A700010207088888888700508080600002050AB
:101A800070888888887005080806000028507088CB
:101A900088888870050808060000500070888888CB
:101AA0008870050505060000885020508805070746
:101AB000060000709898A8C8C870050808060000BD
:101AC0004020888888888870050808060000102053
:101AD00088888888887005080806000020500088DB
:101AE0008888887005080806000050008888888863
:101AF00088700508080600001020888850202020E3
:101B000005070706000080F088F080808005070741
:101B1000060000708890A09088B0050808060000B4
:101B2000402000700878887805080806000010201A
:101B300000700878887805080806000020500070BA
:101B40000878887805080806000028500070087892
:101B50008878050707060000500070087888780527
:101B600008080600002050207008788878060505CF
:101B700006000078147C907C0507070600FE70883C
:101B8000808870204005080806000040200070880A
:101B9000F880700508080600001020007088F880A2
:101BA000700508080600002050007088F880700555
:101BB000070706000050007088F8807003080806C8
:101BC0000100804000C0404040E0030808060100DA
:101BD000408000C0404040E003080806010040A0EB
:101BE00000C0404040E0060A0A0600FEA4A800FC2F
:101BF0008480808084FC060A0A0600FE549400FC5F
:101C00008404040484FC050808060000285000B081
:101C1000C888888805080806000040200070888869
:101C20008870040A0A0602FE3040809090909090DE
:101C30009090040A0A0600FEC020109090909090A8
:101C40009090060707060001448C8C8480403C0677
:101C5000070706000188C4C4840408F005050506CA
:101C600000012000F8002005080806000040F0C828
:101C70008888987810050808060000E0F8888888A9
:101C80008888F80505050600012030F83020050891
:101C9000080600002070F820202020E00509090631
:101CA00000FF2070A8A8B888885020050909060000
:101CB000FFE080C0B0A8A83028280509090600FF69
:101CC000F8A88888888888A8F8050A0A0600FE20EF
:101CD0005050505088A8A8887000000000000000F4
:101CE00000000000007FFFE0000000000000000096
:101CF000000000007000E000000000000000000094
:101D0000000000630C600000000000000000000004
:101D10000000470E2000000000000000000000004E
:101D2000004F0F2000000000000000000000000035
:101D30005F0FA00000000000000000000000005E37
:101D400007A07F80003FC0003FC00041040040600A
:101D500020FBC00079E00079E00020820040F02004
:101D6000F3C00076E00076E00020820040F020EB37
:101D7000C0007EE0007EE0004104004060207B80E7
:101D8000003DC00039C0008208005E07A07B8000D3
:101D90003BC0003EC0010410005F0FA0FBC00077F5
:101DA000E00076E0010410004F0F20FBC00070E05F
:101DB0000079E000820800470E20FFC0007FE000AD
:101DC0007FE000410400630C603F00001F80001FA3
:101DD00080000000007000E01E00000F00000F00F7
:101DE00001FFFF807FFFE00C0000060000060001FD
:101DF000FFFF800000000000000000000000000065
:101E000000007FFFE0000000000000000000000074
:101E1000007000E000000000000000000000000072
:101E200061F86000000000000000000000000041B8
:101E3000F82000000000000000000000000040F05A
:101E400020000000000000000000000000406020B2
:101E50000000000000000000000000005801A07F0A
:101E600080003FC0003FC0004104005C63A0FBC095
:101E70000079E00079E0002082005EF7A0F3C00066
:101E800076E00076E0002082005EF7A0EBC0007EE6
:101E9000E0007EE0004104005C63A07B80003DC068
:101EA0000039C0008208005801A07B80003BC000C0
:101EB0003EC001041000406020FBC00077E00076C7
:101EC000E00104100040F020FBC00070E00079E069
:101ED0000082080041F820FFC0007FE0007FE000A2
:101EE00041040061F8603F00001F80001F80000077
:101EF00000007000E01E00000F00000F0001FFFF57
:101F0000807FFFE00C0000060000060001FFFF805C
:101F10000000005900B02000B02000B02000B02028
:101F2000002D2D3A2D2D004E6F204361726400501C
:101F300072696E742066726F6D2053440053746F23
:101F400070205072696E7400526573756D65205013
:101F500072696E74005061757365205072696E7499
:101F600000436F6E66696775726174696F6E0054C5
:101F7000656D7065726174757265004D6F76656D23
:101F8000656E740054756E6500496E666F207363EC
:101F90007265656E00F92E2E004D61696E004D323E
:101FA00034004D3233202573004D383420582059E9
:101FB000205A204500526573746F7265204661692E
:101FC0006C73616665004C6F6164206D656D6F7246
:101FD000790053746F7265206D656D6F7279004181
:101FE0006476616E6365642053657474696E6773AB
:101FF000004D61696E004531737470732F6D6D0013
:102000004531737470732F6D6D0045737465707313
:102010002F6D6D004573746570732F6D6D005A736D
:10202000746570732F6D6D005A73746570732F6DC6
:102030006D005973746570732F6D6D0059737465FD
:1020400070732F6D6D005873746570732F6D6D0014
:102050005873746570732F6D6D00412D72657472C5
:1020600061637400412D7265747261637400416D27
:102070006178206500416D6178206500416D61786F
:10208000207A00416D6178207A00416D6178207975
:1020900000416D6178207900416D617820780041C0
:1020A0006D61782078005654726176206D696E00FB
:1020B0005654726176206D696E00566D696E0056D9
:1020C0006D696E00566D6178206500566D617820EF
:1020D0006500566D6178207A00566D6178207A002F
:1020E000566D6178207900566D6178207900566DC3
:1020F0006178207800566D617820780056652D6AE9
:1021000065726B0056652D6A65726B00567A2D6A92
:1021100065726B00567A2D6A65726B005678792D60
:102120006A65726B005678792D6A65726B0041633F
:1021300063656C00416363656C005A204F6666738B
:102140006574005A204F666673657400436F6E664F
:10215000696775726174696F6E00436F6F6C646F4D
:10216000776E0054474C41534500504F4C59434102
:102170005242004C4159574F4F44004C4159425232
:1021800049434B004E2D56454E5400414C4C4F593F
:1021900020393130005043545045004252494447A1
:1021A0004500414253004849505300504C410043C0
:1021B0007573746F6D2054656D70004D61696E00AC
:1021C00054474C41534520436F6E6600504F4C5965
:1021D0004341524220436F6E66004C41594252497E
:1021E000434B20436F6E66004E2D56454E542043A0
:1021F0006F6E6600414C4C4F592039313020436F8F
:102200006E6600504354504520436F6E6600425244
:102210004944474520436F6E660041425320436F57
:102220006E66004849505320436F6E6600504C4123
:1022300020436F6E66005049442D43005049442DA1
:1022400043005049442D44005049442D4400504916
:10225000442D49005049442D49005049442D500017
:102260005049442D50002002204661637400200232
:102270002046616374002002204D61780020022016
:102280004D6178002002204D696E002002204D69CA
:102290006E004F6666004F6E20004F6666004F6E00
:1022A00020004175746F74656D700046616E207317
:1022B000706565640046616E2073706565640042F8
:1022C000656400426564004E6F7A7A6C65004E6FFB
:1022D0007A7A6C650054656D7065726174757265AB
:1022E0000053746F7265206D656D6F727900426581
:1022F0006400426564004E6F7A7A6C65004E6F7AB6
:102300007A6C650046616E20737065656400466195
:102310006E20737065656400437573746F6D20542F
:10232000656D700053746F7265206D656D6F7279A5
:102330000042656400426564004E6F7A7A6C650005
:102340004E6F7A7A6C650046616E207370656564C5
:102350000046616E20737065656400437573746F29
:102360006D2054656D700053746F7265206D656DDE
:102370006F72790042656400426564004E6F7A7A3C
:102380006C65004E6F7A7A6C650046616E207370E2
:102390006565640046616E20737065656400437511
:1023A00073746F6D2054656D700053746F72652087
:1023B0006D656D6F72790042656400426564004E20
:1023C0006F7A7A6C65004E6F7A7A6C650046616E42
:1023D0002073706565640046616E20737065656486
:1023E00000437573746F6D2054656D700053746F86
:1023F0007265206D656D6F7279004265640042659B
:1024000064004E6F7A7A6C65004E6F7A7A6C650064
:1024100046616E2073706565640046616E2073705E
:1024200065656400437573746F6D2054656D70004D
:1024300053746F7265206D656D6F727900426564CB
:1024400000426564004E6F7A7A6C65004E6F7A7A4E
:102450006C650046616E2073706565640046616E50
:1024600020737065656400437573746F6D205465E7
:102470006D700053746F7265206D656D6F727900B9
:1024800042656400426564004E6F7A7A6C65004E66
:102490006F7A7A6C650046616E20737065656400C2
:1024A00046616E20737065656400437573746F6D6B
:1024B0002054656D700053746F7265206D656D6F8B
:1024C00072790042656400426564004E6F7A7A6CEE
:1024D00065004E6F7A7A6C650046616E2073706598
:1024E00065640046616E20737065656400437573B2
:1024F000746F6D2054656D700053746F7265206D3C
:10250000656D6F72790042656400426564004E6FCC
:102510007A7A6C65004E6F7A7A6C650046616E203F
:1025200073706565640046616E2073706565640054
:10253000437573746F6D2054656D700053746F72C2
:1025400065206D656D6F7279004265640042656457
:10255000004E6F7A7A6C65004E6F7A7A6C65004631
:10256000616E2073706565640046616E20737065EE
:10257000656400437573746F6D2054656D70004D14
:102580006F76652041786973004732380041757471
:102590006F20486F6D65004D383400446973616287
:1025A0006C65205374657070657273004D61696E5F
:1025B000004D6F766520302E316D6D004D6F766564
:1025C00020316D6D004D6F76652031306D6D004DA1
:1025D0006F76656D656E74004578747275646572AA
:1025E000004D6F7665205A004D6F76652059004D7D
:1025F0006F76652058004D6F7665204178697300CD
:102600004578747275646572005A00590058004D1F
:10261000363030004368616E67652066696C616DB5
:10262000656E7400466C6F7700466C6F770046618C
:102630006E2073706565640046616E207370656519
:10264000640042656400426564004E6F7A7A6C658E
:10265000004E6F7A7A6C6500537065656400537044
:10266000656564004D61696E004361726420726546
:102670006D6F766564004361726420696E73657284
:10268000746564000000000000000000000000000D
:10269000000000000000000000000000000000003A
:1026A000000000000000000C000000000000000C12
:1026B00000000000000000120000000000000023E5
:1026C0000000000000000021000000000000004C9D
:1026D000800000000000005E80000000000000920A
:1026E00040000000000000A14000000000000121A7
:1026F000200000000000027F9000000000000200A7
:1027000010000000000007FFF800000000000400B7
:10271000080000000000080004000000000008009D
:102720000600000000001000020000000000301E43
:10273000010000000000207F81000000000041FF38
:10274000E0800000000043FCF08000000000873BB8
:102750007840000000018EDBFC60000000010FEB00
:10276000CC20000000021FEDB610000000021FDEAA
:10277000B6100000000439CD7F080000000436E0E8
:10278000FF08000000087EC0BB84000000187F0026
:102790005D86000000107FC0ED82000000203CC07C
:1027A0007301000000203B337F01000000701BE735
:1027B0007E03800000C81DEEDE04C00000880FDE2E
:1027C000DC04400001240FDF3C092000012607DB68
:1027D000F8192000027203E7F0139000025101FF84
:1027E000E02290000489007F802448000904801EB4
:1027F000004824000BFE400000DFF4001000400001
:10280000008002001FFFFFFFFFFFFE00000000002E
:1028100000000000000000000000000000000000B8
:10282000000000001022103C3C0E1F00102210047B
:102830002211040010221008221104001022100896
:102840003C1104001022101022110400102210204C
:10285000221104001E1C1E3C3C0E0400000000005F
:102860000000000000000000000000000000000068
:102870000000000000000000000000000000000058
:102880000000000000000000000000000000000048
:102890000000000000000000000000000000000038
:1028A0000000000000000000000000000000000028
:1028B0000000000000000000000000000000000018
:1028C00000006563686F3A0048617264636F646515
:1028D000642044656661756C742053657474696E18
:1028E0006773204C6F616465640053746F72656434
:1028F0002073657474696E6773207265747269659C
:10290000766564002044002049002020204D3330AB
:10291000312050005049442073657474696E6773A8
:102920003A00205A0020590020204D3230362058DD
:1029300000486F6D65206F666673657420286D6D45
:10294000293A00204500205A00205800204200204B
:10295000540020204D323035205300416476616EA2
:10296000636564207661726961626C65733A2053B5
:102970003D4D696E20666565647261746520286DE1
:102980006D2F73292C20543D4D696E207472617631
:10299000656C20666565647261746520286D6D2FB5
:1029A00073292C20423D6D696E696D756D207365CC
:1029B000676D656E742074696D6520286D73292CB0
:1029C00020583D6D6178696D756D205859206A6594
:1029D000726B20286D6D2F73292C20205A3D6D615C
:1029E00078696D756D205A206A65726B20286D6D4F
:1029F0002F73292C2020453D6D6178696D756D2000
:102A000045206A65726B20286D6D2F732900205454
:102A10000020204D323034205300416363656C65E3
:102A2000726174696F6E3A20533D616363656C65D2
:102A3000726174696F6E2C20543D726574726163AB
:102A40007420616363656C65726174696F6E0020E8
:102A50004500205A0020590020204D3230312058A6
:102A6000004D6178696D756D20416363656C6572B9
:102A70006174696F6E20286D6D2F7332293A0020C2
:102A80004500205A0020590020204D323033205874
:102A9000004D6178696D756D20666565647261745D
:102AA000657320286D6D2F73293A00204531002071
:102AB0004500205A0020590020204D39322058006E
:102AC00053746570732070657220756E69743A0076
:102AD00053657474696E67732053746F7265640014
:102AE0006563686F3A004572726F723A0053544FD3
:102AF000505045442E20005072696E7465722073E8
:102B0000746F707065642064756520746F206572E1
:102B1000726F72732E204669782074686520657222
:102B2000726F7220616E6420757365204D3939397A
:102B300020746F20726573746172742E202854653E
:102B40006D7065726174757265206973207265734A
:102B500065742E20536574206974206166746572F3
:102B60002072657374617274696E6729004B494CF9
:102B70004C45442E20005072696E74657220686165
:102B80006C7465642E206B696C6C28292063616C01
:102B90006C656421006F6B00526573656E643A204A
:102BA000002200556E6B6E6F776E20636F6D6D61E6
:102BB0006E643A2022004368616E67652066696C26
:102BC000616D656E74006C636420636F6E74726116
:102BD00073742076616C75653A20007A5F6D696E5A
:102BE0003A2000795F6D696E3A2000785F6D696EFA
:102BF0003A20005A3A00593A0020436F756E74200B
:102C0000583A2000453A005A3A00593A00583A00DA
:102C10004649524D574152455F4E414D453A4D61EF
:102C2000726C696E2056313B20537072696E746508
:102C3000722F6772626C206D617368757020666FA9
:102C4000722067656E36204649524D574152455FA6
:102C500055524C3A687474703A2F2F7777772E6DEF
:102C6000656E64656C2D70617274732E636F6D2078
:102C700050524F544F434F4C5F56455253494F4E5D
:102C80003A312E30204D414348494E455F5459500A
:102C9000453A54415A2045585452554445525F4391
:102CA0004F554E543A3120555549443A3030303022
:102CB000303030302D303030302D303030302D301D
:102CC0003030302D30303030303030303030303007
:102CD0000A0054415A204F66662E0054415A205231
:102CE000656164792E0042656420646F6E652E0014
:102CF00020423A0020453A00543A00426564204898
:102D0000656174696E672E0048656174696E67203D
:102D1000646F6E652E0020573A0020453A00543A01
:102D20000048656174696E672E2E2E002042403A7D
:102D30000020403A00202F003A00205400202F00AD
:102D400020423A00202F006F6B20543A0025692062
:102D50006D696E2C2025692073656300456E6420C3
:102D600066696C65206C69737400426567696E20E2
:102D700066696C65206C697374004E6F206D6F76A8
:102D8000652E00526573756D696E67207072696E8D
:102D900074005761697420666F7220757365722EB6
:102DA0002E2E00536C6565702E2E2E00000095436C
:102DB0000080894300007A43FFFFFF00000000000D
:102DC0000000000000000000000000000000000003
:102DD000000000000095430080894300007A430012
:102DE00000A0400000A04000008040256920686FDE
:102DF000757273202569206D696E75746573004462
:102E00006F6E65207072696E74696E672066696C9A
:102E1000650053544F505045442E20005072696E47
:102E20007465722073746F707065642064756520BA
:102E3000746F206572726F72732E204669782074E9
:102E40006865206572726F7220616E6420757365AB
:102E5000204D39393920746F207265737461727432
:102E60002E202854656D70657261747572652069D5
:102E7000732072657365742E205365742069742005
:102E800061667465722072657374617274696E67CD
:102E900029006F6B004E6F204C696E65204E756D7A
:102EA000626572207769746820636865636B737507
:102EB0006D2C204C617374204C696E653A20004E75
:102EC0006F20436865636B73756D20776974682044
:102ED0006C696E65206E756D6265722C204C617335
:102EE00074204C696E653A2000636865636B737586
:102EF0006D206D69736D617463682C204C6173740F
:102F0000204C696E653A20004C696E65204E756DE7
:102F1000626572206973206E6F74204C6173742037
:102F20004C696E65204E756D6265722B312C204C9C
:102F3000617374204C696E653A20004D3131300068
:102F4000446F6E6520736176696E672066696C6593
:102F50002E006F6B004D3239002020506C616E6E78
:102F6000657242756666657242797465733A2000CF
:102F70002046726565204D656D6F72793A2000417B
:102F80007567203235203230313500436F6D7069FE
:102F90006C65643A200028416C657068204F626A55
:102FA000656374732C20496E632C2054415A202091
:102FB000636F6E6669672900207C20417574686FB5
:102FC000723A200041756720323520323031352089
:102FD00031323A34393A353100204C61737420551E
:102FE0007064617465643A2000312E302E30004DDB
:102FF00061726C696E200020536F66747761726530
:1030000020526573657400205761746368646F674C
:10301000205265736574002042726F776E206F7561
:1030200074205265736574002045787465726E6112
:103030006C20526573657400506F7765725570002F
:103040007374617274002200656E717565696E67D4
:103050002022002200656E717565696E672022006E
:103060007C3C3E5E2B3D3F2F5B5D3B2C2A225C006F
:103070004572726F723A004572723A204D4158544F
:10308000454D50204245440054656D706572617431
:10309000757265206865617465642062656420737B
:1030A00077697463686564206F66662E204D4158A9
:1030B00054454D50207472696767657265642021BC
:1030C00021004572723A204D494E54454D50003A08
:1030D00020457874727564657220737769746368CB
:1030E0006564206F66662E204D494E54454D502034
:1030F0007472696767657265642021004572723A6F
:10310000204D415854454D50003A20457874727511
:10311000646572207377697463686564206F66669E
:103120002E204D415854454D502074726967676593
:10313000726564202100202D20496E76616C6964DF
:10314000206578747275646572206E756D62657243
:103150002021001000AD0330016A0150022B0170E4
:10316000030A019004F500B005E500D006D800F090
:1031700007CE001009C500300ABE00500BB7007022
:103180000CB100900DAB00B00EA600D00FA200F065
:10319000109D001012990030139500501492007089
:1031A000158E0090168B00B0178700D0188400F0A1
:1031B000198100101B7E00301C7B00501D790070AF
:1031C0001E7600901F7300B0207000D0216E00F0BA
:1031D000226B0010246900302566005026630070C1
:1031E00027610090285E00B0295C00D02A5900F0C9
:1031F0002B5600102D5400302E5100502F4E0070D1
:10320000304B0090314800B0324500D0334200F0DE
:10321000343E0010363B00303737005038330070F2
:10322000392E00903A2900B03B2300D03C1B00F01F
:103230003D1100103F0100F03F0000504944204183
:1032400075746F74756E652066696E697368656400
:10325000212050757420746865204B702C204B69B8
:1032600020616E64204B6420636F6E7374616E74B2
:103270007320696E746F20436F6E66696775726143
:1032800074696F6E2E6800504944204175746F74E4
:10329000756E65206661696C6564212074696D6571
:1032A0006F75740020403A006F6B20543A006F6BCA
:1032B00020423A00504944204175746F74756E6520
:1032C000206661696C6564212054656D706572616A
:1032D0007475726520746F6F206869676800204B91
:1032E000643A2000204B693A2000204B703A2000BD
:1032F00020436C6173696320504944200020547559
:103300003A2000204B753A2000206D61783A200069
:10331000206D696E3A200020643A200020626961C5
:10332000733A20001000C90210012C014001220153
:1033300070011801B0010E01F00104015002FA0001
:10334000B002F0003003E600D003DC009004D200AD
:103350007005C800A006BE000008B400B009AA00AD
:10336000D00BA000600E960060118C00001582004A
:1033700020197800C01D6E00A0226400B0275A00FA
:10338000902C500000314600E0343C0010383200F0
:10339000903A2800603C1E00A03D1400803E0A00C8
:1033A000203F00004D383420582059205A20450035
:1033B0006563686F3A0043616E6E6F7420656E746A
:1033C0006572207375626469723A20004D32340070
:1033D0004D3233202573006175746F25692E6700A7
:1033E0004572726F723A006572726F7220777269FD
:1033F00074696E6720746F2066696C65004E6F7427
:10340000205344207072696E74696E67002F0053F8
:1034100044207072696E74696E67206279746520E9
:10342000002E0044656C6574696F6E206661696C7E
:1034300065642C2046696C653A200046696C6520FD
:1034400064656C657465643A002E006F70656E206B
:103450006661696C65642C2046696C653A2000578A
:10346000726974696E6720746F2066696C653A20B2
:10347000002E006F70656E206661696C65642C209B
:1034800046696C653A20002E006F70656E2066619B
:10349000696C65642C2046696C653A200046696C4D
:1034A000652073656C6563746564002053697A6593
:1034B0003A200046696C65206F70656E65643A203D
:1034C000002E006F70656E206661696C65642C204B
:1034D00046696C653A20004E6F77206672657368A6
:1034E0002066696C653A20004E6F7720646F696EC4
:1034F000672066696C653A20002220706F73002295
:1035000020706172656E743A2200535542524F55D5
:1035100054494E452043414C4C2074617267657498
:103520003A2200747279696E6720746F2063616C4F
:103530006C207375622D67636F64652066696C65C6
:1035400073207769746820746F6F206D616E7920C5
:103550006C6576656C732E204D4158206C657665E0
:103560006C2069733A0053442063617264206F6B6E
:10357000006F70656E526F6F74206661696C656470
:1035800000766F6C756D652E696E69742066616971
:103590006C656400534420696E6974206661696CCF
:1035A000006563686F3A0020746F6F206C6F6E6700
:1035B00020657874727573696F6E207072657665B8
:1035C0006E7465640020636F6C6420657874727536
:1035D00073696F6E2070726576656E746564000144
:1035E000050800FF060121023520FFFF07FF06FF47
:1035F000090050221656808080800080153353A029
:10360000A0A00257575050F850F85050025757207A
:1036100070A07028702013355580A040A02002476C
:103620005740A0A040A0A0502513538080801226B0
:103630005640808080804012265680404040408026
:103640000245559060F060900255552020F82020EA
:10365000113353604080044151F011335340E04036
:1036600002465610102040808012365640A0A0A07E
:10367000A04012365640C0404040E002465660909E
:10368000106080F0024656F02060109060024656AE
:103690002060A0F02020024656F080E010906002EA
:1036A00046566080E0909060024656F01020204020
:1036B000400246566090609090600246566090903E
:1036C000701060122555C0C000C0C0113656606031
:1036D00000604080123656204080804020034353D3
:1036E000F000F012365680402020408012365640BE
:1036F000A020400040015858304898A8A890403079
:10370000024656609090F09090024656E090E0900D
:1037100090E0024656609080809060024656E090AD
:10372000909090E0024656F080E08080F00246568D
:10373000F080E0808080024656609080B090600209
:1037400046569090F0909090123656E0404040409F
:10375000E002465670202020A04002465690A0C0AD
:10376000A0A0900246568080808080F0024656904D
:10377000F0F090909002465690D0F0B0B090024693
:1037800056609090909060024656E09090E0808065
:10379000014757609090D0B06010024656E090907C
:1037A000E09090024656609040209060123656E0BD
:1037B00040404040400246569090909090600246B3
:1037C00056909090906060024656909090F0F090E5
:1037D000024656909060609090025656888850201D
:1037E0002020024656F010204080F0123656E0802D
:1037F000808080E0024656808040201010123656AD
:10380000E020202020E016325240A0014151F01665
:10381000225280400244547090907002465680803C
:10382000E09090E0123454608080600246561010A0
:103830007090907002445460B0C0600246562050B0
:1038400040E040400145556090701060024656804F
:1038500080E09090901236564000C04040E0113712
:10386000572000202020A040024656808090E09003
:1038700090123656C040404040E0025454D0A8A8B0
:10388000A8024454E09090900244546090906001EB
:103890004555E090E0808001455570907010100211
:1038A0004454A0D0808012345460C020C0024656D8
:1038B0004040E040502002445490909070123454A4
:1038C000A0A0A04002545488A8A85002445490607C
:1038D00060900145559090709060024454F02040F3
:1038E000F0024757304020C02040302216568080DA
:1038F00080808080024757C02040304020C0064270
:103900005250A0FFFFFFFFFFFFFFFFFFFFFFFFFF82
:10391000FFFFFFFFFFFFFFFFFFFFFFFFFFFFFFFFB7
:10392000FFFFFFFF09005022165680008080808034
:103930000146562070A0A070200246562050E0405C
:1039400050A002555588705070880256568850F81D
:1039500020F82022175780808000808080024757FF
:103960007080E0907010E0173151A002565670A898
:10397000C8C8A87014355560A06000E003435350D8
:10398000A050123353E02020143151E002565670FB
:10399000E8D8E8D870173151E015335340A04012F1
:1039A000355540E04000E014355540A02040E0147B
:1039B0003555C020C020C016225240800145559088
:1039C0009090E08002565678E8E868282824115143
:1039D00080112252408014355540C04040E01435DB
:1039E0005540A04000E0034353A050A00247578039
:1039F0008080A060F0200247578080A0D010207007
:103A000002475780408060A0F020123656400040A8
:103A100080A04002475740206090F09090024757A6
:103A200020406090F0909002475760906090F09036
:103A30009002475750A06090F09090024757900036
:103A40006090F0909002475760906090F0909002E4
:103A5000465670A0A0F0A0B00147576090808090BB
:103A600060400247574020F080E080F00247572036
:103A700040F080E080F00247576090F080E080F0F6
:103A80000247579000F080E080F01237578040E006
:103A9000404040E01237572040E0404040E01237BD
:103AA0005740A0E0404040E0123757A000E04040BF
:103AB00040E00256567048E848487002475750A008
:103AC00090D0B09090024757402060909090600254
:103AD00047572040609090906002475760906090F8
:103AE00090906002475750A06090909060024757B6
:103AF00090006090909060123353A040A002465610
:103B000070B0B0D0D0E002475740209090909060C5
:103B100002475720409090909060024757609090E5
:103B2000909090600247579000909090906002575C
:103B3000571020885020202002465680E09090E0C8
:103B4000800246566090A0A090A0024757402000F7
:103B5000709090700247572040007090907002471C
:103B6000572050007090907002475750A0007090FE
:103B700090700246565000709090700247576090C7
:103B80006070909070025454F068B07811355560B0
:103B90008080604002475740200060B0C06002470C
:103BA0005720400060B0C06002475760900060B08E
:103BB000C060024656500060B0C060123757804067
:103BC00000C04040E0123757204000C04040E012A3
:103BD000375740A000C04040E0123656A000C04019
:103BE00040E0024757A040A0107090600247575035
:103BF000A000E090909002475740200060909060B5
:103C00000247572040006090906002475760900044
:103C10006090906002475750A0006090906002460C
:103C2000569000609090601235554000E0004002D0
:103C3000445470B0D0E002475740200090909070FC
:103C400002475720400090909070024757609000C4
:103C50009090907002465690009090907001485855
:103C600020400090907090600147578080E090E085
:103C70008080014757900090907090600000210074
:103C8000240027002A002D0030003300010100002D
:103C9000040107010A0100002200250028002B0072
:103CA0002E003100340002010000050108010B0163
:103CB000000020002300260029002C002F003200E5
:103CC00000010000030106010901050505050705BE
:103CD00008080808020202020A0A08080404040488
:103CE00001010101010101010303030303030303B4
:103CF000040707070C0C0C0C0C0C0C0C0202020243
:103D000006060606060606060B0B0B0B0B0B0B0B2B
:103D100007070A0A0A0A0A0A050505040102102013
:103D200020080810204010204080020102010804F1
:103D30000201010204081020408080402010080485
:103D400002018004020180402010080402010804DE
:103D50000201010204081020408001020408102022
:103D600040801008040880102040044080100000AB
:103D7000090A02080B0C0D070603040100000000ED
:103D80000000000000000000000000000000000033
:103D90000000000000000000000011100F000000F3
:103DA0000000000000000000000000000000000013
:103DB0000000000002494E46494E4954594E414EBA
:103DC000CDCCCC3D0AD7233C17B7D13877CC2B329A
:103DD0009595E6241FB14F0A000020410000C8421B
:103DE00000401C4620BCBE4CCA1B0E5AAEC59D747A
:103DF0000D94D8050D94F6050D9408060D944F0604
:103E00000D943D080D94E1050D941F060D94461187
:103E10000D944C0A0D9407060D94DC0D702FBF8491
:103E2000A79DFC1EA29D11241FBECFEFD1E2DEBFD5
:103E3000CDBF00E00CBF14E0A0E0B2E0E8E4F5E3A1
:103E400002E00BBF02C007900D92AC3BB107D9F75F
:103E50001BBE15E1ACEBB4E001C01D92AE3FB10753
:103E6000E1F71EE3C4E2DEE304C02297FE010F94F3
:103E70004A1ACC31D107C9F70F9496110D94981AAC
:103E80000C940000A0E0B0E0E8E4FFE10D94671AB4
:103E9000EC015B016115710519F0FB0191838083D1
:103EA000F9908F2D90E00F944E1A892BC9F7FDE2FF
:103EB000FF1621F4F990EE24E39405C02BE2F216EC
:103EC00009F4F990EE248E0101501040C80165EB11
:103ED0007DE343E050E072D2892BF9F48E010E5F4E
:103EE0001F4FC80168EB7DE345E050E067D2892BA6
:103EF00019F48E01095F1F4FA114B10419F0F501E7
:103F000011830083E0FC04C070E090E080E813C0FF
:103F100070E090E080E86FEF07C1C8016DEB7DE3D2
:103F200043E050E04BD2892B69F4A114B10429F489
:103F300070E090E080EC6FE7F7C02296F501D18346
:103F4000C083F6CF8824992440E050E060E070E020
:103F5000EF2DE053EA30A0F5F2E0EF2A8E2D90E04D
:103F60009C0128703070E2FE06C0232B79F508947E
:103F7000811C911C2BC0232B19F0089481089108F7
:103F8000DB01CA0112E0880F991FAA1FBB1F1A95F7
:103F9000D1F7480F591F6A1F7B1F440F551F661F1B
:103FA000771F4E0F511D611D711D483929E95207B8
:103FB00029E9620729E1720748F084E0E82A06C08F
:103FC000EE3F31F4E3FC39C098E0E92AF990C0CF24
:103FD000E53311F0E53189F529912D3219F4E0E14D
:103FE000EE2A05C02B3219F081E090E003C0299140
:103FF00082E090E0E22FE053EA3018F0C81BD90BC2
:104000001CC020E030E0FCE020383F075CF4C90130
:10401000880F991F880F991F280F391F220F331FF0
:104020002E0F311DE991E053EA3068F3E4FE03C03E
:10403000309521953F4F820E931ECE2CDD24E1FE5C
:1040400007C0A114B10421F02197F501D183C083E9
:10405000CB01BA010F94B3167B018C01F3E0CF22A0
:10406000DD2423E0C216D10421F417FB109517F9C3
:10407000109557016801C801B70120E030E040E029
:1040800050E00F941316882309F44AC097FE0DC020
:1040900024EDE22E2DE3F22E9094819491089394D6
:1040A000C0E2D0E000E010E012C09CEEE92E9DE3FB
:1040B000F92EF6CFF7012591359145915491C6011E
:1040C000B5010F94F3185B016C018C1A9D0A8C16D4
:1040D0009D0684F7D595C7950F5F1F4F06301105D4
:1040E00029F08CEF9FEFE80EF91EF1CFC501D60144
:1040F0007C018D018C2D880F8D2D881F8F3F51F0F5
:10410000C601B50120E030E040E050E00F94131606
:10411000882331F482E290E09093FD158093FC15A2
:104120007E2D9F2D802F612F272F392F482F562F1F
:10413000B901CA01CDB7DEB7ECE00D94831A2F9216
:104140003F925F926F927F928F929F92AF92BF92B7
:10415000CF92DF92EF92FF920F931F93CF93DF9353
:104160008C011B01EA016115710519F0FB019183B6
:104170008083209749F0CE010297839728F020E0B2
:1041800030E040E050E0F6C0F801A1908F018A2DA8
:1041900090E00F944E1A892BB9F7FDE2AF1631F477
:1041A000F801A1908F015524539407C0FBE2AF168C
:1041B00019F4F801A1908F015524209719F0C0310E
:1041C000D105C1F4F0E3AF1679F4F80180818837A6
:1041D00011F0883549F4F801A1800E5F1F4FF2E01D
:1041E0005F2AC0E1D0E006C0209721F480E3A81642
:1041F000E9F427C0C830D10531F1C930D10524F424
:10420000C230D10531F50CC0CA30D10589F0C031BA
:10421000D105F9F4C12CD12CE12CB8E0FB2E28C03B
:10422000C12CD12CE12CA0E4FA2E22C0CAE0D0E0AF
:10423000FCECCF2EFCECDF2EFCECEF2EFCE0FF2E96
:1042400017C0C8E0D0E0C12CD12CE12CE0E1FE2E5B
:104250000FC09E01442737FD4095542F60E070E069
:1042600080E090E80F940B1AC901DA016C017D011E
:1042700020E030E040E050E060E03E01882477FC40
:104280008094982C70EDB72EBA0CE9E0EB1570F421
:104290008A2D81548A3118F499ECB92E06C08A2DE2
:1042A00081568A3150F589EAB82EBA0C8B2D90E0F0
:1042B0008C179D0714F56F3FE1F0C216D306E40694
:1042C000F506B0F0CA01B901A40193010F94C51914
:1042D0009B01AC012B0D311D411D511D2130F0E022
:1042E0003F07F0E04F07F0E85F0710F461E001C01E
:1042F0006FEFF801A1908F01C5CF2114310481F037
:10430000662331F001501040F1011183008308C091
:1043100051FE1AC002501040F1011183008314C0F5
:1043200067FF12C050FC05C02FEF3FEF4FEF5FE774
:1043300004C020E030E040E050E882E290E090935A
:10434000FD158093FC1516C050FE08C05095409591
:10435000309521953F4F4F4F5F4F0CC057FF0AC01C
:1043600082E290E09093FD158093FC152FEF3FEFD4
:104370004FEF5FE7B901CA01DF91CF911F910F9114
:10438000FF90EF90DF90CF90BF90AF909F908F9075
:104390007F906F905F903F902F900895FB01DC011C
:1043A00005900D920020E1F70895FC010590002092
:1043B000E9F7809590958E0F9F1F0895FB01DC0112
:1043C0004150504088F08D9181341CF08B350CF4B5
:1043D000805E659161341CF06B350CF4605E861B69
:1043E000611171F3990B0895881BFCCFFB01DC016F
:1043F0004150504048F005900D920020C9F701C08F
:104400001D9241505040E0F70895FB01559155230E
:10441000A9F0BF01DC014D9145174111E1F759F4B5
:10442000CD010590002049F04D9140154111C9F38F
:10443000FB014111EFCF81E090E001970895FB016E
:10444000DC0104C08D910190801921F4415050404D
:10445000C8F7881B990B0895FB01DC0102C001908D
:104460000D9241505040D8F70895FB01DC010D90AA
:104470000020E9F7119701900D920020E1F70895CF
:10448000FC018191861721F08823D9F79927089597
:104490003197CF010895FB01DC0101900D920020BE
:1044A000E1F70895FB01DC014150504030F08D915F
:1044B0000190801919F40020B9F7881B990B089511
:1044C000FB01DC014150504048F001900D9200206A
:1044D000C9F701C01D9241505040E0F70895AEE089
:1044E000B0E0E5E7F2E20D946F1A0E891F898EE0C5
:1044F0008C831A8309838FEF9FE79E838D839E01B0
:10450000265E3F4FCE010196688D798DA9010AD0B4
:104510002F813885020F131FF80110822E96E4E0D8
:104520000D948B1AABE0B0E0E8E9F2E20D94611A69
:104530003C012B015A01FC0117821682838181FD07
:1045400003C06FEF7FEFB9C19AE0892E1E01089476
:10455000211C311CF3012381F20123FD859123FFEE
:1045600081912F01882309F4A5C1853239F423FDF7
:10457000859123FF81912F01853221F490E0B301D1
:10458000B7D1E8CF982FFF24EE249924FFE1FF153F
:10459000D0F09B3269F09C3228F4903259F093327B
:1045A00091F40EC09D3249F0903369F441E024C08B
:1045B00052E0F52A84E0F82A28C098E0F92A25C0BC
:1045C000E0E1FE2A22C0F7FC29C0892F80538A30FF
:1045D00070F4F6FE05C0989C902C1124980E15C01E
:1045E000E89CE02C1124E80EF0E2FF2A0EC09E3277
:1045F00029F4F6FC5FC140E4F42A07C09C3619F4A4
:1046000050E8F52A02C0983649F4F20123FD95914D
:1046100023FF91912F01992309F0B8CF892F855459
:10462000833018F08052833038F444E050E0A40E18
:10463000B51E5FE359830FC0933631F0933779F09D
:10464000933509F052C01FC0F5018081898342E093
:1046500050E0A40EB51E610101E010E011C0F501AB
:10466000C080D180F6FC03C06FEF7FEF02C0692DE0
:1046700070E042E050E0A40EB51EC6012ED18C01C0
:104680005FE7F52213C0F501C080D180F6FC03C0BE
:104690006FEF7FEF02C0692D70E042E050E0A40EA2
:1046A000B51EC6010FD18C0150E8F52AF3FE06C0F5
:1046B00018C080E290E0B3011BD1EA948E2D90E007
:1046C00008171907B0F30DC0F601F7FC8591F7FE46
:1046D00081916F0190E0B3010BD1E110EA94015098
:1046E00010400115110581F7E2C0943611F099369A
:1046F00061F5F7FE08C0F5012081318142815381C7
:1047000084E090E00AC0F501808191819C014427FA
:1047100037FD4095542F82E090E0A80EB91E9FE629
:10472000F92257FF09C050954095309521953F4F8C
:104730004F4F5F4FE0E8FE2ACA01B901A1012AE00C
:1047400030E002D1D82ED2183FC0953729F41F2D62
:104750001F7E2AE030E01DC01F2D197F9F3661F0BB
:10476000903720F4983509F0A5C00FC0903739F084
:10477000983709F09FC004C028E030E00AC01061FB
:1047800014FD146020E130E004C014FD166020E147
:1047900032E017FF08C0F501608171818281938149
:1047A00044E050E008C0F50180819181BC0180E0C7
:1047B00090E042E050E0A40EB51EA101C5D0D82E75
:1047C000D2188FE7F82EF122F6FE0BC05EEFF5222D
:1047D000D91438F4F4FE07C0F2FC05C08FEEF822BD
:1047E00002C01D2D01C0192DF4FE0DC0FE01ED0DFE
:1047F000F11D8081803319F499EEF92208C01F5F02
:10480000F2FE05C003C08F2D867809F01F5F0F2DC3
:10481000F3FC13C0F0FE0EC01E1510F09D2C0AC054
:104820009D2C9E0C911A1E2D05C080E290E0B301D4
:104830005FD01F5F1E15C8F304C01E1510F4E11AE7
:1048400001C0EE2404FF0EC080E390E0B30150D01D
:1048500002FF1BC001FD03C088E790E00EC088E5A1
:1048600090E00BC0802F867881F001FF02C08BE2C0
:1048700001C080E2F7FC8DE290E0B30139D005C0C1
:1048800080E390E0B30134D09A94D914C8F3DA9459
:10489000F101ED0DF11D808190E0B30129D0DD2003
:1048A000B1F705C080E290E0B30122D0EA94EE2097
:1048B000C9F750CEF30166817781CB012B96E2E1F7
:1048C0000D947D1AFC010590615070400110D8F7DD
:1048D000809590958E0F9F1F0895FC016150704048
:1048E00001900110D8F7809590958E0F9F1F089525
:1048F0000F931F93CF93DF938C01EB018B8181FF8B
:104900001BC082FF0DC02E813F818C819D812817A5
:10491000390764F4E881F9810193F983E88306C0DB
:10492000E885F985802F1995892B31F48E819F8137
:1049300001969F838E8302C00FEF1FEFC801DF91A6
:10494000CF911F910F910895FA01AA27283051F1B4
:10495000203181F1E8946F936E7F6E5F7F4F8F4FB0
:104960009F4FAF4FB1E03ED0B4E03CD0670F781F0F
:10497000891F9A1FA11D680F791F8A1F911DA11DF4
:104980006A0F711D811D911DA11D20D009F468942D
:104990003F912AE0269F11243019305D3193DEF6D5
:1049A000CF010895462F4770405D4193B3E00FD08B
:1049B000C9F7F6CF462F4F70405D4A3318F0495D76
:1049C00031FD4052419302D0A9F7EACFB4E0A69559
:1049D0009795879577956795BA95C9F7009761057B
:1049E000710508959B01AC010A2E069457954795D1
:1049F00037952795BA95C9F7620F731F841F951FC6
:104A0000A01D08951092F0041092F2041092F40484
:104A1000089580938D030895EFE6F0E08081826031
:104A2000808308951F93FC011FB7F89480819181C2
:104A3000A281B3818093CA049093CB04A093CC0449
:104A4000B093CD04FB0180819181A281B3818093D9
:104A5000CE049093CF04A093D004B093D104FA0174
:104A600080819181A281B3818093D2049093D304F9
:104A7000A093D404B093D504F90180819181A281DF
:104A8000B3818093D6049093D704A093D804B093B5
:104A9000D9041FBF1F910895FC012FB7F89480819E
:104AA0009181A281B3818093D6049093D704A0937F
:104AB000D804B093D9042FBF0895E82F8FB7F89486
:104AC000F0E0EE0FFF1FEE0FFF1FE653FB4F2081BC
:104AD0003181428153818FBFB901CA01089580910C
:104AE0006F008D7F80936F0006C08091ED148F5F03
:104AF0008F708093ED149091EC148091ED149817C1
:104B000051F41092BD041092BC0480916F00826039
:104B100080936F0008959091EC148091ED14981794
:104B200051F3E3CFE5E4F1E0949108C08091C00037
:104B300085FFFCCF9093C600319694919923B1F7ED
:104B4000E1E4F1E0949108C08091C00085FFFCCFC2
:104B50009093C600319694919923B1F788E20F940F
:104B60001711BC0188E895E04AE050E00E945830F7
:104B700089E20F941711BC0188E895E04AE050E003
:104B80000E9458308091C00085FFFCCF8AE080935E
:104B9000C600EDE3F1E0949108C08091C00085FF6C
:104BA000FCCF9093C600319694919923B1F785E498
:104BB0000F941711BC0188E895E04AE050E00E948C
:104BC000583087E20F941711BC0188E895E04AE05D
:104BD00050E00E9458308091C00085FFFCCF8AE0F1
:104BE0008093C600E9E3F1E0949108C08091C00091
:104BF00085FFFCCF9093C600319694919923B1F72D
:104C000084E40F941711BC0188E895E04AE050E075
:104C10000E94583083E40F941711BC0188E895E096
:104C20004AE050E00E9458308091C00085FFFCCFE0
:104C30008AE08093C600E4E3F1E0949108C080919B
:104C4000C00085FFFCCF9093C600319694919923C4
:104C5000B1F781E40F941711BC0188E895E04AE0B0
:104C600050E00E94583082E40F941711BC0188E88C
:104C700095E04AE050E00E9458308091C00085FFE6
:104C8000FCCF8AE08093C600EFE2F1E0949108C087
:104C90008091C00085FFFCCF9093C600319694911F
:104CA0009923B1F78FE30F941711BC0188E895E0C1
:104CB0004AE050E00E94583080E40F941711BC0184
:104CC00088E895E04AE050E00E9458308091C000AA
:104CD00085FFFCCF8AE08093C60008950F931F9351
:104CE000182F042F67FD19C0823081F0833028F41B
:104CF000882341F0813089F407C0833049F0843043
:104D000061F408C088E207C085E405C084E403C0FC
:104D100081E401C08FE30F94E51007FD1AC0123043
:104D200081F0133028F4112341F0113091F407C0C1
:104D3000133049F0143069F408C089E207C087E2F3
:104D400005C083E403C082E401C080E4602F0F94B7
:104D5000E5101F910F910895643089F0653028F4B3
:104D6000613041F0623099F407C0683051F0603131
:104D700071F40AC060E001C061E040E004C060E09E
:104D800001C061E041E0AACF61E041E0A7CF089512
:104D90000F931F93182F062F86E260E00F94E51003
:104DA0001EBD0DB407FEFDCF8EB50EBD0DB407FEC2
:104DB000FDCF8EB586E261E00F94E5101F910F9153
:104DC0000895EBE1F4E0E80FF11D808190E0E0CF81
:104DD000CF93DF9389E261E00F94321087E261E0C4
:104DE0000F94321083E461E00F94321082E461E0AA
:104DF0000F94321080E461E00F943210C0E0D0E0F4
:104E0000FE01EA5EFB4F8C2F6081A6DF2196C53044
:104E1000D105B1F7DF91CF910895CF93DF930F9430
:104E2000310E86E261E00F943210C0E0D0E0FE0166
:104E3000E55EFB4FDE01A05EBB4F6C91808190E090
:104E400070E0A6DF2196C530D10589F7DF91CF91BB
:104E50000895E3DFBDDFEAE0F1E0808182608083D6
:104E60008081816080838081846080838081806490
:104E700080838081806880830F9A179A0E9A169A91
:104E80000D9A159A0C9A149A0B9A139A26982E9AA0
:104E900025982D9A24982C9A389A4098179A10920F
:104EA000030B399A4198169A1092040B3A9A429839
:104EB000159A1092050B3B9A4398149A3C9A449881
:104EC000A1E8B0E08C918F7E8C938C9188608C935C
:104ED000E0E8F0E080818D7F808380818E7F808319
:104EE00080818F73808380818F7C80838C91887F89
:104EF00082608C9380E090E4909389008093880096
:104F00001092850010928400EFE6F0E080818260CC
:104F1000808381E080938D03789408959091EC14C0
:104F20008091ED14981739F00E942CD90E94B19EFF
:104F30000E940786F3CF0895F1DF179A1092030BB2
:104F4000169A1092040B159A1092050B149A089554
:104F50001F920F920FB60F920BB60F921124AF92C1
:104F6000BF92CF92DF92EF92FF920F931F932F93F6
:104F70003F934F935F936F937F938F939F93AF93E1
:104F8000BF93CF93DF93EF93FF938091BC049091F5
:104F9000BD04892B09F096C19091EC148091ED1419
:104FA000981719F4E0E0F0E014C08091ED1490E05F
:104FB00021E530E0829FF001839FF00D929FF00D7C
:104FC0001124E452F04FE05BFF4F81E08083E05515
:104FD000F040F093BD04E093BC04309709F46CC139
:104FE000E05BFF4F81E08083E055F0401092FC04CD
:104FF0001092FD041092FE041092FF0460AD71AD9A
:105000002CE96134720718F060E47CE904C03EE4E6
:105010006132730730F0769567957695679584E0F1
:1050200007C047E26131740730F07695679582E0FA
:105030008093F50407C08093F5046032710510F485
:1050400060E270E06052704058E060307507E8F050
:10505000472F50E0440F551F440F551F4D5A5E4FC8
:105060009A012E5F3F4FF901859194919C01AA27E7
:10507000639FC001629F810D9A1F06948A1F9A1F29
:105080001124FA01459154911EC0CB019695879544
:105090008C7F8D5A9A4FFC0145915491FC013296B8
:1050A00025913491862F90E087709070FC012E9F9F
:1050B000C0012F9F900D3E9F900D1124B3E0969557
:1050C0008795BA95E1F7481B590B44365105A8F46A
:1050D000E0E0F2E007C08091C00085FFFCCF319690
:1050E0009093C60090819923B1F788E895E04AE053
:1050F00050E00E947F3044E650E050930105409319
:1051000000058091F504992787FD909590930305FC
:1051100080930205E091BC04F091BD0464AD75ADCF
:105120007093FB046093FA04FCE961347F0718F084
:1051300060E47CE904C02EE46132720730F07695B9
:1051400067957695679584E007C037E2613173070C
:1051500030F07695679582E08093F50408C081E091
:105160008093F5046032710510F460E270E06052E3
:10517000704048E060307407E8F0472F50E0440F7B
:10518000551F440F551F4D5A5E4F9A012E5F3F4FDA
:10519000F901859194919C01AA27639FC001629FA8
:1051A000810D9A1F06948A1F9A1F1124FA014591B6
:1051B00054911EC0CB01969587958C7F8D5A9A4F3E
:1051C000FC0145915491FC01329625913491862F32
:1051D00090E087709070FC012E9FC0012F9F900D72
:1051E0003E9F900D112433E0969587953A95E1F70F
:1051F000481B590B44365105A0F4E0E0F2E007C02B
:105200008091C00085FFFCCF31969093C6009081BD
:105210009923B1F788E895E04AE050E070D744E67A
:1052200050E0CA01A0E0B0E08093F6049093F70448
:10523000A093F804B093F904509389004093880038
:10524000E091BC04F091BD0480899189A289B38961
:10525000B695A79597958795B095A09590958195CA
:105260009F4FAF4FBF4F8093DA049093DB04A0931E
:10527000DC04B093DD048093DE049093DF04A093FC
:10528000E004B093E1048093E2049093E304A093DC
:10529000E404B093E5048093E6049093E704A093BC
:1052A000E804B093E9041092EA041092EB0410921F
:1052B000EC041092ED0406C080ED97E09093890015
:1052C00080938800C091BC04D091BD04209709F45C
:1052D000ACC488A18093EE0480FF0AC08FB7F89415
:1052E00090910B019D7F90930B018FBF8FEF09C0B1
:1052F0008FB7F89490910B01926090930B018FBF40
:1053000081E0809389038091EE0481FF0AC08FB70A
:10531000F89490910B01916090930B018FBF8FEFE8
:1053200009C08FB7F89490910B019E7F90930B0169
:105330008FBF81E080938A038091EE0480FF3CC0A0
:1053400080918D038823C1F183B1829586958695DE
:1053500083708095282F217080FF2CC08091EF04EE
:10536000882341F188819981AA81BB811816190689
:105370001A061B06FCF48091CA049091CB04A091FC
:10538000CC04B091CD048093BE049093BF04A0934D
:10539000C004B093C10481E08093F00488899989A6
:1053A000AA89BB898093EA049093EB04A093EC0450
:1053B000B093ED042093EF048091EE0481FF3BC095
:1053C00080918D038823B9F183B18295869587708A
:1053D0008095282F217080FF2CC08091F1048823B4
:1053E00041F18C819D81AE81BF81181619061A0684
:1053F0001B06FCF48091CE049091CF04A091D004C0
:10540000B091D1048093C2049093C304A093C404C8
:10541000B093C50481E08093F20488899989AA89B0
:10542000BB898093EA049093EB04A093EC04B093BF
:10543000ED042093F1048091EE0482FF47C09FB7F2
:10544000F89480910B018B7F80930B019FBF8FEFAE
:1054500080938B0380918D03882309F442C083B12C
:1054600082958F708095282F217080FF2CC08091AD
:10547000F304882341F188859985AA85BB85181690
:1054800019061A061B06FCF48091D2049091D304ED
:10549000A091D404B091D5048093C6049093C7041E
:1054A000A093C804B093C90481E08093F404888970
:1054B0009989AA89BB898093EA049093EB04A0930D
:1054C000EC04B093ED042093F3040BC08FB7F89471
:1054D00090910B01946090930B018FBF81E08093BA
:1054E0008B038091EE0483FF0AC08FB7F8949091EC
:1054F0000B01906490930B018FBF8FEF09C08FB7A2
:10550000F89490910B019F7B90930B018FBF81E0EA
:1055100080938C0360E06AC18091C00087FF19C04E
:105520004091C600E0918405F091850531969F0178
:105530002F773070319780918605909187052817D5
:10554000390739F0EC5FFA4F40833093850520939B
:105550008405288139814A815B818091DA049091A8
:10556000DB04A091DC04B091DD04280F391F4A1F31
:105570005B1F2093DA043093DB044093DC045093E8
:10558000DD0412161306140615066CF5409A888978
:105590009989AA89BB89281B390B4A0B5B0B20937D
:1055A000DA043093DB044093DC045093DD04209153
:1055B000CA043091CB044091CC045091CD04809129
:1055C0008903992787FD9095A92FB92F820F931FE3
:1055D000A41FB51F8093CA049093CB04A093CC045E
:1055E000B093CD0440982C813D814E815F818091A4
:1055F000DE049091DF04A091E004B091E104280F53
:10560000391F4A1F5B1F2093DE043093DF04409351
:10561000E0045093E10412161306140615066CF507
:10562000419A88899989AA89BB89281B390B4A0B19
:105630005B0B2093DE043093DF044093E00450932F
:10564000E1042091CE043091CF044091D0045091D8
:10565000D10480918A03992787FD9095A92FB92FAE
:10566000820F931FA41FB51F8093CE049093CF0485
:10567000A093D004B093D1044198288539854A85F8
:105680005B858091E2049091E304A091E404B091E1
:10569000E504280F391F4A1F5B1F2093E204309353
:1056A000E3044093E4045093E50412161306140631
:1056B00015066CF5429A88899989AA89BB89281BA5
:1056C000390B4A0B5B0B2093E2043093E3044093C5
:1056D000E4045093E5042091D2043091D304409126
:1056E000D4045091D50480918B03992787FD909520
:1056F000A92FB92F820F931FA41FB51F8093D20427
:105700009093D304A093D404B093D50442982C85ED
:105710003D854E855F858091E6049091E704A091D8
:10572000E804B091E904280F391F4A1F5B1F20933A
:10573000E6043093E7044093E8045093E90412161A
:105740001306140615066CF5439A88899989AA8967
:10575000BB89281B390B4A0B5B0B2093E604309363
:10576000E7044093E8045093E9042091D604309173
:10577000D7044091D8045091D90480918C03992783
:1057800087FD9095A92FB92F820F931FA41FB51FD6
:105790008093D6049093D704A093D804B093D904EF
:1057A00043988091EA049091EB04A091EC04B091AD
:1057B000ED040196A11DB11D8093EA049093EB04C2
:1057C000A093EC04B093ED042091EA043091EB0433
:1057D0004091EC045091ED0488899989AA89BB898C
:1057E000281739074A075B0730F46F5F8091F5048B
:1057F00068170CF491CE2091EA043091EB044091AB
:10580000EC045091ED048C899D89AE89BF89821783
:105810009307A407B50708F4E2C0E090F604F090FF
:10582000F7040091F8041091F904AC8CBD8CCE8C77
:10583000DF8CA8019701C601B501AA27279FB12DCA
:10584000389FF001489FF00D479FE00DF11D289F04
:10585000B00DE11DFA1F379FB00DE11DFA1F469FE5
:10586000B00DE11DFA1F369FB10DEA1FFA1FB69564
:10587000EA1FFA1F11248CAD9DAD8E0F9F1F9093D0
:10588000FB048093FA0428AD39AD4AAD5BADA0E0CE
:10589000B0E0281739074A075B0720F43093FB0470
:1058A0002093FA046091FA047091FB048CE961344E
:1058B000780718F060E47CE904C09EE4613279075F
:1058C00030F0769567957695679584E007C0E7E2B6
:1058D00061317E0730F07695679582E08093F5041C
:1058E00008C081E08093F5046032710510F460E235
:1058F00070E060527040F8E060307F07E8F0472FBA
:1059000050E0440F551F440F551F4D5A5E4F9A01EA
:105910002E5F3F4FF901859194919C01AA27639FC7
:10592000C001629F810D9A1F06948A1F9A1F11243D
:10593000FA01459154911EC0CB01969587958C7FB5
:105940008D5A9A4FFC0145915491FC013296259154
:105950003491862F90E087709070FC012E9FC001DB
:105960002F9F900D3E9F900D1124B3E09695879543
:10597000BA95E1F7481B590B44365105A0F4E0E015
:10598000F2E007C08091C00085FFFCCF3196909374
:10599000C60090819923B1F788E895E04AE050E08D
:1059A000AED344E650E050938900409388009A01BA
:1059B00040E050E08091F6049091F704A091F80443
:1059C000B091F904820F931FA41FB51F8093F604B2
:1059D0009093F704A093F804B093F90401C12091C7
:1059E000EA043091EB044091EC045091ED04888D71
:1059F000998DAA8DBB8D82179307A407B50708F070
:105A0000E3C06091FC047091FD048091FE049091CC
:105A1000FF042C8D3D8D4E8D5F8DAA27639FB12D88
:105A2000749FF001849FF00D839FE00DF11D649F32
:105A3000B00DE11DFA1F739FB00DE11DFA1F829F8B
:105A4000B00DE11DFA1F729FB10DEA1FFA1FB69546
:105A5000EA1FFA1F11248091FA049091FB048E171B
:105A60009F0738F4C05CDF4F68817981C054D04013
:105A700003C0BC016E1B7F0BC05CDF4F28813981E6
:105A80004A815B81CB01A0E0B0E082179307A407B5
:105A9000B50708F4B901FCE961347F0718F060E448
:105AA0007CE904C02EE46132720730F07695679588
:105AB0007695679584E007C037E26131730730F06F
:105AC0007695679582E08093F50408C081E0809325
:105AD000F5046032710510F460E270E060527040CD
:105AE00048E060307407E8F0472F50E0440F551F3E
:105AF000440F551F4D5A5E4F9A012E5F3F4FF901DB
:105B0000859194919C01AA27639FC001629F810D9A
:105B10009A1F06948A1F9A1F1124FA0145915491E5
:105B20001EC0CB01969587958C7F8D5A9A4FFC01AC
:105B300045915491FC01329625913491862F90E045
:105B400087709070FC012E9FC0012F9F900D3E9F8B
:105B5000900D112423E0969587952A95E1F7481B2F
:105B6000590B44365105A0F4E0E0F2E007C0809103
:105B7000C00085FFFCCF31969093C6009081992399
:105B8000B1F788E895E04AE050E0B9D244E650E049
:105B900050938900409388009A0140E050E0809142
:105BA000FC049091FD04A091FE04B091FF04820FCB
:105BB000931FA41FB51F8093FC049093FD04A09332
:105BC000FE04B093FF040CC0809100059091010584
:105BD0009093890080938800809102058093F5045A
:105BE0002091EA043091EB044091EC045091ED04D3
:105BF000E091BC04F091BD0480899189A289B389A8
:105C0000281739074A075B0780F01092BD041092ED
:105C1000BC049091EC148091ED14981731F08091B0
:105C2000ED148F5F8F708093ED14FF91EF91DF91F2
:105C3000CF91BF91AF919F918F917F916F915F9124
:105C40004F913F912F911F910F91FF90EF90DF9017
:105C5000CF90BF90AF900F900BBE0F900FBE0F90E4
:105C60001F9018958091F004882349F48091F204E4
:105C7000882329F48091F404882309F49CC0E3E587
:105C8000F9E0949108C08091C00085FFFCCF90930B
:105C9000C600319694919923B1F7E5E9F9E0949122
:105CA00008C08091C00085FFFCCF9093C60031965C
:105CB00094919923B1F78091F0048823F1F06091D9
:105CC000BE047091BF048091C0049091C1040F94F0
:105CD000B51620917B0F30917C0F40917D0F509134
:105CE0007E0F0F941A16AB01BC0181E999E00E9466
:105CF00072A281E899E00E942A858091F2048823AB
:105D0000F1F06091C2047091C3048091C404909139
:105D1000C5040F94B51620917F0F3091800F4091EC
:105D2000810F5091820F0F941A16AB01BC018DE7C1
:105D300099E00E9472A28DE699E00E942A858091E6
:105D4000F4048823F1F06091C6047091C704809137
:105D5000C8049091C9040F94B5162091830F309117
:105D6000840F4091850F5091860F0F941A16AB0146
:105D7000BC0189E699E00E9472A289E599E00E943F
:105D80002A85E4E1F2E007C08091C00085FFFCCFE6
:105D900031969093C60090819923B1F78091C0000D
:105DA00085FFFCCF8AE08093C6001092F004109229
:105DB000F2041092F40408951F920F920FB60F92FE
:105DC0000BB60F9211242F933F934F938F939F9372
:105DD000EF93FF934091C600E0918405F091850513
:105DE00031969F012F773070319780918605909181
:105DF00087052817390739F0EC5FFA4F4083309355
:105E0000850520938405FF91EF919F918F914F918C
:105E10003F912F910F900BBE0F900FBE0F901F90D0
:105E200018959A01AB01203081EE380780E04807D1
:105E300080E0580749F182E08093C00060E079E09B
:105E40008DE390E00F942D1A215030404040504097
:105E5000CA01B90122E030E040E050E00F942D1A71
:105E60003093C5002093C4008091C100806180936D
:105E7000C1008091C10088608093C1008091C10001
:105E800080688093C10008951092C00020E130E046
:105E9000E7CF209186053091870580918405909108
:105EA00085058217930719F42FEF3FEF0EC0F90114
:105EB000EC5FFA4F80812F5F3F4F2F773070309328
:105EC000870520938605282F30E0C9010895809129
:105ED00086059091870590938505809384050895A4
:105EE00008952F923F924F925F926F927F928F927E
:105EF0009F92AF92BF92CF92DF92EF92FF920F9359
:105F00001F93DF93CF93CDB7DEB7A0970FB6F8946A
:105F1000DEBF0FBECDBF1C016A017B0141155105DB
:105F20006105710541F440E350E060E070E020E07D
:105F300030E08BD055C0882499245401422E55243A
:105F40006624772401E010E00C0F1D1F080D191DB9
:105F5000C701B601A30192010F940B1AF8016083E7
:105F60000894811C911CA11CB11CC701B601A3019E
:105F700092010F940B1AC901DA016C017D01C11461
:105F8000D104E104F104F1F681E0E82EF12CEC0EED
:105F9000FD1EE80CF91C3E010894611C711CD50122
:105FA000C4010197A109B1096C01C818D90815C02D
:105FB000F601EE0DFF1D40814A3010F4405D01C036
:105FC000495C552747FD5095652F752FC10120E08D
:105FD00030E03BD00894E108F1086E147F0441F7EB
:105FE000A0960FB6F894DEBF0FBECDBFCF91DF9164
:105FF0001F910F91FF90EF90DF90CF90BF90AF90E7
:106000009F908F907F906F905F904F903F902F90D8
:1060100008952115310539F48091C00085FFFCCF2A
:106020004093C60008955DCFEF92FF920F931F93A8
:106030009A01E62EFF2400E010E0B801A701E9DF95
:106040001F910F91FF90EF900895EF92FF920F93A1
:106050001F93CF93DF93EC017A018B01211531055A
:1060600039F48091C00085FFFCCFE092C60019C0D2
:106070002A303105A9F477FF0FC04DE250E060E00F
:1060800070E020E030E0E1DF10950095F094E094BE
:10609000E11CF11C011D111DCE01B801A7012AE070
:1060A00020DFDF91CF911F910F91FF90EF90089526
:1060B000EF92FF920F931F937B019A010027F7FC49
:1060C0000095102FB801A701C0DF1F910F91FF901D
:1060D000EF9008950F931F938C014DE050E060E026
:1060E00070E020E030E0B1DFC8014AE050E060E05D
:1060F00070E020E030E0A9DF1F910F910895CF926A
:10610000DF92EF92FF920F931F938C019A016B0124
:10611000EE24FF24B701A6017CDFC801DBDF1F915D
:106120000F91FF90EF90DF90CF9008959F92AF92E4
:10613000BF92CF92DF92EF92FF920F931F93CF9374
:10614000DF93EC017A018B01922ECB01BA0120E0A2
:1061500030E040E050E00F941316882364F4CE0141
:106160004DE250E060E070E020E030E06EDF17FBD1
:10617000109517F9109520E030E040E05FE3AA2485
:106180000BC0CA01B90120E030E040E251E40F94B5
:106190001A169B01AC01A394A91498F3C801B70186
:1061A0000F943A157B018C010F9487165B016C01EB
:1061B0000F94B3169B01AC01C801B7010F943915B8
:1061C0007B018C01CE01B601A5012AE030E021DF80
:1061D000992099F1E5E1F2E007C08091C00085FFC8
:1061E000FCCF31969093C60090819923B1F725C0DA
:1061F000C801B70120E030E040E251E40F94F31809
:106200007B018C010F9482165B016C01CC24B7FCDE
:10621000C094DC2CCE01B601A5012AE030E015DFE8
:10622000C601B5010F94B5169B01AC01C801B701B9
:106230000F9439157B018C019A949920C9F6DF914E
:10624000CF911F910F91FF90EF90DF90CF90BF9073
:10625000AF909F9008956ACF0895382F20E09FB7A0
:10626000F894809105018B7F809305019FBF37FFD4
:1062700002C0A39A01C0A3989FB7F894809105012A
:106280008460809305019FBF2F5F283011F0330F8A
:10629000E6CF08951092CC05089580910B0890E008
:1062A000969587959695879581700895FC01208134
:1062B000822F90E06AE070E00F94F819CB016AE059
:1062C00070E00F94F819805D80933A08822F90E077
:1062D0006AE070E00F94F819805D80933B0810929B
:1062E0003C088AE398E00895FC0160817181828115
:1062F000938120E030E040E251E40F94F3180F94D2
:1063000082169B0177FF02C08DE201C08BE2809371
:106310003A0837FF03C0309521953F4FC90168EE19
:1063200073E00F94F819CB016AE070E00F94F8194C
:10633000805D80933B08C90164E670E00F94F81912
:10634000CB016AE070E00F94F819805D80933C08FF
:10635000C9016AE070E00F94F819CB016AE070E0BF
:106360000F94F819805D80933D088EE280933E087B
:10637000C9016AE070E00F94F819805D80933F08CE
:10638000109240088AE398E00895FC0160817181D1
:106390008281938120E030E040E251E40F94F318D1
:1063A0000F9482169B0177FF03C0309521953F4FD4
:1063B000C90168EE73E00F94F819CB016AE070E050
:1063C0000F94F819805D80933A08C90164E670E083
:1063D0000F94F819CB016AE070E00F94F819805D12
:1063E00080933B08C9016AE070E00F94F819CB0173
:1063F0006AE070E00F94F819805D80933C088EE2AB
:1064000080933D08C9016AE070E00F94F819805D3F
:1064100080933E0810923F088AE398E00895EF9237
:10642000FF920F931F93FC016081718182819381A0
:1064300020E030E048EC52E40F94F3180F948216F9
:106440007B018C0197FD12C020E137E240E050E073
:106450000F942D1ACA01B9012AE030E040E050E063
:106460000F942D1A605D60933A0803C08DE280930B
:106470003A0817FF08C010950095F094E094E11CCD
:10648000F11C011D111DC801B70128EE33E040E0E9
:1064900050E00F942D1ACA01B9012AE030E040E023
:1064A00050E00F942D1A605D60933B08C801B7015E
:1064B00024E630E040E050E00F942D1ACA01B90103
:1064C0002AE030E040E050E00F942D1A605D6093C8
:1064D0003C088EE280933D08C801B7012AE030E015
:1064E00040E050E00F942D1ACA01B9012AE030E0D3
:1064F00040E050E00F942D1A605D60933E08C801A3
:10650000B7012AE030E040E050E00F942D1A605DC2
:1065100060933F08109240088AE398E01F910F9122
:10652000FF90EF900895FC01808191818436910560
:106530005CF064E670E00F94F819CB016AE070E05B
:106540000F94F819805D01C080E280933A08808141
:1065500091818A3091055CF06AE070E00F94F8193F
:10656000CB016AE070E00F94F819805D01C080E211
:1065700080933B08808191816AE070E00F94F81964
:10658000805D80933C0810923D088AE398E008956E
:10659000DF93CF930F920F92CDB7DEB7FC016081EE
:1065A0007181828193810F9482167A836983CE01EF
:1065B0000196B9DF0F900F90CF91DF910895EF9280
:1065C000FF920F931F93FC01E080F1800281138101
:1065D000C801B70120E030E040E050E00F942118FE
:1065E00018161CF4C801B70103C0C801B7019058C0
:1065F0000F9482167B018C0180E1E81687E2F80691
:1066000080E0080780E01807A4F0C801B70120E186
:1066100037E240E050E00F942D1ACA01B9012AE098
:1066200030E040E050E00F942D1A605D60933A082E
:106630000CC080E280933A0898EEE91693E0F906E0
:1066400090E0090790E01907A4F0C801B70128EE0F
:1066500033E040E050E00F942D1ACA01B9012AE05E
:1066600030E040E050E00F942D1A605D60933B08ED
:1066700008C080933B0894E6E916F1040105110572
:10668000A4F0C801B70124E630E040E050E00F94E8
:106690002D1ACA01B9012AE030E040E050E00F9421
:1066A0002D1A605D60933C0808C080933C089AE016
:1066B000E916F10401051105A4F0C801B7012AE0AB
:1066C00030E040E050E00F942D1ACA01B9012AE0F1
:1066D00030E040E050E00F942D1A605D60933D087B
:1066E00002C080933D08C801B7012AE030E040E0D5
:1066F00050E00F942D1A605D60933E0810923F08A1
:106700008AE398E01F910F91FF90EF900895EF9228
:10671000FF920F931F93FC016081718182819381AD
:1067200020E030E040E251E40F94F3180F94821619
:1067300097FF02C02DE201C02BE220933A087B01B3
:106740008C0197FF08C010950095F094E094E11C2F
:10675000F11C011D111DC801B70120E137E240E025
:1067600050E00F942D1ACA01B9012AE030E040E050
:1067700050E00F942D1A605D60933B08C801B7018B
:1067800028EE33E040E050E00F942D1ACA01B90121
:106790002AE030E040E050E00F942D1A605D6093F5
:1067A0003C08C801B70124E630E040E050E00F9417
:1067B0002D1ACA01B9012AE030E040E050E00F9400
:1067C0002D1A605D60933D08C801B7012AE030E0F2
:1067D00040E050E00F942D1ACA01B9012AE030E0E0
:1067E00040E050E00F942D1A605D60933E088EE209
:1067F00080933F08C801B7012AE030E040E050E054
:106800000F942D1A605D60934008109241088AE34E
:1068100098E01F910F91FF90EF900895EF92FF92F3
:106820000F931F93FC01608171818281938120E02D
:1068300030E048EC52E40F94F3180F94821697FF5F
:1068400002C02DE201C02BE220933A087B018C01AB
:1068500097FF08C010950095F094E094E11CF11C9E
:10686000011D111DC801B70120E137E240E050E0F1
:106870000F942D1ACA01B9012AE030E040E050E03F
:106880000F942D1A605D60933B08C801B70128EE94
:1068900033E040E050E00F942D1ACA01B9012AE01C
:1068A00030E040E050E00F942D1A605D60933C08AA
:1068B000C801B70124E630E040E050E00F942D1A03
:1068C000CA01B9012AE030E040E050E00F942D1AEF
:1068D000605D60933D088EE280933E08C801B70179
:1068E0002AE030E040E050E00F942D1ACA01B901CF
:1068F0002AE030E040E050E00F942D1A605D609394
:106900003F08C801B7012AE030E040E050E00F94B2
:106910002D1A605D60934008109241088AE398E068
:106920001F910F91FF90EF9008950F93DF93CF93F6
:1069300000D00F92CDB7DEB7009103010295069506
:106940000770009501708091030186FF026020911D
:106950000D0830910E0840910F08509110082983BE
:106960003A834B835C830F948B0E29813A814B8150
:106970005C81261737074807590710F4629B0460AB
:1069800000930B0890910B08917080910B0881FD8A
:10699000926080911108981729F19130B1F09130EF
:1069A00028F0923041F09330E9F40AC0813079F058
:1069B0008230C1F412C0882351F0833099F40DC0A5
:1069C000823029F0813071F408C0833021F4809145
:1069D00089058F5F05C0882329F48091890581503E
:1069E00080938905909311080F900F900F900F904E
:1069F000CF91DF910F910895CF93DF93EC0104C005
:106A00008FEC97E00F947011FE012196649166233C
:106A1000B9F7DF91CF910895EF92FF920F931F93F3
:106A2000CF93DF93F82EEB01142FE22E4E3311F0AB
:106A30004B3FA9F483ED97E061E00F949F0D4CE08C
:106A4000F49EA00111244D5F83ED97E060E020E803
:106A50000CE00F94ED0883ED97E060E003C083ED58
:106A600097E061E00F949F0D109208082F2D30E001
:106A70002F5F3F4FC901880F991F820F931F880F07
:106A8000991F880F991F809309081E3321F08FECFE
:106A900097E0612F03C08FEC97E060E20F947011D4
:106AA00001E106C08FEC97E00F9470112196015020
:106AB000FE0164916623B1F706C08FEC97E060E2B7
:106AC0000F94701101500023C1F78FEC97E06E2DE9
:106AD0000F9470118FEC97E060E20F94701183EDCA
:106AE00097E061E00F949F0DDF91CF911F910F917F
:106AF000FF90EF900895EF92FF920F931F93DF9313
:106B0000CF93CDB7DEB72C970FB6F894DEBF0FBE8C
:106B1000CDBF83ED97E061E00F949F0D8091420817
:106B200080FF11C080910C0B90910D0B892B59F0B7
:106B300083ED97E069E041E02FE003E179EDE72E96
:106B40007CE1F72E0AC083ED97E069E041E02FE099
:106B500003E156EFE52E5DE1F52E0F940A0C83ED6F
:106B600097E06AE24AE228E007E00F94ED0883ED3F
:106B700097E062E34CE222E005E00F94ED0883ED3C
:106B800097E06AE241E32AE004E00F94080983ED0C
:106B900097E062E34BE20F94880D83ED97E066E3A4
:106BA00041E329E40F94080983ED97E064EA79E072
:106BB0000F94540A809149088823B9F18091180AEA
:106BC000882311F16091C20A7091C30A8091C40AAE
:106BD0009091C50A6115710581059105A9F06D595E
:106BE0007F4F8F4F9F4F24E630E040E050E00F94FE
:106BF0000B1A6091CA0A7091CB0A8091CC0A9091CD
:106C0000CD0A0F940B1A01C020E087E4289FC00131
:106C1000112464E670E00F94F819262F83ED97E0B5
:106C200067E342E302E00F94ED0880E580930808F3
:106C30008FE2809309088091100B9091110BA09125
:106C4000120BB091130B0097A105B105E1F10F9460
:106C50008B0E20E63AEE40E050E00F940B1A7901DB
:106C60008A016091100B7091110B8091120B909121
:106C7000130B20E63AEE40E050E00F940B1AE21AB4
:106C8000F30AC7016CE370E00F94E4196983CE0145
:106C900001960CDBBC018FEC97E00F9494118FEC04
:106CA00097E06AE30F947011C7016CE370E00F94F2
:106CB000E4198A83CE010296F9DABC018FEC97E0E1
:106CC0000F94941103C081E29FE196DE83ED97E07B
:106CD00064EA79E00F94540A16E0109308081093C0
:106CE00009086091EF0C7091F00C882777FD809572
:106CF000982F0F94B51620E030E040E05FE30F944A
:106D00003A150F9482167C836B83CE0103960BDCBD
:106D1000BC018FEC97E00F9494118EE19FE16CDE43
:106D2000109308088BE1809309086091F50C70912D
:106D3000F60C8091F70C9091F80C20E030E040E0E8
:106D40005FE30F943A150F9482167E836D83CE0114
:106D50000596E9DBBC018FEC97E00F9494118BE171
:106D60009FE14ADE6091EF0C7091F00C882777FD6F
:106D70008095982F0F94B5162091F50C3091F60C54
:106D80004091F70C5091F80C0F94211818164CF004
:106D900083ED97E06DE041E122E002E00F94ED0821
:106DA00012C083ED97E060E00F949F0D83ED97E0B4
:106DB0006DE041E122E002E00F94ED0883ED97E001
:106DC00061E00F949F0D83ED97E064EA79E00F9402
:106DD000540A8FE1809308081BE1109309088FEC97
:106DE00097E067E172E00F94941183ED97E064EA15
:106DF00079E00F94540A87E38093080810930908F8
:106E00008FEC97E067E172E00F94941183ED97E0C7
:106E100064EA79E00F94540A01E50093080886E0DB
:106E2000809309086091F10C7091F20C882777FD2E
:106E30008095982F0F94B51620E030E040E05FE396
:106E40000F943A150F94821678876F83CE010796B8
:106E50006ADBBC018FEC97E00F94941188E19FE10D
:106E6000CBDD00930808109309086091FB0C70912A
:106E7000FC0C8091FD0C9091FE0C20E030E040E095
:106E80005FE30F943A150F9482167A876987CE01D3
:106E9000099649DBBC018FEC97E00F94941185E1D2
:106EA0009FE1AADD6091F10C7091F20C882777FDCB
:106EB0008095982F0F94B5162091FB0C3091FC0C07
:106EC0004091FD0C5091FE0C0F94211818164CF0B7
:106ED00083ED97E068E542E122E002E00F94ED08DF
:106EE00012C083ED97E060E00F949F0D83ED97E073
:106EF00068E542E122E002E00F94ED0883ED97E0BF
:106F000061E00F949F0D83ED97E064EA79E00F94C0
:106F1000540A88E6809308088BE180930908209141
:106F20000C0B30910D0B84E690E0AC01249FC00166
:106F3000259F900D349F900D112460E071E00F9417
:106F4000F8196F5F7F4F7C876B87CE010B96EBDA6A
:106F5000BC018FEC97E00F9494118FEC97E06BE1FC
:106F600072E00F94941183ED97E064EA79E00F9456
:106F7000540A83ED97E060E04DE120E80AE00F94C9
:106F8000ED0883ED97E060E00F949F0D82E0809321
:106F9000080815E2109309088FEC97E06DE172E0A4
:106FA0000F94941183ED97E068E041E20F94880D0F
:106FB00083ED97E068E043E20F94880D8AE08093C8
:106FC0000808109309088BED9AE0DFD9BC018FEC1B
:106FD00097E00F9494118BE28093080810930908AE
:106FE00083E19FE109DD83ED97E061E341E20F94E6
:106FF000880D83ED97E061E343E20F94880D83E30E
:1070000080930808109309088FED9AE0BED9BC015F
:107010008FEC97E00F94941183E580930808109308
:1070200009088FEC97E06FE172E00F94941183ED03
:1070300097E069E541E20F94880D83ED97E069E5FB
:1070400043E20F94880D8BE580930808109309089C
:1070500083EE9AE049D9BC018FEC97E00F9494112C
:1070600083ED97E061E00F949F0D83ED97E060EA78
:1070700072E10F94540A83E08093080881E38093BF
:1070800009088FEC97E06DEF0F94701183ED97E096
:1070900064EA79E00F94540A8CE08093080880E356
:1070A0008093090884EC93E03EDABC018FEC97E012
:1070B0000F9494118FEC97E065E20F94701183EDBB
:1070C00097E064EA79E00F94540A109208088DE37F
:1070D000809309088FEC97E06EE873E00F949411A9
:1070E0002C960FB6F894DEBF0FBECDBFCF91DF91C7
:1070F0001F910F91FF90EF90089582E08093B3036A
:107100000F948B0E6C507E4F8F4F9F4F60930D08E6
:1071100070930E0880930F08909310086E9A8FE476
:1071200067E174E020E030E040E050E00F944B1263
:107130006AE070E080E090E00F94990E8FE40D9487
:10714000D71180911B08882321F0815080931B0860
:1071500003C081E08093B3038091B303882321F0BF
:10716000CADC8AE080931B0880910B0882FF0FC065
:1071700083ED91E49093B2038093B10310921208CF
:10718000109213081092140810921508B6DF20917F
:10719000C4033091C5032436310554F4809112089C
:1071A00090911308280F391F253631056CF41AC049
:1071B00025363105BCF08091120890911308280FF4
:1071C000391F2436310574F41092120810921308F6
:1071D000109214081092150884E690E09093C5036D
:1071E0008093C4032091C4033091C5032436310534
:1071F00089F480911208909113088B3091051CF04E
:10720000865A9F4F0DC02FEF863F9207ACF48259EC
:107210009F4F06C08091120890911308820F931F10
:107220009093C5038093C403109212081092130820
:1072300010921408109215088091C4039091C50310
:107240000A9734F48AE090E09093C5038093C403D6
:107250008091C4039091C503885E934034F087EE1B
:1072600093E09093C5038093C4030895AF92BF92B7
:10727000CF92DF92EF92FF920F931F9380911208AB
:1072800090911308A0911408B0911508815090486E
:10729000A040B04040F010921208109213081092D3
:1072A00014081092150860911208709113088091CB
:1072B00014089091150825E030E040E050E00F946C
:1072C0000B1A79018A0180910C0890E0A0E0B0E0EF
:1072D000E816F9060A071B0710F420930C08009122
:1072E0000C0880910B0890E0969587959695879568
:1072F000FF24F394F82210E0E3E1AE2EB12CC12C70
:10730000D12CEE24E394002379F58091B3038823F4
:10731000B9F08091120890911308A0911408B091CF
:1073200015080597A105B10528F4812F6FEC75E2CA
:107330004BEF04C0812F6FEC75E240E22BEF6CDB6A
:10734000FF2009F4DBC08091120890911308A091EE
:107350001408B09115080597A105B10508F0CEC035
:10736000CCDE8BE29DE3BDC0013009F03DC08091D1
:10737000B3038823F1F06091120870911308809193
:1073800014089091150825E030E040E050E00F949B
:107390000B1A213031054105510529F4812F65EC87
:1073A00075E24EE304C0812F65EC75E240E22AEFFE
:1073B00033DBFF2009F4A2C060911208709113081A
:1073C000809114089091150825E030E040E050E0ED
:1073D0000F940B1A213031054105510509F08EC07B
:1073E0008CDE83EC9CE37DC0023009F03DC08091CF
:1073F000B3038823F1F06091120870911308809113
:1074000014089091150825E030E040E050E00F941A
:107410000B1A223031054105510529F4812F6CEBFF
:1074200075E24EE304C0812F6CEB75E240E22AEF77
:10743000F3DAFF2009F462C060911208709113081A
:10744000809114089091150825E030E040E050E06C
:107450000F940B1A223031054105510509F04EC039
:107460004CDE86EB9CE33DC0033009F047C08091C1
:10747000B3038823F1F06091120870911308809192
:1074800014089091150825E030E040E050E00F949A
:107490000B1A233031054105510529F4812F61EB89
:1074A00075E24EE304C0812F61EB75E240E22AEF02
:1074B000B3DAFF2019F160911208709113088091DE
:1074C00014089091150825E030E040E050E00F945A
:1074D0000B1A233031054105510581F40EDE89EA8E
:1074E0009CE39093B2038093B10310921208109220
:1074F0001308109214081092150838C080911208D1
:1075000090911308A0911408B09115084497A10513
:10751000B10540F0A0921208B0921308C09214086E
:10752000D092150860911208709113088091140888
:107530009091150825E030E040E050E00F940B1AE0
:10754000422F80910C0890E0049630E08217930758
:1075500044F4445040930C08E092B303042F0150CC
:107560001FEF1F5F153010F40F5FCDCE1F910F91ED
:10757000FF90EF90DF90CF90BF90AF900895CF92A3
:10758000DF92EF92FF920F931F93809112089091D8
:107590001308A0911408B091150881509048A0409C
:1075A000B04040F010921208109213081092140884
:1075B00010921508609112087091130880911408B8
:1075C0009091150825E030E040E050E00F940B1A50
:1075D00079018A0180910C0890E0A0E0B0E0E81603
:1075E000F9060A071B0710F420930C08F0900C080A
:1075F00080910B0890E09695879596958795EE2457
:10760000E394E82200E0A5E0DA2ECC24C394FF2026
:1076100079F58091B3038823B9F080911208909195
:107620001308A0911408B09115080597A105B1059C
:1076300028F4802F66EF75E24BEF04C0802F66EFD1
:1076400075E240E22BEFE8D9EE2009F490C080917A
:10765000120890911308A0911408B091150805978D
:10766000A105B10508F083C048DD86E399E30FC1A9
:1076700081E0F81609F03DC08091B3038823F1F052
:107680006091120870911308809114089091150868
:1076900025E030E040E050E00F940B1A2130310536
:1076A0004105510529F4802F6FEE75E24EE304C0C9
:1076B000802F6FEE75E240E22AEFAED9EE2009F49A
:1076C00056C060911208709113088091140890912F
:1076D000150825E030E040E050E00F940B1A21300F
:1076E00031054105510509F042C007DD88EF93E8F7
:1076F000CEC022E0F216D9F58091B3038823F1F0D1
:1077000060911208709113088091140890911508E7
:1077100025E030E040E050E00F940B1A22303105B4
:107720004105510529F4802F68EE75E24EE304C04F
:10773000802F68EE75E240E22AEF6ED9EE20B9F0B4
:1077400060911208709113088091140890911508A7
:1077500025E030E040E050E00F940B1A2230310574
:107760004105510521F4C9DC86E493E890C060919D
:10777000360870913708809138089091390820E0D8
:1077800030E040E251E40F94131688230CF08CC0D3
:1077900083E0F81609F03DC08091B3038823F1F02F
:1077A0006091120870911308809114089091150847
:1077B00025E030E040E050E00F940B1A2330310513
:1077C0004105510529F4802F61EE75E24EE304C0B6
:1077D000802F61EE75E240E22AEF1ED9EE2009F417
:1077E00065C06091120870911308809114089091FF
:1077F000150825E030E040E050E00F940B1A2330EC
:1078000031054105510509F051C077DC84E992E862
:107810003EC024E0F21609F049C08091B3038823EA
:10782000F1F0609112087091130880911408909102
:10783000150825E030E040E050E00F940B1A2430AA
:1078400031054105510529F4802F68ED75E24EE3BD
:1078500004C0802F68ED75E240E22AEFDDD8EE200B
:1078600029F1609112087091130880911408909189
:10787000150825E030E040E050E00F940B1A24306A
:1078800031054105510591F438DC80E192E890938F
:10789000B2038093B1031092120810921308109251
:1078A0001408109215084EC013E001C015E0609155
:1078B000120870911308809114089091150825E022
:1078C00030E040E050E00F940B1A812F90E0A0E0F0
:1078D000B0E0281739074A075B0780F01D9DC001FB
:1078E00011240197AA2797FDA095BA2F809312081B
:1078F00090931308A0931408B09315086091120890
:1079000070911308809114089091150825E030E0DB
:1079100040E050E00F940B1A422F80910C0890E049
:10792000049630E08217930744F4445040930C08C7
:10793000C092B303F42EFA940FEF0F5F053010F4EA
:10794000F39465CE1F910F91FF90EF90DF90CF9051
:1079500008958DEC9CECACECBDE3809336089093DD
:107960003708A0933808B093390809CE80E090E03A
:10797000A0E8BFE38093360890933708A0933808B7
:10798000B0933908FCCD80E090E0A0E2B1E48093B0
:10799000360890933708A0933808B0933908EFCD94
:1079A0000F931F93DF93CF93CDB7DEB76E970FB6CC
:1079B000F894DEBF0FBECDBF00D000D0EDB7FEB74C
:1079C00031969E012F5F3F4FADB7BEB712963C93E5
:1079D0002E93119722EA3FE1338322839583848398
:1079E0000E946F228E010B5F1F4FEDB7FEB73696D8
:1079F0000FB6F894FEBF0FBEEDBF08C0992787FDF4
:107A000090950F94561AD8018D938D01F8018081BD
:107A10008823A1F7CE0101960E94C7C38EE99FE19A
:107A20000E944EC31092120810921308109214086C
:107A30001092150881EA98E39093B2038093B10302
:107A40006E960FB6F894DEBF0FBECDBFCF91DF911B
:107A50001F910F910895AF92BF92CF92DF92EF9254
:107A6000FF920F931F938091120890911308A09199
:107A70001408B091150881509048A040B04040F0E3
:107A80001092120810921308109214081092150800
:107A90006091120870911308809114089091150854
:107AA00025E030E040E050E00F940B1A79018A01A4
:107AB00080910C0890E0A0E0B0E0E816F9060A0713
:107AC0001B0710F420930C0800910C0880910B0800
:107AD00090E09695879596958795FF24F394F822E4
:107AE00010E083E1A82EB12CC12CD12CEE24E3941C
:107AF000002381F58091B3038823C1F0809112089F
:107B000090911308A0911408B09115080597A1054C
:107B1000B10528F4812F6CEA75E24BEF04C0812F88
:107B20006CEA75E240E22BEF0E940C35FF2009F46D
:107B3000E0C08091120890911308A0911408B091B0
:107B400015080597A105B10508F0D3C0D6DA83ED75
:107B500091E4C2C0013009F03EC08091B303882394
:107B6000F9F06091120870911308809114089091B7
:107B7000150825E030E040E050E00F940B1A21306A
:107B800031054105510529F4812F6BE975E24EE37A
:107B900004C0812F6BE975E240E220E20E940C35BF
:107BA000FF2009F4A6C0609112087091130880911B
:107BB00014089091150825E030E040E050E00F9463
:107BC0000B1A213031054105510509F092C095DAB3
:107BD00087E995E240C0023009F040C08091B303CC
:107BE0008823F9F0609112087091130880911408AD
:107BF0009091150825E030E040E050E00F940B1A1A
:107C0000223031054105510529F4812F6DE875E2D7
:107C10004EE304C0812F6DE875E240E220E20E944D
:107C20000C35FF2009F465C06091120870911308AB
:107C3000809114089091150825E030E040E050E074
:107C40000F940B1A223031054105510509F051C03E
:107C500054DA89E895E20E944EC383C0033009F0EC
:107C600048C08091B3038823F9F0609112087091A5
:107C70001308809114089091150825E030E040E049
:107C800050E00F940B1A233031054105510529F4BA
:107C9000812F6FE775E24EE304C0812F6FE775E235
:107CA00040E22AEF0E940C35FF2019F16091120882
:107CB00070911308809114089091150825E030E028
:107CC00040E050E00F940B1A233031054105510577
:107CD00081F413DA86E399E39093B2038093B103BE
:107CE000109212081092130810921408109215089E
:107CF00038C08091120890911308A0911408B09197
:107D000015084497A105B10540F0A0921208B09261
:107D10001308C0921408D09215086091120870914F
:107D20001308809114089091150825E030E040E098
:107D300050E00F940B1A422F80910C0890E00496AB
:107D400030E08217930744F4445040930C08E092CB
:107D5000B303042F01501FEF1F5F153010F40F5FA6
:107D6000C7CE1F910F91FF90EF90DF90CF90BF9003
:107D7000AF90089587E498E00E949FE010920C086D
:107D800008953F924F925F926F927F928F929F924F
:107D9000AF92BF92CF92DF92EF92FF920F931F9319
:107DA000CF93DF938091B303882309F098C2809129
:107DB0000B0882FD94C2A7C21092120810921308F9
:107DC000109214081092150860911208709113080F
:107DD000809114089091150825E030E040E050E0D3
:107DE0000F940B1A79018A0180910C0890E0A0E0B1
:107DF000B0E0E816F9060A071B0710F420930C08F8
:107E0000A0900C0880910B0890E096958795969528
:107E10008795992493949822EE2433243394562CF6
:107E20005A94F5E04F2EAA2091F58091B303882350
:107E3000C1F08091120890911308A0911408B0919C
:107E400015080597A105B10528F48E2D69E97FE194
:107E50004BEF04C08E2D69E97FE140E22BEF0E94D9
:107E60000C359920A1F08091120890911308A091EF
:107E70001408B09115080597A105B10540F43DD946
:107E800083ED91E49093B2038093B10326C18BE913
:107E900098E06BE478E00E94D4CB80914B088F325D
:107EA00019F4FF24F3942AC021E0A21629F5809149
:107EB000B3038823F9F06091120870911308809140
:107EC00014089091150825E030E040E050E00F9450
:107ED0000B1A213031054105510529F48E2D65E934
:107EE0007FE14EE304C08E2D65E97FE140E220E2B0
:107EF0000E940C359920E1F4E2E0FE2E8E2D90E0F8
:107F00009C01220F331F280F391F220F331F220F0E
:107F1000331F53E0852E820E01969C01220F331FE2
:107F2000280F391FB22EBB0CBB0CCC24DD2486C11C
:107F300060911208709113088091140890911508AF
:107F400025E030E040E050E00F940B1A213031057D
:107F50004105510589F6D1D80DDFD5C1FA1409F0D4
:107F600069C1652D6C1987E498E00E94BDEC809191
:107F700073089091B303882309F4B8C0992309F4D6
:107F80008AC0609112087091130880911408909132
:107F9000150825E030E040E050E00F940B1A8F2DDB
:107FA00090E0A0E0B0E0281739074A075B0709F026
:107FB00045C080915808882319F4CBE4D8E004C068
:107FC00010926A08C8E5D8E083ED97E061E00F946D
:107FD0009F0D83ED97E060E0482D20E80CE00F94C2
:107FE000ED0883ED97E060E00F949F0D1092080874
:107FF000B09209088FEC97E060E20F9470118FEC5B
:1080000097E069EF0F94701112E106C08FEC97E0D2
:108010000F9470112196115068816623B9F706C03C
:108020008FEC97E060E20F94701111501123C1F7AB
:1080300083ED97E061E00F949F0D2DC0809158086B
:10804000882319F4CBE4D8E004C010926A08C8E58C
:10805000D8E010920808B09209088FEC97E060E22F
:108060000F9470118FEC97E069EF0F94701112E18B
:1080700006C08FEC97E00F94701121961150688123
:108080006623B9F706C08FEC97E060E20F94701199
:1080900011501123C1F7992009F4CCC06091120846
:1080A00070911308809114089091150825E030E034
:1080B00040E050E00F940B1A8F2D90E0A0E0B0E06C
:1080C000281739074A075B0709F0B4C016D887E4B8
:1080D00098E06BE478E00E94F2E0109212081092AF
:1080E000130810921408109215080DC1992309F471
:1080F00080C06091120870911308809114089091CB
:10810000150825E030E040E050E00F940B1A8F2D69
:1081100090E0A0E0B0E0281739074A075B0709F0B4
:1081200040C080915808882319F4CBE4D8E004C0FB
:1081300010926B08C8E5D8E083ED97E061E00F94FA
:108140009F0D83ED97E060E0482D20E80CE00F9450
:10815000ED0883ED97E060E00F949F0D1092080802
:10816000B09209088FEC97E060E20F94701113E170
:1081700006C08FEC97E00F94701121961150688122
:108180006623B9F706C08FEC97E060E20F94701198
:1081900011501123C1F783ED97E061E00F949F0D1B
:1081A00028C080915808882319F4CBE4D8E004C093
:1081B00010926B08C8E5D8E010920808B092090840
:1081C0008FEC97E060E20F94701113E106C08FEC22
:1081D00097E00F9470112196115068816623B9F7CA
:1081E00006C08FEC97E060E20F94701111501123DC
:1081F000C1F79920F9F060911208709113088091ED
:1082000014089091150825E030E040E050E00F940C
:108210000B1A8F2D90E0A0E0B0E0281739074A072D
:108220005B0741F40E947D388BE498E068E578E0D4
:10823000B7DB69C0F3940894C11CD11CC614D704E1
:1082400008F48CCE60911208709113088091140884
:108250009091150825E030E040E050E00F940B1AB3
:108260008F2D90E0A0E0B0E0281739074A075B07A0
:1082700080F0F49CC00111240197AA2797FDA095D6
:10828000BA2F8093120890931308A0931408B09308
:10829000150860911208709113088091140890914C
:1082A000150825E030E040E050E00F940B1A422F13
:1082B00080910C0890E0049630E0821793074CF40C
:1082C000445040930C083092B303A42EAA94EE2499
:1082D000EA94E39484E08E15B0F0A394A4CD87E4EF
:1082E00098E00E945DEC3C01809112089091130887
:1082F000A0911408B091150881509048A040B0405A
:1083000008F05ACD61CDDF91CF911F910F91FF9071
:10831000EF90DF90CF90BF90AF909F908F907F9025
:108320006F905F904F903F900895CF93DF9310929E
:10833000490887E498E060E00E94C6E10E946F254A
:1083400089EA9FE10E944EC38091DB0F882301F1EF
:108350001092DB0F80910A0BC82FD0E0CC0FDD1FED
:10836000C151D34F68817981882777FD8095982FF7
:108370000F94B5162091090430910A0440910B0422
:1083800050910C040F942118181614F419821882B5
:10839000DF91CF91089587E498E00C9493E087E40F
:1083A00098E00C949AE0CF92DF92EF92FF920F93B5
:1083B0001F938091120890911308A0911408B09116
:1083C000150881509048A040B04040F0109212082B
:1083D0001092130810921408109215086091120858
:1083E00070911308809114089091150825E030E0F1
:1083F00040E050E00F940B1A79018A0180910C083B
:1084000090E0A0E0B0E0E816F9060A071B0710F4B8
:1084100020930C08F0900C0880910B0890E0969542
:10842000879596958795EE24E394E82200E015E081
:10843000D12ECC24C394FF2079F58091B3038823F7
:10844000C1F08091120890911308A0911408B09186
:1084500015080597A105B10528F4802F69E87FE18B
:108460004BEF04C0802F69E87FE140E22BEF0E94D0
:108470000C35EE2089F08091120890911308A0919C
:108480001408B09115080597A105B10528F40E94BC
:108490007D3881EA98E371C20E94C9F3882329F4E8
:1084A00080914908882309F4C1C281E0F81611F0CF
:1084B00082E0BFC08091B3038823F9F06091120875
:1084C00070911308809114089091150825E030E010
:1084D00040E050E00F940B1A213031054105510561
:1084E00029F4802F64E87FE14EE304C0802F64E824
:1084F0007FE140E22AEF0E940C35EE2009F4E3C050
:1085000060911208709113088091140890911508D9
:1085100025E030E040E050E00F940B1A21303105A7
:108520004105510509F0CFC00E947D3884E49FE6E3
:1085300024C28091B3038823F9F0609112087091EE
:108540001308809114089091150825E030E040E070
:1085500050E00F940B1A213031054105510529F4E3
:10856000802F6BE77FE14EE304C0802F6BE77FE154
:1085700040E22AEF0E940C35EE2009F459C06091C8
:10858000120870911308809114089091150825E045
:1085900030E040E050E00F940B1A213031054105E6
:1085A000510509F045C00E947D388BE29DE3E5C18D
:1085B00022E0F216E9F58091B3038823F9F0609187
:1085C000120870911308809114089091150825E005
:1085D00030E040E050E00F940B1A223031054105A5
:1085E000510529F4802F6FE67FE14EE304C0802F10
:1085F0006FE67FE140E22AEF0E940C35EE20C1F0E9
:1086000060911208709113088091140890911508D8
:1086100025E030E040E050E00F940B1A22303105A5
:108620004105510529F40E947D388AEA9AE8A5C1DE
:1086300083E08F1509F048C08091B303882319F1B6
:108640006091120870911308809114089091150898
:1086500025E030E040E050E00F940B1A8F2D90E0C1
:10866000A0E0B0E0281739074A075B0729F4802FFC
:1086700061E67FE14EE304C0802F61E67FE140E2E6
:108680002AEF0E940C35EE20E1F060911208709103
:108690001308809114089091150825E030E040E01F
:1086A00050E00F940B1A8F2D90E0A0E0B0E0281757
:1086B00039074A075B0729F40E947D3882E295E476
:1086C0005CC18F2D01C082E0182F1F5F80914A0886
:1086D000882309F40BC18091180A882309F4DFC0AC
:1086E00080914908882309F449C01F1509F08DC0FD
:1086F0008091B303882319F16091120870911308D7
:10870000809114089091150825E030E040E050E099
:108710000F940B1A8F2D90E0A0E0B0E028173907D6
:108720004A075B0729F4802F65E57FE14EE304C02B
:10873000802F65E57FE140E220E20E940C35EE20CB
:1087400009F463C0609112087091130880911408B5
:108750009091150825E030E040E050E00F940B1AAE
:10876000812F90E0A0E0B0E0281739074A075B07A7
:1087700009F04BC00E947D3812DE5DC11F1509F063
:1087800044C08091B303882319F16091120870915D
:108790001308809114089091150825E030E040E01E
:1087A00050E00F940B1A8F2D90E0A0E0B0E0281756
:1087B00039074A075B0729F4802F68E47FE14EE31D
:1087C00004C0802F68E47FE140E220E20E940C3583
:1087D000EE20D9F06091120870911308809114086E
:1087E0009091150825E030E040E050E00F940B1A1E
:1087F000812F90E0A0E0B0E0281739074A075B0717
:1088000021F40E947D38C7DD16C11F5F1F1509F0D6
:10881000C1C08091B303882319F16091120870914F
:108820001308809114089091150825E030E040E08D
:1088300050E00F940B1A812F90E0A0E0B0E02817D1
:1088400039074A075B0729F4802F6DE37FE14EE388
:1088500004C0802F6DE37FE140E220E20E940C35EE
:10886000EE2009F497C0609112087091130880916E
:1088700014089091150825E030E040E050E00F9496
:108880000B1A812F90E0A0E0B0E0281739074A07C3
:108890005B0709F07FC00E947D3847DDCCC01F1503
:1088A00009F078C08091B303882309F449C060912E
:1088B000120870911308809114089091150825E012
:1088C00030E040E050E00F940B1A8F2D90E0A0E0D4
:1088D000B0E0281739074A075B0721F4802F6FE2C1
:1088E0007FE125C0802F6FE27FE126C01F1509F0D0
:1088F00051C08091B303882319F1609112087091DF
:108900001308809114089091150825E030E040E0AC
:1089100050E00F940B1A8F2D90E0A0E0B0E02817E4
:1089200039074A075B0729F4802F67E27FE14EE3AE
:1089300004C0802F67E27FE140E22AEF0E940C35FD
:10894000EE2041F160911208709113088091140893
:108950009091150825E030E040E050E00F940B1AAC
:10896000812F90E0A0E0B0E0281739074A075B07A5
:1089700089F40E947D3881EC9EE39093B20380934A
:10898000B10310921208109213081092140810925A
:10899000150851C01F5F60911208709113088091F3
:1089A00014089091150825E030E040E050E00F9465
:1089B0000B1A812F90E0A0E0B0E0281739074A0792
:1089C0005B0780F01D9DC00111240197AA2797FD28
:1089D000A095BA2F8093120890931308A0931408BF
:1089E000B0931508609112087091130880911408D3
:1089F0009091150825E030E040E050E00F940B1A0C
:108A0000422F80910C0890E0049630E08217930783
:108A100044F4445040930C08C092B303F42EFA94EB
:108A20000FEF0F5F053038F4F39405CD81E0F816B1
:108A300009F0BECD7ECD1F910F91FF90EF90DF909A
:108A4000CF900895AF92BF92CF92DF92EF92FF92B4
:108A50000F931F938091120890911308A09114080E
:108A6000B091150881509048A040B04040F010925D
:108A700012081092130810921408109215086091B1
:108A8000120870911308809114089091150825E040
:108A900030E040E050E00F940B1A79018A01809198
:108AA0000C0890E0A0E0B0E0E816F9060A071B0702
:108AB00010F420930C0800910C0880910B0890E0B2
:108AC0009695879596958795FF24F394F82210E064
:108AD00088E1A82EB12CC12CD12CEE24E3940023E4
:108AE00089F58091B3038823C1F080911208909199
:108AF0001308A0911408B09115080597A105B105B8
:108B000028F4812F61EF7FE14BEF04C0812F61EFEB
:108B10007FE140E22BEF0E940C35FF2009F423C1D6
:108B20008091120890911308A0911408B091150833
:108B30000597A105B10508F016C10E947D3883EDA7
:108B400091E441C0013009F04BC08091B303882308
:108B5000F9F06091120870911308809114089091B7
:108B6000150825E030E040E050E00F940B1A21306A
:108B700031054105510529F4812F6FED7FE14EE369
:108B800004C0812F6FED7FE140E22AEF0E940C3597
:108B9000FF2009F4E8C060911208709113088091D9
:108BA00014089091150825E030E040E050E00F9463
:108BB0000B1A213031054105510509F0D4C00E943E
:108BC0007D388EE397E49093B2038093B1031092C3
:108BD0001208109213081092140810921508FBC086
:108BE000023009F03FC08091B3038823F9F060910F
:108BF000120870911308809114089091150825E0CF
:108C000030E040E050E00F940B1A2230310541056E
:108C1000510529F4812F62ED7FE14EE304C0812FDD
:108C200062ED7FE140E220E20E940C35FF2009F472
:108C30009AC0609112087091130880911408909165
:108C4000150825E030E040E050E00F940B1A223088
:108C500031054105510509F086C00E947D380E940A
:108C6000D98EB9C0033009F03FC08091B303882387
:108C7000F9F0609112087091130880911408909196
:108C8000150825E030E040E050E00F940B1A233047
:108C900031054105510529F4812F66EC7FE14EE352
:108CA00004C0812F66EC7FE140E220E20E940C3597
:108CB000FF2009F458C06091120870911308809148
:108CC00014089091150825E030E040E050E00F9442
:108CD0000B1A233031054105510509F044C00E94AB
:108CE0007D380E94D19877C00430E9F58091B303B4
:108CF0008823F9F06091120870911308809114088C
:108D00009091150825E030E040E050E00F940B1AF8
:108D1000243031054105510529F4812F65EB7FE1B0
:108D20004EE304C0812F65EB7FE140E220E20E9428
:108D30000C35FF20C1F060911208709113088091EA
:108D400014089091150825E030E040E050E00F94C1
:108D50000B1A243031054105510529F40E947D3854
:108D60000E945A9338C08091120890911308A091E4
:108D70001408B09115084997A105B10540F0A092DB
:108D80001208B0921308C0921408D092150860918E
:108D9000120870911308809114089091150825E02D
:108DA00030E040E050E00F940B1A422F80910C0805
:108DB00090E0049630E08217930744F444504093C7
:108DC0000C08E092B303042F01501FEF1F5F153012
:108DD00010F40F5F84CE1F910F91FF90EF90DF9002
:108DE000CF90BF90AF900895FF920F931F93CF93B2
:108DF000DF93EB01022FF32EE22FF32FDF010D9013
:108E00000020E9F7122F1A1B1C5E1092080890E050
:108E100001969C01220F331F280F391F220F331F89
:108E2000220F331F209309088FEC97E0642F0F94D3
:108E3000701106C08FEC97E00F94701121961150BD
:108E4000FE0164916623B1F78FEC97E06AE30F941B
:108E5000701106C08FEC97E060E20F947011115012
:108E60001123C1F78FEC97E0602F7F2D0F949411A1
:108E7000DF91CF911F910F91FF9008952F923F9214
:108E80004F925F926F927F928F929F92AF92BF921A
:108E9000CF92DF92EF92FF920F931F93DF93CF93C6
:108EA000CDB7DEB7A0970FB6F894DEBF0FBECDBF2B
:108EB0008091120890911308A0911408B0911508A0
:108EC00081509048A040B04040F01092120810929B
:108ED00013081092140810921508609112087091EE
:108EE0001308809114089091150825E030E040E0C7
:108EF00050E00F940B1A79018A0180910C0890E0E0
:108F0000A0E0B0E0E816F9060A071B0710F420936A
:108F10000C0800910C0880910B0890E096958795BD
:108F200096958795FF24F394F82210E08DE1C82EE2
:108F3000D12CCC0EDD1EB9E1AB2EB12CAC0EBD1E7A
:108F4000A5E18A2E912C8C0E9D1EF1E16F2E712CC5
:108F50006C0E7D1EEDE04E2E512C4C0E5D1E79E008
:108F6000272E312C2C0E3D1E002309F040C080918D
:108F7000B3038823C1F08091120890911308A09147
:108F80001408B09115080597A105B10528F4812FA3
:108F90006CE471E24BEF04C0812F6CE471E240E2BB
:108FA0002BEF0E940C35FF2011F40C943E5480915D
:108FB000120890911308A0911408B0911508059714
:108FC000A105B10510F00C943E540E947D3882E258
:108FD00095E49093B2038093B1031092120810921B
:108FE000130810921408109215080C947D54013047
:108FF00009F08DC08091B303882339F16091120884
:1090000070911308809114089091150825E030E0C4
:1090100040E050E00F940B1A213031054105510515
:1090200051F486E09BE00E940F329C01812F63E4A3
:1090300071E24EE309C086E09BE00E940F329C0182
:10904000812F63E471E240E2CFDEFF2011F40C9443
:109050003E54609112087091130880911408909109
:10906000150825E030E040E050E00F940B1A213065
:1090700031054105510511F00C943E540E947D3894
:109080008091B1039091B20390931D0880931C08C6
:10909000809112089091130890931F0880931E08E6
:1090A00082E08093B30386E896E79093B2038093BF
:1090B000B1038AE391E2909321088093200886E02F
:1090C0009BE0909323088093220882E390E0A0E045
:1090D000B0E08093240890932508A0932608B093CD
:1090E000270888E893E1A0E0B0E0809328089093F7
:1090F0002908A0932A08B0932B086091060B709161
:10910000070B8091080B9091090B0C947F52023051
:1091100009F08DC08091B303882339F16091120862
:1091200070911308809114089091150825E030E0A3
:1091300040E050E00F940B1A2230310541055105F3
:1091400051F483EA9FE00E94DF329C01812F64E3A7
:1091500071E24EE309C083EA9FE00E94DF329C0186
:10916000812F64E371E240E23FDEFF2011F40C94B2
:109170003E546091120870911308809114089091E8
:10918000150825E030E040E050E00F940B1A223043
:1091900031054105510511F00C943E540E947D3873
:1091A0008091B1039091B20390931D0880931C08A5
:1091B000809112089091130890931F0880931E08C5
:1091C00082E08093B30383EE95E79093B20380939C
:1091D000B1038EE291E2909321088093200883EA04
:1091E0009FE0909323088093220885E090E0A0E020
:1091F000B0E08093240890932508A0932608B093AC
:1092000027088EED93E0A0E0B0E0809328089093CB
:109210002908A0932A08B0932B086091A30F70919E
:10922000A40F8091A50F9091A60F0C945F5103306D
:1092300009F08DC08091B303882339F16091120841
:1092400070911308809114089091150825E030E082
:1092500040E050E00F940B1A2330310541055105D1
:1092600051F48BEA9FE00E94C8329C01812F65E295
:1092700071E24EE309C08BEA9FE00E94C8329C0174
:10928000812F65E271E240E2AFDDFF2011F40C9422
:109290003E546091120870911308809114089091C7
:1092A000150825E030E040E050E00F940B1A233021
:1092B00031054105510511F00C943E540E947D3852
:1092C0008091B1039091B20390931D0880931C0884
:1092D000809112089091130890931F0880931E08A4
:1092E00082E08093B30389E297E79093B20380937F
:1092F000B1038CE191E290932108809320088BEADE
:109300009FE0909323088093220881E090E0A0E002
:10931000B0E08093240890932508A0932608B0938A
:1093200027088EED93E0A0E0B0E0809328089093AA
:109330002908A0932A08B0932B086091AB0F709175
:10934000AC0F8091AD0F9091AE0F0C94335404305C
:1093500009F08DC08091B303882339F16091120820
:1093600070911308809114089091150825E030E061
:1093700040E050E00F940B1A2430310541055105AF
:1093800051F48FEA9FE00E940E349C01812F64E12A
:1093900071E24EE309C08FEA9FE00E940E349C0107
:1093A000812F64E171E240E21FDDFF2011F40C9493
:1093B0003E546091120870911308809114089091A6
:1093C000150825E030E040E050E00F940B1A2430FF
:1093D00031054105510511F00C943E540E947D3831
:1093E0008091B1039091B20390931D0880931C0863
:1093F000809112089091130890931F0880931E0883
:1094000082E08093B3038DE994E79093B203809355
:10941000B1038CE091E290932108809320088FEAB9
:109420009FE090932308809322088AE090E0A0E0D8
:10943000B0E08093240890932508A0932608B09369
:10944000270888EB92E8A1E0B0E080932808909389
:109450002908A0932A08B0932B086091AF0F709150
:10946000B00F8091B10F9091B20F0C947F520530E4
:1094700009F08DC08091B303882339F160911208FF
:1094800070911308809114089091150825E030E040
:1094900040E050E00F940B1A25303105410551058D
:1094A00051F483EB9FE00E94C8329C01812F64E05D
:1094B00071E24EE309C083EB9FE00E94C8329C0139
:1094C000812F64E071E240E28FDCFF2011F40C9404
:1094D0003E54609112087091130880911408909185
:1094E000150825E030E040E050E00F940B1A2530DD
:1094F00031054105510511F00C943E540E947D3810
:109500008091B1039091B20390931D0880931C0841
:10951000809112089091130890931F0880931E0861
:1095200082E08093B30389E297E79093B20380933C
:10953000B1038CEF90E2909321088093200883EB95
:109540009FE0909323088093220881E090E0A0E0C0
:10955000B0E08093240890932508A0932608B09348
:1095600027088EED93E0A0E0B0E080932808909368
:109570002908A0932A08B0932B086091B30F70912B
:10958000B40F8091B50F9091B60F0C943354063000
:1095900009F08DC08091B303882339F160911208DE
:1095A00070911308809114089091150825E030E01F
:1095B00040E050E00F940B1A26303105410551056B
:1095C00051F48BE69FE00E94C8329C01812F65EF29
:1095D00070E24EE309C08BE69FE00E94C8329C0116
:1095E000812F65EF70E240E2FFDBFF2011F40C9465
:1095F0003E54609112087091130880911408909164
:10960000150825E030E040E050E00F940B1A2630BA
:1096100031054105510511F00C943E540E947D38EE
:109620008091B1039091B20390931D0880931C0820
:10963000809112089091130890931F0880931E0840
:1096400082E08093B30389E297E79093B20380931B
:10965000B1038EEE90E290932108809320088BE670
:109660009FE0909323088093220881E090E0A0E09F
:10967000B0E08093240890932508A0932608B09327
:10968000270887EE93E0A0E0B0E08093280890934D
:109690002908A0932A08B0932B0860916B0F709152
:1096A0006C0F80916D0F90916E0F0C9433540730B6
:1096B00009F08DC08091B303882339F160911208BD
:1096C00070911308809114089091150825E030E0FE
:1096D00040E050E00F940B1A273031054105510549
:1096E00051F48FE69FE00E94C8329C01812F67EE03
:1096F00070E24EE309C08FE69FE00E94C8329C01F1
:10970000812F67EE70E240E26FDBFF2011F40C94D2
:109710003E54609112087091130880911408909142
:10972000150825E030E040E050E00F940B1A273098
:1097300031054105510511F00C943E540E947D38CD
:109740008091B1039091B20390931D0880931C08FF
:10975000809112089091130890931F0880931E081F
:1097600082E08093B30389E297E79093B2038093FA
:10977000B10380EE90E290932108809320088FE659
:109780009FE0909323088093220881E090E0A0E07E
:10979000B0E08093240890932508A0932608B09306
:1097A000270887EE93E0A0E0B0E08093280890932C
:1097B0002908A0932A08B0932B0860916F0F70912D
:1097C000700F8091710F9091720F0C943354083088
:1097D00009F08CC08091B303882339F1609112089D
:1097E00070911308809114089091150825E030E0DD
:1097F00040E050E00F940B1A283031054105510527
:1098000051F483E79FE00E94C8329C01812F69EDEB
:1098100070E24EE309C083E79FE00E94C8329C01DA
:10982000812F69ED70E240E2DFDAFF2011F40C9441
:109830003E54609112087091130880911408909121
:10984000150825E030E040E050E00F940B1A283076
:1098500031054105510511F00C943E540E947D38AC
:109860008091B1039091B20390931D0880931C08DE
:10987000809112089091130890931F0880931E08FE
:1098800082E08093B30389E297E79093B2038093D9
:10989000B10382ED90E2909321088093200883E742
:1098A0009FE0909323088093220881E090E0A0E05D
:1098B000B0E08093240890932508A0932608B093E5
:1098C000270887EE93E0A0E0B0E08093280890930B
:1098D0002908A0932A08B0932B086091730F709108
:1098E000740F8091750F9091760FBDC7093009F004
:1098F0008AC08091B303882339F160911208709176
:109900001308809114089091150825E030E040E09C
:1099100050E00F940B1A293031054105510551F4DF
:1099200087E79FE00E94C8329C01812F6BEC70E2B8
:109930004EE309C087E79FE00E94C8329C01812F57
:109940006BEC70E240E250DAFF2009F497C76091B7
:10995000120870911308809114089091150825E061
:1099600030E040E050E00F940B1A293031054105FA
:10997000510509F083C70E947D388091B103909111
:10998000B20390931D0880931C0880911208909157
:10999000130890931F0880931E0882E08093B303FE
:1099A00089E297E79093B2038093B10384EC90E24D
:1099B000909321088093200887E79FE090932308E5
:1099C0008093220881E090E0A0E0B0E0809324083A
:1099D00090932508A0932608B093270887EE93E07C
:1099E000A0E0B0E08093280890932908A0932A086B
:1099F000B0932B086091770F7091780F8091790F59
:109A000090917A0F30C70A3009F086C08091B30375
:109A1000882339F16091120870911308809114081D
:109A20009091150825E030E040E050E00F940B1ACB
:109A30002A3031054105510551F48FE99FE00E941C
:109A4000C8329C01812F6FEB70E24EE309C08FE9B1
:109A50009FE00E94C8329C01812F6FEB70E240E2D0
:109A6000C3D9FF2009F40AC7609112087091130846
:109A7000809114089091150825E030E040E050E016
:109A80000F940B1A2A3031054105510509F0F6C62D
:109A90000E947D388091B1039091B20390931D088C
:109AA00080931C08809112089091130890931F08CE
:109AB00080931E0882E08093B30389E297E7909336
:109AC000B2038093B1038AEB90E2909321088093D4
:109AD00020088FE99FE0909323088093220810923A
:109AE000240810922508109226081092270887EE65
:109AF00093E0A0E0B0E08093280890932908A09319
:109B00002A08B0932B0860919F0F7091A00F80914D
:109B1000A10F9091A20FA7C60B3009F086C08091CB
:109B2000B303882339F16091120870911308809172
:109B300014089091150825E030E040E050E00F94C3
:109B40000B1A2B3031054105510551F487EB9FE08D
:109B50000E94C8329C01812F60EB70E24EE309C085
:109B600087EB9FE00E94C8329C01812F60EB70E27E
:109B700040E23AD9FF2009F481C660911208709141
:109B80001308809114089091150825E030E040E01A
:109B900050E00F940B1A2B3031054105510509F0A7
:109BA0006DC60E947D388091B1039091B20390936D
:109BB0001D0880931C0880911208909113089093BF
:109BC0001F0880931E0882E08093B30389E297E721
:109BD0009093B2038093B10386EA90E290932108B8
:109BE0008093200887EB9FE09093230880932208BE
:109BF0001092240810922508109226081092270827
:109C000087EE93E0A0E0B0E08093280890932908C5
:109C1000A0932A08B0932B086091B70F7091B80FEA
:109C20008091B90F9091BA0F1EC60C3009F0A7C0F1
:109C30008091B303882309F443C0609112087091A6
:109C40001308809114089091150825E030E040E059
:109C500050E00F940B1A2C30310541055105C1F429
:109C600060918F0F7091900F8091910F9091920F52
:109C70000F94B31669837A838B839C83CE010196FC
:109C80000E94DF329C01812F6FE970E24EE317C022
:109C900060918F0F7091900F8091910F9091920F22
:109CA0000F94B3166D837E838F839887CE010596BC
:109CB0000E94DF329C01812F6FE970E240E294D86C
:109CC000FF2009F4DBC560911208709113088091A0
:109CD00014089091150825E030E040E050E00F9422
:109CE0000B1A2C3031054105510509F0C7C50E94FA
:109CF0007D388091B1039091B20390931D088093B9
:109D00001C08809112089091130890931F0880936B
:109D10001E0882E08093B3038BE493E79093B20331
:109D20008093B10388E990E2909321088093200802
:109D30008FE89FE0909323088093220881E090E0D1
:109D4000A0E0B0E08093240890932508A093260813
:109D5000B09327088EED93E0A0E0B0E08093280850
:109D600090932908A0932A08B0932B0860918F0F35
:109D70007091900F8091910F9091920FFAC10D30D8
:109D800009F0A6C08091B303882309F442C0609112
:109D9000120870911308809114089091150825E01D
:109DA00030E040E050E00F940B1A2D3031054105B2
:109DB0005105B9F46091930F7091940F8091950FB4
:109DC0009091960F0F94B31669877A878B879C873B
:109DD000C1010E94DF329C01812F61E970E24EE3F4
:109DE00016C06091930F7091940F8091950F909190
:109DF000960F0F94B3166D877E878F87988BC2015D
:109E00000E94DF329C01812F61E970E240E20E94F2
:109E1000F446FF2009F432C56091120870911308CE
:109E2000809114089091150825E030E040E050E062
:109E30000F940B1A2D3031054105510509F01EC54F
:109E40000E947D388091B1039091B20390931D08D8
:109E500080931C08809112089091130890931F081A
:109E600080931E0882E08093B3038BE493E7909382
:109E7000B2038093B1038AE890E290932108809323
:109E8000200883E99FE0909323088093220881E0D3
:109E900090E0A0E0B0E08093240890932508A09380
:109EA0002608B09327088EED93E0A0E0B0E0809301
:109EB000280890932908A0932A08B0932B08609152
:109EC000930F7091940F8091950F9091960F51C1BF
:109ED0000E3009F0A6C08091B303882309F442C074
:109EE00060911208709113088091140890911508E0
:109EF00025E030E040E050E00F940B1A2E303105A1
:109F000041055105B9F46091970F7091980F8091B8
:109F1000990F90919A0F0F94B316698B7A8B8B8B54
:109F20009C8BC3010E94DF329C01812F63E870E2A9
:109F30004EE316C06091970F7091980F8091990F22
:109F400090919A0F0F94B3166D8B7E8B8F8B988F99
:109F5000C4010E94DF329C01812F63E870E240E27D
:109F60000E94F446FF2009F489C4609112087091A0
:109F70001308809114089091150825E030E040E026
:109F800050E00F940B1A2E3031054105510509F0B0
:109F900075C40E947D388091B1039091B203909373
:109FA0001D0880931C0880911208909113089093CB
:109FB0001F0880931E0882E08093B3038BE493E72D
:109FC0009093B2038093B1038CE790E290932108C1
:109FD0008093200887E99FE09093230880932208CC
:109FE00081E090E0A0E0B0E0809324089093250801
:109FF000A0932608B09327088EED93E0A0E0B0E090
:10A000008093280890932908A0932A08B0932B08DE
:10A010006091970F7091980F8091990F90919A0F7E
:10A02000A8C00F3009F0BEC08091B303882309F4A3
:10A0300042C06091120870911308809114089091A9
:10A04000150825E030E040E050E00F940B1A2F3067
:10A05000310541055105B9F460919B0F70919C0F3A
:10A0600080919D0F90919E0F0F94B316698F7A8FF8
:10A070008B8F9C8FC5010E94DF329C01812F65E789
:10A0800070E24EE316C060919B0F70919C0F80911F
:10A090009D0F90919E0F0F94B3166D8F7E8F8F8FB3
:10A0A00098A3C6010E94DF329C01812F65E770E210
:10A0B00040E20E94F446FF2009F4E0C360911208D8
:10A0C00070911308809114089091150825E030E0F4
:10A0D00040E050E00F940B1A2F3031054105510537
:10A0E00009F0CCC30E947D388091B1039091B203F6
:10A0F00090931D0880931C0880911208909113087A
:10A1000090931F0880931E0882E08093B3038BE432
:10A1100093E79093B2038093B1038EE690E290931D
:10A120002108809320088BE99FE090932308809377
:10A13000220881E090E0A0E0B0E0809324089093B2
:10A140002508A0932608B09327088EED93E0A0E0A1
:10A15000B0E08093280890932908A0932A08B09330
:10A160002B0860919B0F70919C0F80919D0F909197
:10A170009E0F0F94B3162AE037ED43E25CE30F9491
:10A18000F3180F9487166093120870931308809346
:10A1900014089093150889ED93EF90932D08809300
:10A1A0002C08ABC3003109F08FC08091B303882322
:10A1B00041F16091120870911308809114089091F8
:10A1C000150825E030E040E050E00F940B1A2031F4
:10A1D00031054105510551F487EA9FE00E94DF32C5
:10A1E0009C01812F64E670E24EE309C087EA9FE09C
:10A1F0000E94DF329C01812F64E670E240E20E94FF
:10A20000F446FF2009F43AC36091120870911308D4
:10A21000809114089091150825E030E040E050E06E
:10A220000F940B1A203131054105510509F026C361
:10A230000E947D388091B1039091B20390931D08E4
:10A2400080931C08809112089091130890931F0826
:10A2500080931E0882E08093B30383EE95E790938A
:10A26000B2038093B1038AE590E290932108809332
:10A27000200887EA9FE0909323088093220881E0DA
:10A2800090E0A0E0B0E08093240890932508A0938C
:10A290002608B09327088EED93E0A0E0B0E080930D
:10A2A000280890932908A0932A08B0932B0860915E
:10A2B000A70F7091A80F8091A90F9091AA0F2AE083
:10A2C00037ED43E25CE3CDC2013109F08BC08091F0
:10A2D000B303882341F160911208709113088091B3
:10A2E00014089091150825E030E040E050E00F940C
:10A2F0000B1A213131054105510551F48BE79FE0DF
:10A300000E940E349C01812F60E570E24EE309C08B
:10A310008BE79FE00E940E349C01812F60E570E284
:10A3200040E20E94F446FF2009F4A8C2609112089E
:10A3300070911308809114089091150825E030E081
:10A3400040E050E00F940B1A2131310541055105D1
:10A3500009F094C20E947D388091B1039091B203BC
:10A3600090931D0880931C08809112089091130807
:10A3700090931F0880931E0882E08093B3038DE9B9
:10A3800094E79093B2038093B10386E490E29093B4
:10A390002108809320088BE79FE090932308809307
:10A3A000220884EF91E0A0E0B0E08093240890932D
:10A3B0002508A0932608B09327088CED91E4AFE020
:10A3C000B0E08093280890932908A0932A08B093BE
:10A3D0002B0860917B0F70917C0F80917D0F909185
:10A3E0007E0F8DC0023109F08FC08091B3038823A6
:10A3F00041F16091120870911308809114089091B6
:10A40000150825E030E040E050E00F940B1A2231AF
:10A4100031054105510551F48FE79FE00E940E344C
:10A420009C01812F6CE370E24EE309C08FE79FE04F
:10A430000E940E349C01812F6CE370E240E20E9486
:10A44000F446FF2009F41AC26091120870911308B3
:10A45000809114089091150825E030E040E050E02C
:10A460000F940B1A223131054105510509F006C23E
:10A470000E947D388091B1039091B20390931D08A2
:10A4800080931C08809112089091130890931F08E4
:10A4900080931E0882E08093B3038DE994E7909344
:10A4A000B2038093B10382E390E2909321088093FA
:10A4B00020088FE79FE0909323088093220884EF81
:10A4C00091E0A0E0B0E08093240890932508A09349
:10A4D0002608B09327088CED91E4AFE0B0E08093BC
:10A4E000280890932908A0932A08B0932B0860911C
:10A4F0007F0F7091800F8091810F9091820F20E0EB
:10A5000030E048EC52E4ADC1033109F08BC08091DA
:10A51000B303882341F16091120870911308809170
:10A5200014089091150825E030E040E050E00F94C9
:10A530000B1A233131054105510551F483E89FE0A1
:10A540000E9487339C01812F68E270E24EE309C0CC
:10A5500083E89FE00E9487339C01812F68E270E2CC
:10A5600040E20E94F446FF2009F488C1609112087D
:10A5700070911308809114089091150825E030E03F
:10A5800040E050E00F940B1A23313105410551058D
:10A5900009F074C10E947D388091B1039091B2039B
:10A5A00090931D0880931C088091120890911308C5
:10A5B00090931F0880931E0882E08093B30380E489
:10A5C00095E79093B2038093B1038EE190E290936C
:10A5D00021088093200883E89FE0909323088093CC
:10A5E000220882E390E0A0E0B0E0809324089093FA
:10A5F0002508A0932608B093270886E996E8A1E0ED
:10A60000B0E08093280890932908A0932A08B0937B
:10A610002B086091830F7091840F8091850F90912A
:10A62000860F1BC1043109F08BC08091B3038823CE
:10A6300041F1609112087091130880911408909173
:10A64000150825E030E040E050E00F940B1A24316B
:10A6500031054105510551F487E89FE00E94873399
:10A660009C01812F64E170E24EE309C087E89FE01E
:10A670000E9487339C01812F64E170E240E20E94D6
:10A68000F446FF2009F4FAC0609112087091130893
:10A69000809114089091150825E030E040E050E0EA
:10A6A0000F940B1A243131054105510509F0E6C01C
:10A6B0000E947D388091B1039091B20390931D0860
:10A6C00080931C08809112089091130890931F08A2
:10A6D00080931E0882E08093B30380E495E7909313
:10A6E000B2038093B1038AE090E2909321088093B3
:10A6F000200887E89FE0909323088093220882E354
:10A7000090E0A0E0B0E08093240890932508A09307
:10A710002608B093270886E996E8A1E0B0E0809388
:10A72000280890932908A0932A08B0932B086091D9
:10A73000870F7091880F8091890F90918A0F8DC03B
:10A74000053109F09BC08091B303882341F16091EA
:10A75000120870911308809114089091150825E053
:10A7600030E040E050E00F940B1A253131054105EF
:10A77000510551F48BE89FE00E9487339C01812FA3
:10A7800060E070E24EE309C08BE89FE00E948733EF
:10A790009C01812F60E070E240E20E94F446FF20BD
:10A7A00009F46CC06091120870911308809114082C
:10A7B0009091150825E030E040E050E00F940B1A2E
:10A7C000253131054105510509F058C00E947D38F9
:10A7D0008091B1039091B20390931D0880931C085F
:10A7E000809112089091130890931F0880931E087F
:10A7F00082E08093B30380E495E79093B203809363
:10A80000B10386EF9FE190932108809320088BE8A5
:10A810009FE0909323088093220882E390E0A0E0D9
:10A82000B0E08093240890932508A0932608B09365
:10A83000270886E996E8A1E0B0E080932808909385
:10A840002908A0932A08B0932B0860918B0F709170
:10A850008C0F80918D0F90918E0F20E030E040E2C0
:10A8600051E40F94F3180F948716609312087093B5
:10A87000130880931408909315083FC08091120824
:10A8800090911308A0911408B09115088E36910587
:10A89000A105B10560F08DE690E0A0E0B0E0809306
:10A8A000120890931308A0931408B09315086091B0
:10A8B000120870911308809114089091150825E0F2
:10A8C00030E040E050E00F940B1A422F80910C08CA
:10A8D00090E0049630E0821793074CF44450409384
:10A8E0000C0881E08093B303042F01501FEF1F5F1A
:10A8F000153018F40F5F0C94B447A0960FB6F89477
:10A90000DEBF0FBECDBFCF91DF911F910F91FF90A2
:10A91000EF90DF90CF90BF90AF909F908F907F90FF
:10A920006F905F904F903F902F900895AF92BF929D
:10A93000CF92DF92EF92FF920F931F9380911208B4
:10A9400090911308A0911408B09115088150904877
:10A95000A040B04040F010921208109213081092DC
:10A9600014081092150860911208709113088091D4
:10A9700014089091150825E030E040E050E00F9475
:10A980000B1A79018A0180910C0890E0A0E0B0E0F8
:10A99000E816F9060A071B0710F420930C0800912B
:10A9A0000C0880910B0890E0969587959695879571
:10A9B000FF24F394F82210E038E1A32EB12CC12C2F
:10A9C000D12CEE24E394002309F03DC08091B30321
:10A9D0008823C1F08091120890911308A091140867
:10A9E000B09115080597A105B10528F4812F68E1FC
:10A9F00073E24BEF04C0812F68E173E240E22BEF7A
:10AA00000E940C35FF2009F4FBC18091120890913F
:10AA10001308A0911408B09115080597A105B10578
:10AA200008F0EEC10E947D3880E998E79093B20368
:10AA30008093B10310921208109213081092140818
:10AA40001092150815C2013009F083C08091B3033C
:10AA5000882341F1609112087091130880911408C5
:10AA60009091150825E030E040E050E00F940B1A7B
:10AA7000213031054105510551F48AEC95E00E94E1
:10AA800093329C01812F6EE073E24EE309C08AECA1
:10AA900095E00E9493329C01812F6EE073E240E2C8
:10AAA0000E94F446FF2009F4ABC160911208709136
:10AAB0001308809114089091150825E030E040E0DB
:10AAC00050E00F940B1A213031054105510509F072
:10AAD00097C10E947D388091B1039091B203909309
:10AAE0001D0880931C088091120890911308909380
:10AAF0001F0880931E0882E08093B30380EC97E7E1
:10AB00009093B2038093B10384E093E29093210881
:10AB1000809320088AEC95E0909323088093220884
:10AB200010922408109225081092260810922708E7
:10AB30008FEF90E0A0E0B0E0809328089093290880
:10AB4000A0932A08B0932B088091CA059091CB0559
:10AB50000BC1023009F083C08091B303882341F117
:10AB60006091120870911308809114089091150853
:10AB700025E030E040E050E00F940B1A2230310520
:10AB80004105510551F486EC95E00E9493329C01F9
:10AB9000812F6DEF72E24EE309C086EC95E00E94D2
:10ABA00093329C01812F6DEF72E240E20E94F446E5
:10ABB000FF2009F425C1609112087091130880915B
:10ABC00014089091150825E030E040E050E00F9423
:10ABD0000B1A223031054105510509F011C10E94BF
:10ABE0007D388091B1039091B20390931D088093BA
:10ABF0001C08809112089091130890931F0880936D
:10AC00001E0882E08093B30380EC97E79093B20331
:10AC10008093B10386EF92E29093210880932008FD
:10AC200086EC95E0909323088093220810922408E4
:10AC300010922508109226081092270882E291E0CF
:10AC4000A0E0B0E08093280890932908A0932A08F8
:10AC5000B0932B088091C6059091C70585C003303D
:10AC600009F08FC08091B303882341F160911208ED
:10AC700070911308809114089091150825E030E038
:10AC800040E050E00F940B1A233031054105510587
:10AC900051F488EC95E00E9493329C01812F62EF81
:10ACA00072E24EE309C088EC95E00E9493329C0169
:10ACB000812F62EF72E240E20E94F446FF2009F425
:10ACC0009FC06091120870911308809114089091B0
:10ACD000150825E030E040E050E00F940B1A2330D7
:10ACE00031054105510509F08BC00E947D388091E6
:10ACF000B1039091B20390931D0880931C0880913A
:10AD000012089091130890931F0880931E0882E008
:10AD10008093B30380EC97E79093B2038093B103E1
:10AD20008EEE92E2909321088093200888EC95E0C3
:10AD300090932308809322081092240810922508EB
:10AD4000109226081092270887E890E0A0E0B0E073
:10AD50008093280890932908A0932A08B0932B0881
:10AD60008091C8059091C905AA2797FDA095BA2F93
:10AD70008093120890931308A0931408B0931508B9
:10AD800077C00430E9F58091B3038823F9F060912E
:10AD9000120870911308809114089091150825E00D
:10ADA00030E040E050E00F940B1A243031054105AB
:10ADB000510529F4812F61EE72E24EE304C0812F28
:10ADC00061EE72E240E220E20E940C35FF20C1F009
:10ADD00060911208709113088091140890911508E1
:10ADE00025E030E040E050E00F940B1A24303105AC
:10ADF0004105510529F40E947D380E94D98E38C042
:10AE00008091120890911308A0911408B091150830
:10AE10004997A105B10540F0A0921208B09213081D
:10AE2000C0921408D092150860911208709113080E
:10AE3000809114089091150825E030E040E050E042
:10AE40000F940B1A422F80910C0890E0049630E08A
:10AE50008217930744F4445040930C08E092B303E4
:10AE6000042F01501FEF1F5F153010F40F5FABCDA3
:10AE70001F910F91FF90EF90DF90CF90BF90AF9018
:10AE80000895AF92BF92CF92DF92EF92FF920F930D
:10AE90001F938091120890911308A0911408B0910B
:10AEA000150881509048A040B04040F01092120820
:10AEB000109213081092140810921508609112084D
:10AEC00070911308809114089091150825E030E0E6
:10AED00040E050E00F940B1A79018A0180910C0830
:10AEE00090E0A0E0B0E0E816F9060A071B0710F4AE
:10AEF00020930C0800910C0880910B0890E0969527
:10AF0000879596958795FF24F394F82210E058E1F1
:10AF1000A52EB12CC12CD12CEE24E394002309F0F2
:10AF20003DC08091B3038823C1F0809112089091B5
:10AF30001308A0911408B09115080597A105B10553
:10AF400028F4812F6BE573E24BEF04C0812F6BE592
:10AF500073E240E22BEF0E940C35FF2009F4FBC1A5
:10AF60008091120890911308A0911408B0911508CF
:10AF70000597A105B10508F0EEC10E947D3880E972
:10AF800098E79093B2038093B10310921208109245
:10AF90001308109214081092150815C2013009F018
:10AFA00083C08091B303882341F1609112087091AE
:10AFB0001308809114089091150825E030E040E0D6
:10AFC00050E00F940B1A213031054105510551F421
:10AFD00084EC95E00E9493329C01812F61E573E23D
:10AFE0004EE309C084EC95E00E9493329C01812FCE
:10AFF00061E573E240E20E94F446FF2009F4ABC130
:10B0000060911208709113088091140890911508AE
:10B0100025E030E040E050E00F940B1A213031057C
:10B020004105510509F097C10E947D388091B10317
:10B030009091B20390931D0880931C088091120890
:10B040009091130890931F0880931E0882E08093CC
:10B05000B30380EC97E79093B2038093B10387E446
:10B0600093E2909321088093200884EC95E09093DC
:10B070002308809322081092240810922508109229
:10B080002608109227088FEF90E0A0E0B0E08093B0
:10B09000280890932908A0932A08B0932B08809140
:10B0A000C4059091C5050BC1023009F083C08091A1
:10B0B000B303882341F160911208709113088091C5
:10B0C00014089091150825E030E040E050E00F941E
:10B0D0000B1A223031054105510551F480EC95E001
:10B0E0000E9493329C01812F60E473E24EE309C019
:10B0F00080EC95E00E9493329C01812F60E473E222
:10B1000040E20E94F446FF2009F425C16091120834
:10B1100070911308809114089091150825E030E093
:10B1200040E050E00F940B1A2230310541055105E3
:10B1300009F011C10E947D388091B1039091B20352
:10B1400090931D0880931C08809112089091130819
:10B1500090931F0880931E0882E08093B30380ECD5
:10B1600097E79093B2038093B10389E393E29093BE
:10B1700021088093200880EC95E090932308809329
:10B180002208109224081092250810922608109286
:10B19000270882E291E0A0E0B0E080932808909335
:10B1A0002908A0932A08B0932B088091C00590919C
:10B1B000C10585C0033009F08FC08091B303882397
:10B1C00041F16091120870911308809114089091D8
:10B1D000150825E030E040E050E00F940B1A2330D2
:10B1E00031054105510551F482EC95E00E949332FE
:10B1F0009C01812F65E373E24EE309C082EC95E088
:10B200000E9493329C01812F65E373E240E20E9429
:10B21000F446FF2009F49FC0609112087091130852
:10B22000809114089091150825E030E040E050E04E
:10B230000F940B1A233031054105510509F08BC0DD
:10B240000E947D388091B1039091B20390931D08C4
:10B2500080931C08809112089091130890931F0806
:10B2600080931E0882E08093B30380EC97E790936D
:10B27000B2038093B10381E393E29093210880931A
:10B28000200882EC95E09093230880932208109286
:10B29000240810922508109226081092270887E8A3
:10B2A00090E0A0E0B0E08093280890932908A09354
:10B2B0002A08B0932B088091C2059091C305AA2754
:10B2C00097FDA095BA2F8093120890931308A0932E
:10B2D0001408B093150877C00430E9F58091B303E2
:10B2E0008823F9F060911208709113088091140876
:10B2F0009091150825E030E040E050E00F940B1AE3
:10B30000243031054105510529F4812F64E273E2AF
:10B310004EE304C0812F64E273E240E220E20E9427
:10B320000C35FF20C1F060911208709113088091D4
:10B3300014089091150825E030E040E050E00F94AB
:10B340000B1A243031054105510529F40E947D383E
:10B350000E94D98E38C08091120890911308A09154
:10B360001408B09115084997A105B10540F0A092C5
:10B370001208B0921308C0921408D0921508609178
:10B38000120870911308809114089091150825E017
:10B3900030E040E050E00F940B1A422F80910C08EF
:10B3A00090E0049630E08217930744F444504093B1
:10B3B0000C08E092B303042F01501FEF1F5F1530FC
:10B3C00010F40F5FABCD1F910F91FF90EF90DF90C6
:10B3D000CF90BF90AF900895AF92BF92CF92DF927F
:10B3E000EF92FF920F931F93809112089091130890
:10B3F000A0911408B091150881509048A040B04029
:10B4000040F0109212081092130810921408109233
:10B41000150860911208709113088091140890919A
:10B42000150825E030E040E050E00F940B1A790158
:10B430008A0180910C0890E0A0E0B0E0E816F906DF
:10B440000A071B0710F420930C0800910C08809148
:10B450000B0890E09695879596958795FF24F39431
:10B46000F82210E078E1A72EB12CC12CD12CEE24CB
:10B47000E394002309F03DC08091B3038823C1F019
:10B480008091120890911308A0911408B0911508AA
:10B490000597A105B10528F4812F6EE973E24BEF02
:10B4A00004C0812F6EE973E240E22BEF0E940C355D
:10B4B000FF2009F4FBC18091120890911308A0911C
:10B4C0001408B09115080597A105B10508F0EEC163
:10B4D0000E947D3880E998E79093B2038093B1038E
:10B4E0001092120810921308109214081092150866
:10B4F00015C2013009F083C08091B303882341F164
:10B5000060911208709113088091140890911508A9
:10B5100025E030E040E050E00F940B1A2130310577
:10B520004105510551F488EB95E00E9493329C014E
:10B53000812F64E973E24EE309C088EB95E00E9435
:10B5400093329C01812F64E973E240E20E94F44649
:10B55000FF2009F4ABC1609112087091130880912B
:10B5600014089091150825E030E040E050E00F9479
:10B570000B1A213031054105510509F097C10E9490
:10B580007D388091B1039091B20390931D08809310
:10B590001C08809112089091130890931F088093C3
:10B5A0001E0882E08093B30380EC97E79093B20388
:10B5B0008093B1038AE893E2909321088093200856
:10B5C00088EB95E09093230880932208109224083A
:10B5D0001092250810922608109227088FEF90E00D
:10B5E000A0E0B0E08093280890932908A0932A084F
:10B5F000B0932B088091B8059091B9050BC102302A
:10B6000009F083C08091B303882341F1609112084F
:10B6100070911308809114089091150825E030E08E
:10B6200040E050E00F940B1A2230310541055105DE
:10B6300051F484EB95E00E9493329C01812F63E8E2
:10B6400073E24EE309C084EB95E00E9493329C01C3
:10B65000812F63E873E240E20E94F446FF2009F480
:10B6600025C160911208709113088091140890917F
:10B67000150825E030E040E050E00F940B1A22302E
:10B6800031054105510509F011C10E947D388091B5
:10B69000B1039091B20390931D0880931C08809190
:10B6A00012089091130890931F0880931E0882E05F
:10B6B0008093B30380EC97E79093B2038093B10338
:10B6C0008CE793E2909321088093200884EB95E027
:10B6D0009093230880932208109224081092250842
:10B6E000109226081092270882E291E0A0E0B0E0D4
:10B6F0008093280890932908A0932A08B0932B08D8
:10B700008091B4059091B50585C0033009F08FC0D4
:10B710008091B303882341F160911208709113085E
:10B72000809114089091150825E030E040E050E049
:10B730000F940B1A233031054105510551F486EB66
:10B7400095E00E9493329C01812F68E773E24EE3FB
:10B7500009C086EB95E00E9493329C01812F68E737
:10B7600073E240E20E94F446FF2009F49FC060911A
:10B77000120870911308809114089091150825E023
:10B7800030E040E050E00F940B1A233031054105C2
:10B79000510509F08BC00E947D388091B1039091D2
:10B7A000B20390931D0880931C0880911208909119
:10B7B000130890931F0880931E0882E08093B303C0
:10B7C00080EC97E79093B2038093B10384E793E210
:10B7D000909321088093200886EB95E090932308AE
:10B7E00080932208109224081092250810922608AF
:10B7F0001092270887E890E0A0E0B0E08093280846
:10B8000090932908A0932A08B0932B088091B6053D
:10B810009091B705AA2797FDA095BA2F809312089B
:10B8200090931308A0931408B093150877C00430C0
:10B83000E9F58091B3038823F9F0609112087091C3
:10B840001308809114089091150825E030E040E03D
:10B8500050E00F940B1A243031054105510529F4AD
:10B86000812F67E673E24EE304C0812F67E673E23F
:10B8700040E220E20E940C35FF20C1F060911208E6
:10B8800070911308809114089091150825E030E01C
:10B8900040E050E00F940B1A24303105410551056A
:10B8A00029F40E947D380E94D98E38C080911208F8
:10B8B00090911308A0911408B09115084997A1051B
:10B8C000B10540F0A0921208B0921308C09214087B
:10B8D000D092150860911208709113088091140895
:10B8E0009091150825E030E040E050E00F940B1AED
:10B8F000422F80910C0890E0049630E08217930765
:10B9000044F4445040930C08E092B303042F0150D8
:10B910001FEF1F5F153010F40F5FABCD1F910F911C
:10B92000FF90EF90DF90CF90BF90AF900895AF92CF
:10B93000BF92CF92DF92EF92FF920F931F9380916D
:10B94000120890911308A0911408B0911508815025
:10B950009048A040B04040F0109212081092130896
:10B960001092140810921508609112087091130833
:10B97000809114089091150825E030E040E050E0F7
:10B980000F940B1A79018A0180910C0890E0A0E0D5
:10B99000B0E0E816F9060A071B0710F420930C081C
:10B9A00000910C0880910B0890E0969587959695EC
:10B9B0008795FF24F394F82210E0F8E1AF2EB12C24
:10B9C000C12CD12CEE24E394002309F03DC08091DA
:10B9D000B3038823C1F08091120890911308A091BD
:10B9E0001408B09115080597A105B10528F4812F19
:10B9F00061EE73E24BEF04C0812F61EE73E240E22F
:10BA00002BEF0E940C35FF2009F4FBC18091120836
:10BA100090911308A0911408B09115080597A105FD
:10BA2000B10508F0EEC10E947D3880E998E7909357
:10BA3000B2038093B103109212081092130810926F
:10BA400014081092150815C2013009F083C08091C6
:10BA5000B303882341F1609112087091130880911B
:10BA600014089091150825E030E040E050E00F9474
:10BA70000B1A213031054105510551F482EB95E057
:10BA80000E9493329C01812F67ED73E24EE309C05F
:10BA900082EB95E00E9493329C01812F67ED73E267
:10BAA00040E20E94F446FF2009F4ABC16091120805
:10BAB00070911308809114089091150825E030E0EA
:10BAC00040E050E00F940B1A21303105410551053B
:10BAD00009F097C10E947D388091B1039091B20323
:10BAE00090931D0880931C08809112089091130870
:10BAF00090931F0880931E0882E08093B30380EC2C
:10BB000097E79093B2038093B1038DEC93E2909307
:10BB100021088093200882EB95E09093230880937E
:10BB200022081092240810922508109226081092DC
:10BB300027088FEF90E0A0E0B0E080932808909372
:10BB40002908A0932A08B0932B088091B205909100
:10BB5000B3050BC1023009F083C08091B303882381
:10BB600041F160911208709113088091140890912E
:10BB7000150825E030E040E050E00F940B1A223029
:10BB800031054105510551F48EEA95E00E9493324A
:10BB90009C01812F66EC73E24EE309C08EEA95E0CA
:10BBA0000E9493329C01812F66EC73E240E20E9476
:10BBB000F446FF2009F425C1609112087091130822
:10BBC000809114089091150825E030E040E050E0A5
:10BBD0000F940B1A223031054105510509F011C1AE
:10BBE0000E947D388091B1039091B20390931D081B
:10BBF00080931C08809112089091130890931F085D
:10BC000080931E0882E08093B30380EC97E79093C3
:10BC1000B2038093B1038FEB93E29093210880935A
:10BC200020088EEA95E090932308809322081092D2
:10BC3000240810922508109226081092270882E204
:10BC400091E0A0E0B0E08093280890932908A093A9
:10BC50002A08B0932B088091AE059091AF0585C05E
:10BC6000033009F08FC08091B303882341F16091C4
:10BC7000120870911308809114089091150825E01E
:10BC800030E040E050E00F940B1A233031054105BD
:10BC9000510551F480EB95E00E9493329C01812F75
:10BCA0006BEB73E24EE309C080EB95E00E949332A8
:10BCB0009C01812F6BEB73E240E20E94F446FF206F
:10BCC00009F49FC0609112087091130880911408C4
:10BCD0009091150825E030E040E050E00F940B1AF9
:10BCE000233031054105510509F08BC00E947D3894
:10BCF0008091B1039091B20390931D0880931C082A
:10BD0000809112089091130890931F0880931E0849
:10BD100082E08093B30380EC97E79093B203809323
:10BD2000B10387EB93E2909321088093200880EB86
:10BD300095E0909323088093220810922408109293
:10BD40002508109226081092270887E890E0A0E0C6
:10BD5000B0E08093280890932908A0932A08B09314
:10BD60002B088091B0059091B105AA2797FDA09569
:10BD7000BA2F8093120890931308A0931408B093DD
:10BD8000150877C00430E9F58091B3038823F9F0F2
:10BD90006091120870911308809114089091150811
:10BDA00025E030E040E050E00F940B1A24303105DC
:10BDB0004105510529F4812F6AEA73E24EE304C07C
:10BDC000812F6AEA73E240E220E20E940C35FF20F4
:10BDD000C1F060911208709113088091140890913D
:10BDE000150825E030E040E050E00F940B1A2430B5
:10BDF00031054105510529F40E947D380E94D98EF4
:10BE000038C08091120890911308A0911408B09145
:10BE100015084997A105B10540F0A0921208B0920B
:10BE20001308C0921408D0921508609112087091FE
:10BE30001308809114089091150825E030E040E047
:10BE400050E00F940B1A422F80910C0890E004965A
:10BE500030E08217930744F4445040930C08E0927A
:10BE6000B303042F01501FEF1F5F153010F40F5F55
:10BE7000ABCD1F910F91FF90EF90DF90CF90BF90CF
:10BE8000AF900895AF92BF92CF92DF92EF92FF9260
:10BE90000F931F938091120890911308A09114089A
:10BEA000B091150881509048A040B04040F01092E9
:10BEB000120810921308109214081092150860913D
:10BEC000120870911308809114089091150825E0CC
:10BED00030E040E050E00F940B1A79018A01809124
:10BEE0000C0890E0A0E0B0E0E816F9060A071B078E
:10BEF00010F420930C0800910C0880910B0890E03E
:10BF00009695879596958795FF24F394F82210E0EF
:10BF1000B8E1AB2EB12CC12CD12CEE24E39400233C
:10BF200009F03DC08091B3038823C1F080911208CD
:10BF300090911308A0911408B09115080597A105D8
:10BF4000B10528F4812F64E274E24BEF04C0812F25
:10BF500064E274E240E22BEF0E940C35FF2009F40A
:10BF6000FBC18091120890911308A0911408B09120
:10BF700015080597A105B10508F0EEC10E947D38AE
:10BF800080E998E79093B2038093B103109212086E
:10BF900010921308109214081092150815C201305F
:10BFA00009F083C08091B303882341F160911208A6
:10BFB00070911308809114089091150825E030E0E5
:10BFC00040E050E00F940B1A213031054105510536
:10BFD00051F48CEA95E00E9493329C01812F6AE132
:10BFE00074E24EE309C08CEA95E00E9493329C0112
:10BFF000812F6AE174E240E20E94F446FF2009F4D6
:10C00000ABC160911208709113088091140890914F
:10C01000150825E030E040E050E00F940B1A213085
:10C0200031054105510509F097C10E947D38809185
:10C03000B1039091B20390931D0880931C088091E6
:10C0400012089091130890931F0880931E0882E0B5
:10C050008093B30380EC97E79093B2038093B1038E
:10C0600080E194E290932108809320088CEA95E087
:10C070009093230880932208109224081092250898
:10C0800010922608109227088FEF90E0A0E0B0E011
:10C090008093280890932908A0932A08B0932B082E
:10C0A0008091AC059091AD050BC1023009F083C0C1
:10C0B0008091B303882341F16091120870911308B5
:10C0C000809114089091150825E030E040E050E0A0
:10C0D0000F940B1A223031054105510551F488EABD
:10C0E00095E00E9493329C01812F69E074E24EE357
:10C0F00009C088EA95E00E9493329C01812F69E093
:10C1000074E240E20E94F446FF2009F425C16091E8
:10C11000120870911308809114089091150825E079
:10C1200030E040E050E00F940B1A22303105410519
:10C13000510509F011C10E947D388091B1039091A1
:10C14000B20390931D0880931C088091120890916F
:10C15000130890931F0880931E0882E08093B30316
:10C1600080EC97E79093B2038093B10382E094E26E
:10C17000909321088093200888EA95E09093230803
:10C180008093220810922408109225081092260805
:10C190001092270882E291E0A0E0B0E080932808A6
:10C1A00090932908A0932A08B0932B088091A805A2
:10C1B0009091A90585C0033009F08FC08091B30329
:10C1C000882341F16091120870911308809114083E
:10C1D0009091150825E030E040E050E00F940B1AF4
:10C1E000233031054105510551F48AEA95E00E945A
:10C1F00093329C01812F6EEF73E24EE309C08AEA0D
:10C2000095E00E9493329C01812F6EEF73E240E231
:10C210000E94F446FF2009F49FC0609112087091BB
:10C220001308809114089091150825E030E040E053
:10C2300050E00F940B1A233031054105510509F0E8
:10C240008BC00E947D388091B1039091B20390938E
:10C250001D0880931C0880911208909113089093F8
:10C260001F0880931E0882E08093B30380EC97E759
:10C270009093B2038093B1038AEF93E290932108E5
:10C28000809320088AEA95E09093230880932208FF
:10C290001092240810922508109226081092270860
:10C2A00087E890E0A0E0B0E0809328089093290808
:10C2B000A0932A08B0932B088091AA059091AB0512
:10C2C000AA2797FDA095BA2F809312089093130880
:10C2D000A0931408B093150877C00430E9F5809155
:10C2E000B3038823F9F060911208709113088091CC
:10C2F00014089091150825E030E040E050E00F94DC
:10C300000B1A243031054105510529F4812F6DEEBA
:10C3100073E24EE304C0812F6DEE73E240E220E24F
:10C320000E940C35FF20C1F0609112087091130833
:10C33000809114089091150825E030E040E050E02D
:10C340000F940B1A243031054105510529F40E9440
:10C350007D380E94D98E38C08091120890911308C0
:10C36000A0911408B09115084997A105B10540F0B6
:10C37000A0921208B0921308C0921408D092150827
:10C38000609112087091130880911408909115081B
:10C3900025E030E040E050E00F940B1A422F8091EE
:10C3A0000C0890E0049630E08217930744F4445060
:10C3B00040930C08E092B303042F01501FEF1F5F5E
:10C3C000153010F40F5FABCD1F910F91FF90EF90E0
:10C3D000DF90CF90BF90AF900895AF92BF92CF9271
:10C3E000DF92EF92FF920F931F938091120890912A
:10C3F0001308A0911408B091150881509048A040EE
:10C40000B04040F0109212081092130810921408D5
:10C410001092150860911208709113088091140809
:10C420009091150825E030E040E050E00F940B1AA1
:10C4300079018A0180910C0890E0A0E0B0E0E81654
:10C44000F9060A071B0710F420930C0800910C084A
:10C4500080910B0890E09695879596958795FF2497
:10C46000F394F82210E088E1A82EB12CC12CD12C35
:10C47000EE24E394002309F03DC08091B3038823A8
:10C48000C1F08091120890911308A0911408B09106
:10C4900015080597A105B10528F4812F67E674E218
:10C4A0004BEF04C0812F67E674E240E22BEF0E945D
:10C4B0000C35FF2009F4FBC18091120890911308FC
:10C4C000A0911408B09115080597A105B10508F0D1
:10C4D000EEC10E947D3880E998E79093B203809383
:10C4E000B1031092120810921308109214081092BF
:10C4F000150815C2013009F083C08091B303882369
:10C5000041F1609112087091130880911408909184
:10C51000150825E030E040E050E00F940B1A213080
:10C5200031054105510551F486EA95E00E949332A8
:10C530009C01812F6DE574E24EE309C086EA95E027
:10C540000E9493329C01812F6DE574E240E20E94CB
:10C55000F446FF2009F4ABC16091120870911308F2
:10C56000809114089091150825E030E040E050E0FB
:10C570000F940B1A213031054105510509F097C17F
:10C580000E947D388091B1039091B20390931D0871
:10C5900080931C08809112089091130890931F08B3
:10C5A00080931E0882E08093B30380EC97E790931A
:10C5B000B2038093B10383E594E2909321088093C2
:10C5C000200886EA95E09093230880932208109231
:10C5D00024081092250810922608109227088FEF41
:10C5E00090E0A0E0B0E08093280890932908A09301
:10C5F0002A08B0932B088091A6059091A7050BC13E
:10C60000023009F083C08091B303882341F1609127
:10C61000120870911308809114089091150825E074
:10C6200030E040E050E00F940B1A22303105410514
:10C63000510551F482EA95E00E9493329C01812FCA
:10C640006CE474E24EE309C082EA95E00E94933202
:10C650009C01812F6CE474E240E20E94F446FF20CA
:10C6600009F425C160911208709113088091140893
:10C670009091150825E030E040E050E00F940B1A4F
:10C68000223031054105510509F011C10E947D3864
:10C690008091B1039091B20390931D0880931C0880
:10C6A000809112089091130890931F0880931E08A0
:10C6B00082E08093B30380EC97E79093B20380937A
:10C6C000B10385E494E2909321088093200882EAE4
:10C6D00095E09093230880932208109224081092EA
:10C6E0002508109226081092270882E291E0A0E027
:10C6F000B0E08093280890932908A0932A08B0936B
:10C700002B088091A2059091A30585C0033009F004
:10C710008FC08091B303882341F16091120870911A
:10C720001308809114089091150825E030E040E04E
:10C7300050E00F940B1A233031054105510551F497
:10C7400084EA95E00E9493329C01812F61E474E2B7
:10C750004EE309C084EA95E00E9493329C01812F48
:10C7600061E474E240E20E94F446FF2009F49FC0B5
:10C770006091120870911308809114089091150827
:10C7800025E030E040E050E00F940B1A23303105F3
:10C790004105510509F08BC00E947D388091B1039D
:10C7A0009091B20390931D0880931C088091120809
:10C7B0009091130890931F0880931E0882E0809345
:10C7C000B30380EC97E79093B2038093B1038DE3BA
:10C7D00094E2909321088093200884EA95E0909356
:10C7E00023088093220810922408109225081092A2
:10C7F00026081092270887E890E0A0E0B0E0809338
:10C80000280890932908A0932A08B0932B088091B8
:10C81000A4059091A505AA2797FDA095BA2F80930E
:10C82000120890931308A0931408B093150877C0CA
:10C830000430E9F58091B3038823F9F06091120880
:10C8400070911308809114089091150825E030E04C
:10C8500040E050E00F940B1A24303105410551059A
:10C8600029F4812F60E374E24EE304C0812F60E37A
:10C8700074E240E220E20E940C35FF20C1F060919A
:10C88000120870911308809114089091150825E002
:10C8900030E040E050E00F940B1A243031054105A0
:10C8A000510529F40E947D380E94D98E38C08091AC
:10C8B000120890911308A0911408B0911508499797
:10C8C000A105B10540F0A0921208B0921308C092E1
:10C8D0001408D09215086091120870911308809185
:10C8E00014089091150825E030E040E050E00F94E6
:10C8F0000B1A422F80910C0890E0049630E08217CA
:10C90000930744F4445040930C08E092B303042F7F
:10C9100001501FEF1F5F153010F40F5FABCD1F915B
:10C920000F91FF90EF90DF90CF90BF90AF90089560
:10C93000AF92BF92CF92DF92EF92FF920F931F932D
:10C940008091120890911308A0911408B0911508D5
:10C9500081509048A040B04040F0109212081092D0
:10C960001308109214081092150860911208709123
:10C970001308809114089091150825E030E040E0FC
:10C9800050E00F940B1A79018A0180910C0890E015
:10C99000A0E0B0E0E816F9060A071B0710F42093A0
:10C9A0000C0800910C0880910B0890E096958795F3
:10C9B00096958795FF24F394F82210E038E1A32E92
:10C9C000B12CC12CD12CEE24E394002309F03DC0FE
:10C9D0008091B3038823C1F08091120890911308CD
:10C9E000A0911408B09115080597A105B10528F488
:10C9F000812F6AEA74E24BEF04C0812F6AEA74E285
:10CA000040E22BEF0E940C35FF2009F4FBC180911E
:10CA1000120890911308A0911408B0911508059779
:10CA2000A105B10508F0EEC10E947D3880E998E7C4
:10CA30009093B2038093B1031092120810921308DE
:10CA4000109214081092150815C2013009F083C025
:10CA50008091B303882341F160911208709113080B
:10CA6000809114089091150825E030E040E050E0F6
:10CA70000F940B1A213031054105510551F480EA1C
:10CA800095E00E9493329C01812F60EA74E24EE3AC
:10CA900009C080EA95E00E9493329C01812F60EAF0
:10CAA00074E240E20E94F446FF2009F4ABC16091B9
:10CAB000120870911308809114089091150825E0D0
:10CAC00030E040E050E00F940B1A21303105410571
:10CAD000510509F097C10E947D388091B103909172
:10CAE000B20390931D0880931C08809112089091C6
:10CAF000130890931F0880931E0882E08093B3036D
:10CB000080EC97E79093B2038093B10386E994E2B7
:10CB1000909321088093200880EA95E09093230861
:10CB2000809322081092240810922508109226085B
:10CB3000109227088FEF90E0A0E0B0E080932808E3
:10CB400090932908A0932A08B0932B088091A00500
:10CB50009091A1050BC1023009F083C08091B3030D
:10CB6000882341F160911208709113088091140894
:10CB70009091150825E030E040E050E00F940B1A4A
:10CB8000223031054105510551F48CE995E00E94B0
:10CB900093329C01812F6FE874E24EE309C08CE967
:10CBA00095E00E9493329C01812F6FE874E240E28D
:10CBB0000E94F446FF2009F425C16091120870918B
:10CBC0001308809114089091150825E030E040E0AA
:10CBD00050E00F940B1A223031054105510509F040
:10CBE00011C10E947D388091B1039091B20390935E
:10CBF0001D0880931C08809112089091130890934F
:10CC00001F0880931E0882E08093B30380EC97E7AF
:10CC10009093B2038093B10388E894E29093210843
:10CC2000809320088CE995E0909323088093220854
:10CC300010922408109225081092260810922708B6
:10CC400082E291E0A0E0B0E0809328089093290868
:10CC5000A0932A08B0932B0880919C0590919D0584
:10CC600085C0033009F08FC08091B303882341F160
:10CC70006091120870911308809114089091150822
:10CC800025E030E040E050E00F940B1A23303105EE
:10CC90004105510551F48EE995E00E9493329C01C3
:10CCA000812F64E874E24EE309C08EE995E00E94AA
:10CCB00093329C01812F64E874E240E20E94F446C2
:10CCC000FF2009F49FC060911208709113088091B1
:10CCD00014089091150825E030E040E050E00F94F2
:10CCE0000B1A233031054105510509F08BC00E9414
:10CCF0007D388091B1039091B20390931D08809389
:10CD00001C08809112089091130890931F0880933B
:10CD10001E0882E08093B30380EC97E79093B20300
:10CD20008093B10380E894E29093210880932008D7
:10CD30008EE995E0909323088093220810922408AE
:10CD400010922508109226081092270887E890E094
:10CD5000A0E0B0E08093280890932908A0932A08C7
:10CD6000B0932B0880919E0590919F05AA2797FD6F
:10CD7000A095BA2F8093120890931308A0931408DB
:10CD8000B093150877C00430E9F58091B303882388
:10CD9000F9F0609112087091130880911408909135
:10CDA000150825E030E040E050E00F940B1A2430E5
:10CDB00031054105510529F4812F63E774E24EE303
:10CDC00004C0812F63E774E240E220E20E940C3548
:10CDD000FF20C1F06091120870911308809114082F
:10CDE0009091150825E030E040E050E00F940B1AD8
:10CDF000243031054105510529F40E947D380E94F7
:10CE0000D98E38C08091120890911308A09114080F
:10CE1000B09115084997A105B10540F0A0921208FC
:10CE2000B0921308C0921408D092150860911208AD
:10CE300070911308809114089091150825E030E056
:10CE400040E050E00F940B1A422F80910C0890E0C4
:10CE5000049630E08217930744F4445040930C0842
:10CE6000E092B303042F01501FEF1F5F153010F441
:10CE70000F5FABCD1F910F91FF90EF90DF90CF90A0
:10CE8000BF90AF900895AF92BF92CF92DF92EF9292
:10CE9000FF920F931F938091120890911308A09115
:10CEA0001408B091150881509048A040B04040F05F
:10CEB000109212081092130810921408109215087C
:10CEC00060911208709113088091140890911508D0
:10CED00025E030E040E050E00F940B1A79018A0120
:10CEE00080910C0890E0A0E0B0E0E816F9060A078F
:10CEF0001B0710F420930C0800910C0880910B087C
:10CF000090E09695879596958795FF24F394F8225F
:10CF100010E058E1A52EB12CC12CD12CEE24E394C5
:10CF2000002309F03DC08091B3038823C1F08091B4
:10CF3000120890911308A0911408B0911508059754
:10CF4000A105B10528F4812F6DEE74E24BEF04C00A
:10CF5000812F6DEE74E240E22BEF0E940C35FF2032
:10CF600009F4FBC18091120890911308A091140854
:10CF7000B09115080597A105B10508F0EEC10E9412
:10CF80007D3880E998E79093B2038093B1031092C3
:10CF9000120810921308109214081092150815C266
:10CFA000013009F083C08091B303882341F160917F
:10CFB000120870911308809114089091150825E0CB
:10CFC00030E040E050E00F940B1A2130310541056C
:10CFD000510551F48AE995E00E9493329C01812F1A
:10CFE00063EE74E24EE309C08AE995E00E94933251
:10CFF0009C01812F63EE74E240E20E94F446FF2020
:10D0000009F4ABC160911208709113088091140863
:10D010009091150825E030E040E050E00F940B1AA5
:10D02000213031054105510509F097C10E947D3835
:10D030008091B1039091B20390931D0880931C08D6
:10D04000809112089091130890931F0880931E08F6
:10D0500082E08093B30380EC97E79093B2038093D0
:10D06000B10389ED94E290932108809320088AE926
:10D0700095E0909323088093220810922408109240
:10D08000250810922608109227088FEF90E0A0E064
:10D09000B0E08093280890932908A0932A08B093C1
:10D0A0002B0880919A0590919B050BC1023009F0E5
:10D0B00083C08091B303882341F16091120870917D
:10D0C0001308809114089091150825E030E040E0A5
:10D0D00050E00F940B1A223031054105510551F4EF
:10D0E00086E995E00E9493329C01812F62ED74E203
:10D0F0004EE309C086E995E00E9493329C01812F9E
:10D1000062ED74E240E20E94F446FF2009F425C17A
:10D11000609112087091130880911408909115087D
:10D1200025E030E040E050E00F940B1A223031054A
:10D130004105510509F011C10E947D388091B1036C
:10D140009091B20390931D0880931C08809112085F
:10D150009091130890931F0880931E0882E080939B
:10D16000B30380EC97E79093B2038093B1038BEC09
:10D1700094E2909321088093200886E995E09093AB
:10D1800023088093220810922408109225081092F8
:10D1900026081092270882E291E0A0E0B0E0809398
:10D1A000280890932908A0932A08B0932B0880910F
:10D1B00096059091970585C0033009F08FC0809146
:10D1C000B303882341F16091120870911308809194
:10D1D00014089091150825E030E040E050E00F94ED
:10D1E0000B1A233031054105510551F488E995E0CA
:10D1F0000E9493329C01812F67EC74E24EE309C0D8
:10D2000088E995E00E9493329C01812F67EC74E2DB
:10D2100040E20E94F446FF2009F49FC0609112088A
:10D2200070911308809114089091150825E030E062
:10D2300040E050E00F940B1A2330310541055105B1
:10D2400009F08BC00E947D388091B1039091B203A8
:10D2500090931D0880931C088091120890911308E8
:10D2600090931F0880931E0882E08093B30380ECA4
:10D2700097E79093B2038093B10383EC94E2909389
:10D2800021088093200888E995E0909323088093F3
:10D290002208109224081092250810922608109255
:10D2A000270887E890E0A0E0B0E0809328089093FA
:10D2B0002908A0932A08B0932B0880919805909193
:10D2C0009905AA2797FDA095BA2F809312089093ED
:10D2D0001308A0931408B093150877C00430E9F53B
:10D2E0008091B3038823F9F06091120870911308BC
:10D2F000809114089091150825E030E040E050E05E
:10D300000F940B1A243031054105510529F4812F62
:10D3100066EB74E24EE304C0812F66EB74E240E2F8
:10D3200020E20E940C35FF20C1F06091120870913C
:10D330001308809114089091150825E030E040E032
:10D3400050E00F940B1A243031054105510529F4A2
:10D350000E947D380E94D98E38C080911208909129
:10D360001308A0911408B09115084997A105B105BB
:10D3700040F0A0921208B0921308C0921408D09204
:10D38000150860911208709113088091140890910B
:10D39000150825E030E040E050E00F940B1A422FD2
:10D3A00080910C0890E0049630E08217930744F4D3
:10D3B000445040930C08E092B303042F01501FEF38
:10D3C0001F5F153010F40F5FABCD1F910F91FF90D1
:10D3D000EF90DF90CF90BF90AF900895AF92BF9243
:10D3E000CF92DF92EF92FF920F931F9380911208DA
:10D3F00090911308A0911408B0911508815090489D
:10D40000A040B04040F01092120810921308109201
:10D4100014081092150860911208709113088091F9
:10D4200014089091150825E030E040E050E00F949A
:10D430000B1A79018A0180910C0890E0A0E0B0E01D
:10D44000E816F9060A071B0710F420930C08009150
:10D450000C0880910B0890E0969587959695879596
:10D46000FF24F394F82210E078E1A72EB12CC12C10
:10D47000D12CEE24E394002309F03DC08091B30346
:10D480008823C1F08091120890911308A09114088C
:10D49000B09115080597A105B10528F4812F60E327
:10D4A00075E24BEF04C0812F60E375E240E22BEFA1
:10D4B0000E940C35FF2009F4FBC180911208909165
:10D4C0001308A0911408B09115080597A105B1059E
:10D4D00008F0EEC10E947D3880E998E79093B2038E
:10D4E0008093B1031092120810921308109214083E
:10D4F0001092150815C2013009F083C08091B30362
:10D50000882341F1609112087091130880911408EA
:10D510009091150825E030E040E050E00F940B1AA0
:10D52000213031054105510551F484E995E00E940F
:10D5300093329C01812F66E275E24EE309C084E9D3
:10D5400095E00E9493329C01812F66E275E240E2F1
:10D550000E94F446FF2009F4ABC16091120870915B
:10D560001308809114089091150825E030E040E000
:10D5700050E00F940B1A213031054105510509F097
:10D5800097C10E947D388091B1039091B20390932E
:10D590001D0880931C0880911208909113089093A5
:10D5A0001F0880931E0882E08093B30380EC97E706
:10D5B0009093B2038093B1038CE195E2909321089C
:10D5C0008093200884E995E09093230880932208B3
:10D5D000109224081092250810922608109227080D
:10D5E0008FEF90E0A0E0B0E08093280890932908A6
:10D5F000A0932A08B0932B088091940590919505EB
:10D600000BC1023009F083C08091B303882341F13C
:10D610006091120870911308809114089091150878
:10D6200025E030E040E050E00F940B1A2230310545
:10D630004105510551F480E995E00E9493329C0127
:10D64000812F65E175E24EE309C080E995E00E9413
:10D6500093329C01812F65E175E240E20E94F4461D
:10D66000FF2009F425C16091120870911308809180
:10D6700014089091150825E030E040E050E00F9448
:10D680000B1A223031054105510509F011C10E94E4
:10D690007D388091B1039091B20390931D088093DF
:10D6A0001C08809112089091130890931F08809392
:10D6B0001E0882E08093B30380EC97E79093B20357
:10D6C0008093B1038EE095E2909321088093200827
:10D6D00080E995E090932308809322081092240813
:10D6E00010922508109226081092270882E291E0F5
:10D6F000A0E0B0E08093280890932908A0932A081E
:10D70000B0932B08809190059091910585C00330CE
:10D7100009F08FC08091B303882341F16091120812
:10D7200070911308809114089091150825E030E05D
:10D7300040E050E00F940B1A2330310541055105AC
:10D7400051F482E995E00E9493329C01812F6AE0B6
:10D7500075E24EE309C082E995E00E9493329C0194
:10D76000812F6AE075E240E20E94F446FF2009F44E
:10D770009FC06091120870911308809114089091D5
:10D78000150825E030E040E050E00F940B1A2330FC
:10D7900031054105510509F08BC00E947D3880910B
:10D7A000B1039091B20390931D0880931C0880915F
:10D7B00012089091130890931F0880931E0882E02E
:10D7C0008093B30380EC97E79093B2038093B10307
:10D7D00086E095E2909321088093200882E995E005
:10D7E0009093230880932208109224081092250811
:10D7F000109226081092270887E890E0A0E0B0E099
:10D800008093280890932908A0932A08B0932B08A6
:10D810008091920590919305AA2797FDA095BA2F24
:10D820008093120890931308A0931408B0931508DE
:10D8300077C00430E9F58091B3038823F9F0609153
:10D84000120870911308809114089091150825E032
:10D8500030E040E050E00F940B1A243031054105D0
:10D86000510529F4812F69EF74E24EE304C0812F42
:10D8700069EF74E240E220E20E940C35FF20C1F023
:10D880006091120870911308809114089091150806
:10D8900025E030E040E050E00F940B1A24303105D1
:10D8A0004105510529F40E947D380E94D98E38C067
:10D8B0008091120890911308A0911408B091150856
:10D8C0004997A105B10540F0A0921208B092130843
:10D8D000C0921408D0921508609112087091130834
:10D8E000809114089091150825E030E040E050E068
:10D8F0000F940B1A422F80910C0890E0049630E0B0
:10D900008217930744F4445040930C08E092B30309
:10D91000042F01501FEF1F5F153010F40F5FABCDC8
:10D920001F910F91FF90EF90DF90CF90BF90AF903D
:10D930000895AF92BF92CF92DF92EF92FF920F9332
:10D940001F938091120890911308A0911408B09130
:10D95000150881509048A040B04040F01092120845
:10D960001092130810921408109215086091120872
:10D9700070911308809114089091150825E030E00B
:10D9800040E050E00F940B1A79018A0180910C0855
:10D9900090E0A0E0B0E0E816F9060A071B0710F4D3
:10D9A00020930C0800910C0880910B0890E096954C
:10D9B000879596958795FF24F394F82210E0F8E177
:10D9C000AF2EB12CC12CD12CEE24E394002309F00E
:10D9D0003DC08091B3038823C1F0809112089091DB
:10D9E0001308A0911408B09115080597A105B10579
:10D9F00028F4812F63E775E24BEF04C0812F63E7C2
:10DA000075E240E22BEF0E940C35FF2009F4FBC1C8
:10DA10008091120890911308A0911408B0911508F4
:10DA20000597A105B10508F0EEC10E947D3880E997
:10DA300098E79093B2038093B1031092120810926A
:10DA40001308109214081092150815C2013009F03D
:10DA500083C08091B303882341F1609112087091D3
:10DA60001308809114089091150825E030E040E0FB
:10DA700050E00F940B1A213031054105510551F446
:10DA80008EE895E00E9493329C01812F69E675E251
:10DA90004EE309C08EE895E00E9493329C01812FED
:10DAA00069E675E240E20E94F446FF2009F4ABC14A
:10DAB00060911208709113088091140890911508D4
:10DAC00025E030E040E050E00F940B1A21303105A2
:10DAD0004105510509F097C10E947D388091B1033D
:10DAE0009091B20390931D0880931C0880911208B6
:10DAF0009091130890931F0880931E0882E08093F2
:10DB0000B30380EC97E79093B2038093B1038FE562
:10DB100095E290932108809320088EE895E09093F9
:10DB2000230880932208109224081092250810924E
:10DB30002608109227088FEF90E0A0E0B0E08093D5
:10DB4000280890932908A0932A08B0932B08809165
:10DB50008E0590918F050BC1023009F083C0809132
:10DB6000B303882341F160911208709113088091EA
:10DB700014089091150825E030E040E050E00F9443
:10DB80000B1A223031054105510551F48AE895E020
:10DB90000E9493329C01812F68E575E24EE309C033
:10DBA0008AE895E00E9493329C01812F68E575E236
:10DBB00040E20E94F446FF2009F425C1609112085A
:10DBC00070911308809114089091150825E030E0B9
:10DBD00040E050E00F940B1A223031054105510509
:10DBE00009F011C10E947D388091B1039091B20378
:10DBF00090931D0880931C0880911208909113083F
:10DC000090931F0880931E0882E08093B30380ECFA
:10DC100097E79093B2038093B10381E595E29093E7
:10DC20002108809320088AE895E090932308809348
:10DC300022081092240810922508109226081092AB
:10DC4000270882E291E0A0E0B0E08093280890935A
:10DC50002908A0932A08B0932B0880918A059091F7
:10DC60008B0585C0033009F08FC08091B3038823F2
:10DC700041F16091120870911308809114089091FD
:10DC8000150825E030E040E050E00F940B1A2330F7
:10DC900031054105510551F48CE895E00E9493321D
:10DCA0009C01812F6DE475E24EE309C08CE895E09C
:10DCB0000E9493329C01812F6DE475E240E20E9444
:10DCC000F446FF2009F49FC0609112087091130878
:10DCD000809114089091150825E030E040E050E074
:10DCE0000F940B1A233031054105510509F08BC003
:10DCF0000E947D388091B1039091B20390931D08EA
:10DD000080931C08809112089091130890931F082B
:10DD100080931E0882E08093B30380EC97E7909392
:10DD2000B2038093B10389E495E290932108809334
:10DD300020088CE895E090932308809322081092A5
:10DD4000240810922508109226081092270887E8C8
:10DD500090E0A0E0B0E08093280890932908A09379
:10DD60002A08B0932B0880918C0590918D05AA27E5
:10DD700097FDA095BA2F8093120890931308A09353
:10DD80001408B093150877C00430E9F58091B30307
:10DD90008823F9F06091120870911308809114089B
:10DDA0009091150825E030E040E050E00F940B1A08
:10DDB000243031054105510529F4812F6CE375E2CA
:10DDC0004EE304C0812F6CE375E240E220E20E9442
:10DDD0000C35FF20C1F060911208709113088091FA
:10DDE00014089091150825E030E040E050E00F94D1
:10DDF0000B1A243031054105510529F40E947D3864
:10DE00000E94D98E38C08091120890911308A09179
:10DE10001408B09115084997A105B10540F0A092EA
:10DE20001208B0921308C0921408D092150860919D
:10DE3000120870911308809114089091150825E03C
:10DE400030E040E050E00F940B1A422F80910C0814
:10DE500090E0049630E08217930744F444504093D6
:10DE60000C08E092B303042F01501FEF1F5F153021
:10DE700010F40F5FABCD1F910F91FF90EF90DF90EB
:10DE8000CF90BF90AF900895AF92BF92CF92DF92A4
:10DE9000EF92FF920F931F938091120890911308B5
:10DEA000A0911408B091150881509048A040B0404E
:10DEB00040F0109212081092130810921408109259
:10DEC00015086091120870911308809114089091C0
:10DED000150825E030E040E050E00F940B1A79017E
:10DEE0008A0180910C0890E0A0E0B0E0E816F90605
:10DEF0000A071B0710F420930C0800910C0880916E
:10DF00000B0890E09695879596958795FF24F39456
:10DF1000F82210E0B2E2AB2EB12CC12CD12CEE24B1
:10DF2000E394002309F03DC08091B3038823C1F03E
:10DF30008091120890911308A0911408B0911508CF
:10DF40000597A105B10528F4812F64E676E24BEF31
:10DF500004C0812F64E676E240E22BEF0E940C358C
:10DF6000FF2009F412C38091120890911308A09128
:10DF70001408B09115080597A105B10508F005C36F
:10DF80000E947D3883ED91E49093B2038093B103B6
:10DF9000109212081092130810921408109215088B
:10DFA0002CC3013009F087C08091B303882341F16D
:10DFB00060911208709113088091140890911508CF
:10DFC00025E030E040E050E00F940B1A213031059D
:10DFD0004105510551F484EC93E00E9493329C0179
:10DFE000812F6EE576E24EE309C084EC93E00E9457
:10DFF00093329C01812F6EE576E240E20E94F44666
:10E00000FF2009F4C2C26091120870911308809138
:10E0100014089091150825E030E040E050E00F949E
:10E020000B1A213031054105510509F0AEC20E949D
:10E030007D388091B1039091B20390931D08809335
:10E040001C08809112089091130890931F088093E8
:10E050001E0882E08093B30380EC97E79093B203AD
:10E060008093B10388E596E290932108809320087D
:10E0700084EC93E090932308809322088AE090E058
:10E08000A0E0B0E08093240890932508A093260890
:10E09000B093270887EE93E0A0E0B0E080932808D3
:10E0A00090932908A0932A08B0932B088091C40369
:10E0B0009091C5031BC2023009F083C08091B30365
:10E0C000882341F16091120870911308809114081F
:10E0D0009091150825E030E040E050E00F940B1AD5
:10E0E000223031054105510551F48FEE9CE00E942C
:10E0F00093329C01812F61E576E24EE309C08FEEF9
:10E100009CE00E9493329C01812F61E576E240E21F
:10E110000E94F446FF2009F438C260911208709101
:10E120001308809114089091150825E030E040E034
:10E1300050E00F940B1A223031054105510509F0CA
:10E1400024C20E947D388091B1039091B2039093D4
:10E150001D0880931C0880911208909113089093D9
:10E160001F0880931E0882E08093B30380EC97E73A
:10E170009093B2038093B1038AE496E290932108CE
:10E18000809320088FEE9CE09093230880932208D0
:10E190001092240810922508109226081092270841
:10E1A0008CE291E0A0E0B0E08093280890932908E9
:10E1B000A0932A08B0932B088091EF0C9091F00C5B
:10E1C00095C1033009F083C08091B303882341F1E6
:10E1D00060911208709113088091140890911508AD
:10E1E00025E030E040E050E00F940B1A2330310579
:10E1F0004105510551F481EF9CE00E9493329C014E
:10E20000812F66E476E24EE309C081EF9CE00E9434
:10E2100093329C01812F66E476E240E20E94F4464C
:10E22000FF2009F4B2C16091120870911308809127
:10E2300014089091150825E030E040E050E00F947C
:10E240000B1A233031054105510509F09EC10E948A
:10E250007D388091B1039091B20390931D08809313
:10E260001C08809112089091130890931F088093C6
:10E270001E0882E08093B30380EC97E79093B2038B
:10E280008093B10382E496E2909321088093200862
:10E2900081EF9CE090932308809322081092240839
:10E2A00010922508109226081092270887E890E01F
:10E2B000A0E0B0E08093280890932908A0932A0852
:10E2C000B0932B088091F10C9091F20C0FC10430A7
:10E2D00009F083C08091B303882341F16091120853
:10E2E00070911308809114089091150825E030E092
:10E2F00040E050E00F940B1A2430310541055105E0
:10E3000051F48CE09BE00E9493329C01812F68E3E2
:10E3100076E24EE309C08CE09BE00E9493329C01C0
:10E32000812F68E376E240E20E94F446FF2009F480
:10E330002CC160911208709113088091140890917B
:10E34000150825E030E040E050E00F940B1A24302F
:10E3500031054105510509F018C10E947D388091B1
:10E36000B1039091B20390931D0880931C08809193
:10E3700012089091130890931F0880931E0882E062
:10E380008093B30380EC97E79093B2038093B1033B
:10E390008EE296E290932108809320088CE09BE027
:10E3A0009093230880932208109224081092250845
:10E3B00010922608109227088FEF90E0A0E0B0E0BE
:10E3C0008093280890932908A0932A08B0932B08DB
:10E3D00080910C0B90910D0B89C0053009F093C012
:10E3E0008091B303882341F1609112087091130862
:10E3F000809114089091150825E030E040E050E04D
:10E400000F940B1A253031054105510551F486EC66
:10E4100093E00E9493329C01812F69E276E24EE301
:10E4200009C086EC93E00E9493329C01812F69E23F
:10E4300076E240E20E94F446FF2009F4A6C0609113
:10E44000120870911308809114089091150825E026
:10E4500030E040E050E00F940B1A253031054105C3
:10E46000510509F092C00E947D388091B1039091CE
:10E47000B20390931D0880931C088091120890911C
:10E48000130890931F0880931E0882E08093B303C3
:10E4900080EC97E79093B2038093B10384E296E215
:10E4A000909321088093200886EC93E090932308B2
:10E4B000809322088AE090E0A0E0B0E080932408F6
:10E4C00090932508A0932608B093270887EE93E041
:10E4D000A0E0B0E08093280890932908A0932A0830
:10E4E000B0932B088091C6039091C703AA2797FD8C
:10E4F000A095BA2F8093120890931308A093140844
:10E50000B09315087AC0063009F03FC08091B3037C
:10E510008823F9F060911208709113088091140813
:10E520009091150825E030E040E050E00F940B1A80
:10E53000263031054105510529F4812F64E176E249
:10E540004EE304C0812F64E176E240E220E20E94C3
:10E550000C35FF20D1F06091120870911308809162
:10E5600014089091150825E030E040E050E00F9449
:10E570000B1A263031054105510539F40E947D38CA
:10E580008FE096E20E944EC338C0809112089091AD
:10E590001308A0911408B09115088397A105B1053F
:10E5A00040F0A0921208B0921308C0921408D092C2
:10E5B00015086091120870911308809114089091C9
:10E5C000150825E030E040E050E00F940B1A422F90
:10E5D00080910C0890E0049630E08217930744F491
:10E5E000445040930C08E092B303042F01501FEFF6
:10E5F0001F5F153010F40F5F94CC1F910F91FF90A7
:10E60000EF90DF90CF90BF90AF900895CF92DF92C0
:10E61000EF92FF920F931F937C01D62EC72E04ED2D
:10E6200017E08091D4078B51109208088093090855
:10E63000C801019760EA72E10F94540AC7010E9471
:10E64000FC3405501040C8016AE30F947011ED2DA1
:10E65000FC2DDF010D900020E9F72091D4072B510C
:10E66000EA1BFB0B7396CF0133E0880F991F3A9595
:10E67000E1F78E1B9F0B8093080820930908C801BF
:10E680006D2D7C2D0F9494111F910F91FF90EF90A1
:10E69000DF90CF9008950F931F93DF93CF9300D017
:10E6A0000F92CDB7DEB72091240830912508409114
:10E6B0002608509127088091120890911308A09184
:10E6C0001408B091150882179307A407B50744F4FE
:10E6D00020931208309313084093140850931508A0
:10E6E000209128083091290840912A0850912B0840
:10E6F0008091120890911308A0911408B091150808
:10E70000281739074A075B0744F42093120830930F
:10E71000130840931408509315088091B30388237D
:10E72000F9F0009120081091210860911208709171
:10E73000130880911408909115080F94B3162AE0DD
:10E7400037ED43E25CE30F941A1669837A838B8377
:10E750009C83CE0101960E94DF32BC01C80156DFC6
:10E7600080910B0882FF38C0009122081091230885
:10E770006091120870911308809114089091150807
:10E780000F94B3162AE037ED43E25CE30F941A16B8
:10E790000F948716F80160837183828393830E94AC
:10E7A0007D3880911C0890911D089093B20380934E
:10E7B000B10380911E0890911F08A0E0B0E0809303
:10E7C000120890931308A0931408B0931508E091D1
:10E7D0002C08F0912D0819950F900F900F900F9025
:10E7E000CF91DF911F910F9108950F931F93DF93A6
:10E7F000CF9300D00F92CDB7DEB72091240830918F
:10E800002508409126085091270880911208909180
:10E810001308A0911408B091150882179307A40754
:10E82000B50744F42093120830931308409314085A
:10E8300050931508209128083091290840912A0802
:10E8400050912B088091120890911308A091140800
:10E85000B0911508281739074A075B0744F420933D
:10E8600012083093130840931408509315088091B0
:10E87000B3038823F9F000912008109121086091DA
:10E8800012087091130880911408909115080F9444
:10E89000B31620E030E048EC52E40F941A16698376
:10E8A0007A838B839C83CE0101960E940E34BC0137
:10E8B000C801ACDE80910B0882FF36C000912208AF
:10E8C0001091230860911208709113088091140828
:10E8D000909115080F94B31620E030E048EC52E414
:10E8E0000F941A16F80160837183828393830E94C8
:10E8F0007D3880911C0890911D089093B2038093FD
:10E90000B10380911E0890911F08A0E0B0E08093B1
:10E91000120890931308A0931408B0931508E0917F
:10E920002C08F0912D0819950F900F900F900F90D3
:10E93000CF91DF911F910F9108950F931F93DF9354
:10E94000CF9300D00F92CDB7DEB72091240830913D
:10E95000250840912608509127088091120890912F
:10E960001308A0911408B091150882179307A40703
:10E97000B50744F420931208309313084093140809
:10E9800050931508209128083091290840912A08B1
:10E9900050912B088091120890911308A0911408AF
:10E9A000B0911508281739074A075B0744F42093EC
:10E9B000120830931308409314085093150880915F
:10E9C000B3038823F9F00091200810912108609189
:10E9D00012087091130880911408909115080F94F3
:10E9E000B31620E030E048EC52E40F941A16698325
:10E9F0007A838B839C83CE0101960E940E34BC01E6
:10EA0000C80104DE80910B0882FF31C0009122080A
:10EA100010912308609112087091130880911408D6
:10EA2000909115080F94B31620E030E048EC52E4C2
:10EA30000F941A16F80160837183828393830E9476
:10EA40007D3880911C0890911D089093B2038093AB
:10EA5000B10380911E0890911F08A0E0B0E0809360
:10EA6000120890931308A0931408B09315080F9000
:10EA70000F900F900F90CF91DF911F910F910895FC
:10EA80000F931F93DF93CF9300D00F92CDB7DEB7D4
:10EA9000209124083091250840912608509127089C
:10EAA0008091120890911308A0911408B091150854
:10EAB00082179307A407B50744F4209312083093F4
:10EAC000130840931408509315082091280830919A
:10EAD000290840912A0850912B08809112089091A2
:10EAE0001308A0911408B0911508281739074A0790
:10EAF0005B0744F4209312083093130840931408E2
:10EB0000509315088091B3038823F9F000912008F1
:10EB100010912108609112087091130880911408D7
:10EB2000909115080F94B31620E030E040E251E4D4
:10EB30000F941A1669837A838B839C83CE01019686
:10EB40000E948733BC01C80161DD80910B0882FF00
:10EB500031C0009122081091230860911208709131
:10EB6000130880911408909115080F94B31620E0B3
:10EB700030E040E251E40F941A16F801608371838B
:10EB8000828393830E947D3880911C0890911D0898
:10EB90009093B2038093B10380911E0890911F0857
:10EBA000A0E0B0E08093120890931308A09314089B
:10EBB000B09315080F900F900F900F90CF91DF91A9
:10EBC0001F910F9108950F931F93DF93CF9300D060
:10EBD0000F92CDB7DEB720912408309125084091DF
:10EBE0002608509127088091120890911308A0914F
:10EBF0001408B091150882179307A407B50744F4C9
:10EC0000209312083093130840931408509315086A
:10EC1000209128083091290840912A0850912B080A
:10EC20008091120890911308A0911408B0911508D2
:10EC3000281739074A075B0744F4209312083093DA
:10EC4000130840931408509315088091B303882348
:10EC5000F9F000912008109121086091120870913C
:10EC6000130880911408909115080F94B3162AE0A8
:10EC700037ED43E25CE30F941A1669837A838B8342
:10EC80009C83CE0101960E94DF32BC01C801BEDC2C
:10EC900080910B0882FF31C0009122081091230857
:10ECA00060911208709113088091140890911508D2
:10ECB0000F94B3162AE037ED43E25CE30F941A1683
:10ECC000F80160837183828393830E947D388091F1
:10ECD0001C0890911D089093B2038093B10380911A
:10ECE0001E0890911F08A0E0B0E080931208909356
:10ECF0001308A0931408B09315080F900F900F906D
:10ED00000F90CF91DF911F910F9108950F931F9353
:10ED1000DF93CF9300D00F92CDB7DEB720912408B8
:10ED200030912508409126085091270880911208BB
:10ED300090911308A0911408B091150882179307B9
:10ED4000A407B50744F420931208309313084093A6
:10ED500014085093150820912808309129084091F3
:10ED60002A0850912B088091120890911308A091C5
:10ED70001408B0911508281739074A075B0744F4AF
:10ED800020931208309313084093140850931508E9
:10ED90008091B3038823F9F0009120081091210895
:10EDA00060911208709113088091140890911508D1
:10EDB0000F94B31620E030E048EC52E40F941A169A
:10EDC00069837A838B839C83CE0101960E940F32E4
:10EDD000BC01C8011BDC80910B0882FF31C000918F
:10EDE00022081091230860911208709113088091F5
:10EDF0001408909115080F94B31620E030E048EC09
:10EE000052E40F941A16F80160837183828393830E
:10EE10000E947D3880911C0890911D089093B20348
:10EE20008093B10380911E0890911F08A0E0B0E08C
:10EE30008093120890931308A0931408B0931508B8
:10EE40000F900F900F900F90CF91DF911F910F9126
:10EE500008950F931F93DF93CF9300D00F92CDB7F8
:10EE6000DEB7209124083091250840912608509162
:10EE700027088091120890911308A0911408B0916E
:10EE8000150882179307A407B50744F420931208C6
:10EE900030931308409314085093150820912808C4
:10EEA0003091290840912A0850912B08809112082E
:10EEB00090911308A0911408B091150828173907EC
:10EEC0004A075B0744F420931208309313084093D9
:10EED0001408509315088091B3038823C9F000915A
:10EEE00020081091210860911208709113088091F8
:10EEF0001408909115080F94B31669837A838B8355
:10EF00009C83CE0101960E94C832BC01C8017EDB01
:10EF100080910B0882FF2BC00091220810912308DA
:10EF2000609112087091130880911408909115084F
:10EF30000F94B316F80160837183828393830E94D8
:10EF40007D3880911C0890911D089093B2038093A6
:10EF5000B10380911E0890911F08A0E0B0E080935B
:10EF6000120890931308A0931408B09315080F90FB
:10EF70000F900F900F90CF91DF911F910F910895F7
:10EF80000F931F93DF93CF930F920F92CDB7DEB7FE
:10EF90002091240830912508409126085091270897
:10EFA0008091120890911308A0911408B09115084F
:10EFB00082179307A407B50744F4209312083093EF
:10EFC0001308409314085093150820912808309195
:10EFD000290840912A0850912B088091120890919D
:10EFE0001308A0911408B0911508281739074A078B
:10EFF0005B0744F4209312083093130840931408DD
:10F00000509315088091B303882389F0009120085C
:10F010001091210880911208909113089A83898396
:10F02000CE0101960E949332BC01C801EFDA8091B3
:10F030000B0882FF22C0E0912208F0912308809102
:10F04000120890911308918380830E947D388091EB
:10F050001C0890911D089093B2038093B103809196
:10F060001E0890911F08A0E0B0E0809312089093D2
:10F070001308A0931408B09315080F900F90CF9128
:10F08000DF911F910F910895CF92DF92EF92FF923F
:10F090000F931F93CF93DF93082FEB01F42E690199
:10F0A000C9010E94D52161E1E62EE81A10920808F4
:10F0B00010E00F5F1F4FC801880F991F800F911F2D
:10F0C000880F991F880F991F809309088FEC97E08C
:10F0D0006F2D0F94701106C08FEC97E00F94701194
:10F0E0002196EA94FE0164916623B1F78FEC97E0D4
:10F0F0006AE30F94701106C08FEC97E060E20F9402
:10F100007011EA94EE20C1F7C6010E94FC34DF9131
:10F11000CF911F910F91FF90EF90DF90CF900895C6
:10F12000EF92FF920F931F936091E7037091E803B2
:10F130008091E9039091EA030E94C5D460932E0860
:10F1400070932F0880933008909331086091EB03FF
:10F150007091EC038091ED039091EE030E94D1D465
:10F160006093320870933308809334089093350885
:10F170008091120890911308A0911408B09115087D
:10F1800081509048A040B04040F010921208109278
:10F1900013081092140810921508609112087091CB
:10F1A0001308809114089091150825E030E040E0A4
:10F1B00050E00F940B1A79018A0180910C0890E0BD
:10F1C000A0E0B0E0E816F9060A071B0710F4209348
:10F1D0000C0800910C0880910B0890E0969587959B
:10F1E00096958795FF24F394F82210E00023A1F56B
:10F1F0008091B3038823C1F0809112089091130885
:10F20000A0911408B09115080597A105B10528F43F
:10F21000812F65ED72E24BEF04C0812F65ED72E244
:10F2200040E22BEF0E940C35FF2011F40C94CC81AE
:10F230008091120890911308A0911408B0911508BC
:10F240000597A105B10510F00C94CC810E947D3882
:10F250008AEA9AE80C94BF81013009F085C0809158
:10F26000B303882341F160911208709113088091D3
:10F2700014089091150825E030E040E050E00F942C
:10F280000B1A213031054105510551F48FEE9CE0F8
:10F290000E9493329C01812F6EEC72E24EE309C012
:10F2A0008FEE9CE00E9493329C01812F6EEC72E203
:10F2B00040E20E94F446FF2011F40C94CC8160914E
:10F2C000120870911308809114089091150825E098
:10F2D00030E040E050E00F940B1A21303105410539
:10F2E000510511F00C94CC810E947D388091B103BE
:10F2F0009091B20390931D0880931C08809112088E
:10F300009091130890931F0880931E0882E08093C9
:10F31000B30380EC97E79093B2038093B10387EC3B
:10F3200092E290932108809320088FEE9CE09093C6
:10F330002308809322081092240810922508109226
:10F3400026081092270882E291E0A0E0B0E08093C6
:10F35000280890932908A0932A08B0932B0880913D
:10F36000EF0C9091F00C85C0023009F08FC08091B5
:10F37000B303882341F160911208709113088091C2
:10F3800014089091150825E030E040E050E00F941B
:10F390000B1A223031054105510551F481EF9CE0F3
:10F3A0000E9493329C01812F63EC72E24EE309C00C
:10F3B00081EF9CE00E9493329C01812F63EC72E20A
:10F3C00040E20E94F446FF2009F4E6C7609112086B
:10F3D00070911308809114089091150825E030E091
:10F3E00040E050E00F940B1A2230310541055105E1
:10F3F00009F0D2C70E947D388091B1039091B20389
:10F4000090931D0880931C08809112089091130816
:10F4100090931F0880931E0882E08093B30380ECD2
:10F4200097E79093B2038093B1038FEB92E29093AE
:10F4300021088093200881EF9CE09093230880931B
:10F440002208109224081092250810922608109283
:10F45000270887E890E0A0E0B0E080932808909328
:10F460002908A0932A08B0932B088091F10C909161
:10F47000F20CAA2797FDA095BA2F809312089093BB
:10F480001308A0931408B0931508C5C7033009F0FA
:10F4900083C08091B303882341F160911208709179
:10F4A0001308809114089091150825E030E040E0A1
:10F4B00050E00F940B1A233031054105510551F4EA
:10F4C0008CE09BE00E9493329C01812F65EB72E2FD
:10F4D0004EE309C08CE09BE00E9493329C01812F97
:10F4E00065EB72E240E20E94F446FF2009F454C743
:10F4F000609112087091130880911408909115087A
:10F5000025E030E040E050E00F940B1A2330310545
:10F510004105510509F040C70E947D388091B10333
:10F520009091B20390931D0880931C08809112085B
:10F530009091130890931F0880931E0882E0809397
:10F54000B30380EC97E79093B2038093B1038BEA07
:10F5500092E290932108809320088CE09BE09093A6
:10F5600023088093220810922408109225081092F4
:10F570002608109227088FEF90E0A0E0B0E080937B
:10F58000280890932908A0932A08B0932B0880910B
:10F590000C0B90910D0B6DCF043009F051C0809190
:10F5A000B303882369F16091120870911308809168
:10F5B00014089091150825E030E040E050E00F94E9
:10F5C0000B1A8091DB0F243031054105510561F4A0
:10F5D000882319F42AE932E202C02EE932E2812FAF
:10F5E00062EA72E24EE30BC0882319F422E932E2A8
:10F5F00002C026E932E2812F62EA72E240E244DD93
:10F60000FF2009F4C9C66091120870911308809117
:10F6100014089091150825E030E040E050E00F9488
:10F620000B1A243031054105510509F0B5C60E9479
:10F630007D388091DB0F91E089278093DB0FEBC64B
:10F64000053009F087C08091B303882341F16091B0
:10F65000120870911308809114089091150825E004
:10F6600030E040E050E00F940B1A253031054105A1
:10F67000510551F489E094E00E94C8329C01812F29
:10F680006BE872E24EE309C089E094E00E94C83260
:10F690009C01812F6BE872E240E20E94F446FF2059
:10F6A00009F47AC6609112087091130880911408C9
:10F6B0009091150825E030E040E050E00F940B1ADF
:10F6C000253031054105510509F066C60E947D3897
:10F6D0008091B1039091B20390931D0880931C0810
:10F6E000809112089091130890931F0880931E0830
:10F6F00082E08093B30389E297E79093B20380930B
:10F70000B10384E892E2909321088093200889E075
:10F7100094E090932308809322081092240810927A
:10F720002508109226081092270882E291E0A0E0B6
:10F73000B0E08093280890932908A0932A08B093FA
:10F740002B086091090470910A0480910B04909138
:10F750000C0479C3063009F087C08091B303882375
:10F7600041F16091120870911308809114089091F2
:10F77000150825E030E040E050E00F940B1A2630E9
:10F7800031054105510551F485E094E00E94C832ED
:10F790009C01812F6DE772E24EE309C085E094E0A1
:10F7A0000E94C8329C01812F6DE772E240E20E9404
:10F7B000F446FF2009F4F0C5609112087091130817
:10F7C000809114089091150825E030E040E050E069
:10F7D0000F940B1A263031054105510509F0DCC59F
:10F7E0000E947D388091B1039091B20390931D08DF
:10F7F00080931C08809112089091130890931F0821
:10F8000080931E0882E08093B30389E297E7909388
:10F81000B2038093B10386E792E29093210880932C
:10F82000200885E094E090932308809322081092AA
:10F83000240810922508109226081092270882E2C8
:10F8400091E0A0E0B0E08093280890932908A0936D
:10F850002A08B0932B0860910504709106048091EA
:10F86000070490910804EFC2073009F087C0809127
:10F87000B303882341F160911208709113088091BD
:10F8800014089091150825E030E040E050E00F9416
:10F890000B1A273031054105510551F48DE094E0F4
:10F8A0000E940F329C01812F6EE672E24EE309C086
:10F8B0008DE094E00E940F329C01812F6EE672E28F
:10F8C00040E20E94F446FF2009F466C560911208E8
:10F8D00070911308809114089091150825E030E08C
:10F8E00040E050E00F940B1A2730310541055105D7
:10F8F00009F052C50E947D388091B1039091B20306
:10F9000090931D0880931C08809112089091130811
:10F9100090931F0880931E0882E08093B30386E8CB
:10F9200096E79093B2038093B10386E692E29093B8
:10F930002108809320088DE094E090932308809321
:10F94000220810922408109225081092260810927E
:10F95000270884E690E0A0E0B0E080932808909328
:10F960002908A0932A08B0932B0860910D04709188
:10F970000E0480910F04909110048DC0083009F09E
:10F9800091C08091B303882341F160911208709176
:10F990001308809114089091150825E030E040E0AC
:10F9A00050E00F940B1A283031054105510551F4F0
:10F9B00083EE93E00E940E349C01812F60E672E298
:10F9C0004EE309C083EE93E00E940E349C01812F28
:10F9D00060E672E240E20E94F446FF2009F4DCC4D3
:10F9E0006091120870911308809114089091150885
:10F9F00025E030E040E050E00F940B1A283031054C
:10FA00004105510509F0C8C40E947D388091B103B9
:10FA10009091B20390931D0880931C088091120866
:10FA20009091130890931F0880931E0882E08093A2
:10FA3000B3038DE994E79093B2038093B1038AE511
:10FA400092E2909321088093200883EE93E09093B4
:10FA500023088093220884E690E0A0E0B0E0809341
:10FA6000240890932508A0932608B093270888E5DA
:10FA70009EE3AFE0B0E08093280890932908A0931C
:10FA80002A08B0932B086091E3037091E4038091FE
:10FA9000E5039091E60320E030E048EC52E40F9457
:10FAA000F318D1C1093009F09DC08091B3038823B8
:10FAB00041F160911208709113088091140890919F
:10FAC000150825E030E040E050E00F940B1A293093
:10FAD00031054105510551F48EE298E00E940E3443
:10FAE0009C01812F64E572E24EE309C08EE298E04A
:10FAF0000E940E349C01812F64E572E240E20E9474
:10FB0000F446FF2009F448C460911208709113086C
:10FB1000809114089091150825E030E040E050E015
:10FB20000F940B1A293031054105510509F034C4F1
:10FB30000E947D388091B1039091B20390931D088B
:10FB400080931C08809112089091130890931F08CD
:10FB500080931E0882E08093B30385EF93E7909330
:10FB6000B2038093B1038EE492E2909321088093D4
:10FB700020088EE298E0909323088093220881E089
:10FB800090E0A0E0B0E08093240890932508A09333
:10FB90002608B093270888E59EE3AFE0B0E08093A5
:10FBA000280890932908A0932A08B0932B08609105
:10FBB0002E0870912F08809130089091310820E034
:10FBC00030E048EC52E40F94F3180F9487166093DA
:10FBD000120870931308809314089093150884EF0B
:10FBE00094E89FC00A3009F0A1C08091B303882334
:10FBF00041F160911208709113088091140890915E
:10FC0000150825E030E040E050E00F940B1A2A3050
:10FC100031054105510551F482E398E00E940E340C
:10FC20009C01812F68E472E24EE309C082E398E010
:10FC30000E940E349C01812F68E472E240E20E942F
:10FC4000F446FF2009F4A8C36091120870911308CC
:10FC5000809114089091150825E030E040E050E0D4
:10FC60000F940B1A2A3031054105510509F094C350
:10FC70000E947D388091B1039091B20390931D084A
:10FC800080931C08809112089091130890931F088C
:10FC900080931E0882E08093B30385EF93E79093EF
:10FCA000B2038093B10382E492E29093210880939F
:10FCB000200882E398E0909323088093220884E64A
:10FCC00090E0A0E0B0E08093240890932508A093F2
:10FCD0002608B093270888E59EE3AFE0B0E0809364
:10FCE000280890932908A0932A08B0932B086091C4
:10FCF000320870913308809134089091350820E0E3
:10FD000030E048EC52E40F94F3180F948716609398
:10FD1000120870931308809314089093150880EECE
:10FD200094E890932D0880932C0875C30B3009F04C
:10FD300095C08091B303882341F1609112087091BE
:10FD40001308809114089091150825E030E040E0F8
:10FD500050E00F940B1A2B3031054105510551F439
:10FD60008FEE93E00E94C8329C01812F6CE372E217
:10FD70004EE309C08FEE93E00E94C8329C01812FB0
:10FD80006CE372E240E20E94F446FF2009F404C3EF
:10FD900060911208709113088091140890911508D1
:10FDA00025E030E040E050E00F940B1A2B30310595
:10FDB0004105510509F0F0C20E947D388091B103E0
:10FDC0009091B20390931D0880931C0880911208B3
:10FDD0009091130890931F0880931E0882E08093EF
:10FDE000B30389E297E79093B2038093B10386E36C
:10FDF00092E290932108809320088FEE93E09093F5
:10FE000023088093220881E090E0A0E0B0E0809396
:10FE1000240890932508A0932608B093270886E02D
:10FE200097E2A0E0B0E08093280890932908A0937F
:10FE30002A08B0932B086091EF037091F003809132
:10FE4000F1039091F2030F94871660931208709358
:10FE500013088093140890931508DDC20C3009F044
:10FE60003FC08091B3038823F9F06091120870912C
:10FE70001308809114089091150825E030E040E0C7
:10FE800050E00F940B1A2C3031054105510529F42F
:10FE9000812F6DE272E24EE304C0812F6DE272E2C7
:10FEA00040E22AEF0E940C35FF2009F475C26091F0
:10FEB000120870911308809114089091150825E09C
:10FEC00030E040E050E00F940B1A2C303105410532
:10FED000510509F061C20E947D3889E99CE64FC254
:10FEE0000D3009F03FC08091B3038823F9F0609191
:10FEF000120870911308809114089091150825E05C
:10FF000030E040E050E00F940B1A2D3031054105F0
:10FF1000510529F4812F63E272E24EE304C0812F80
:10FF200063E272E240E22AEF0E940C35FF2009F4FE
:10FF300033C2609112087091130880911408909157
:10FF4000150825E030E040E050E00F940B1A2D300A
:10FF500031054105510509F01FC20E947D388EEE22
:10FF600099E60DC20E3009F03FC08091B30388239B
:10FF7000F9F0609112087091130880911408909123
:10FF8000150825E030E040E050E00F940B1A2E30C9
:10FF900031054105510529F4812F6AE172E24EE3F2
:10FFA00004C0812F6AE172E240E22AEF0E940C3520
:10FFB000FF2009F4F1C1609112087091130880913B
:10FFC00014089091150825E030E040E050E00F94CF
:10FFD0000B1A2E3031054105510509F0DDC10E9493
:10FFE0007D3883E497E6CBC10F3009F03FC08091A4
:10FFF000B3038823F9F0609112087091130880917F
:020000021000EC
:1000000014089091150825E030E040E050E00F948E
:100010000B1A2F3031054105510529F4812F6EE06F
:1000200072E24EE304C0812F6EE072E240E22AEFFA
:100030000E940C35FF2009F4AFC160911208709145
:100040001308809114089091150825E030E040E0F5
:1000500050E00F940B1A2F3031054105510509F07E
:100060009BC10E947D3888E994E689C1003109F07E
:100070003FC08091B3038823F9F06091120870911A
:100080001308809114089091150825E030E040E0B5
:1000900050E00F940B1A203131054105510529F428
:1000A000812F63E072E24EE304C0812F63E072E2CD
:1000B00040E22AEF0E940C35FF2009F46DC16091E7
:1000C000120870911308809114089091150825E08A
:1000D00030E040E050E00F940B1A2031310541052B
:1000E000510509F059C10E947D388DEE91E647C156
:1000F000013109F03FC08091B3038823F9F060918A
:10010000120870911308809114089091150825E049
:1001100030E040E050E00F940B1A213131054105E9
:10012000510529F4812F64EF71E24EE304C0812F61
:1001300064EF71E240E22AEF0E940C35FF2009F4DF
:100140002BC160911208709113088091140890914E
:10015000150825E030E040E050E00F940B1A213103
:1001600031054105510509F017C10E947D3882E42F
:100170009FE505C1023109F03FC08091B303882398
:10018000F9F0609112087091130880911408909111
:10019000150825E030E040E050E00F940B1A2231C2
:1001A00031054105510529F4812F68EE71E24EE3D6
:1001B00004C0812F68EE71E240E22AEF0E940C3504
:1001C000FF2009F4E9C06091120870911308809132
:1001D00014089091150825E030E040E050E00F94BD
:1001E0000B1A223131054105510509F0D5C00E9495
:1001F0007D3887E99CE5C3C0033109F03FC0809199
:10020000B3038823F9F0609112087091130880916C
:1002100014089091150825E030E040E050E00F947C
:100220000B1A233131054105510529F4812F6AED5F
:1002300071E24EE304C0812F6AED71E240E22AEFE1
:100240000E940C35FF2009F4A7C06091120870913C
:100250001308809114089091150825E030E040E0E3
:1002600050E00F940B1A233131054105510509F077
:1002700093C00E947D388CEE99E581C0043109F06D
:100280003FC08091B3038823F9F060911208709108
:100290001308809114089091150825E030E040E0A3
:1002A00050E00F940B1A243131054105510529F412
:1002B000812F6CEC71E24EE304C0812F6CEC71E293
:1002C00040E22AEF0E940C35FF2009F465C06091DE
:1002D000120870911308809114089091150825E078
:1002E00030E040E050E00F940B1A24313105410515
:1002F000510509F051C00E947D3881E497E53FC067
:10030000053109F049C08091B3038823F9F0609169
:10031000120870911308809114089091150825E037
:1003200030E040E050E00F940B1A253131054105D3
:10033000510529F4812F60EC71E24EE304C0812F56
:1003400060EC71E240E22AEF0E940C35FF2021F1BF
:10035000609112087091130880911408909115080B
:1003600025E030E040E050E00F940B1A25313105D4
:100370004105510589F40E947D3886E994E5909302
:10038000B2038093B10310921208109213081092D6
:100390001408109215083FC080911208909113081C
:1003A000A0911408B09115088E369105A105B105EC
:1003B00060F08DE690E0A0E0B0E0809312089093AA
:1003C0001308A0931408B093150860911208709157
:1003D0001308809114089091150825E030E040E062
:1003E00050E00F940B1A422F80910C0890E0049675
:1003F00030E0821793074CF4445040930C0881E09E
:100400008093B303042F01501FEF1F5F153018F4C2
:100410000F5F0C94F6781F910F91FF90EF90089565
:10042000CF92DF92EF92FF920F931F9320911208C9
:100430003091130840911408509115082115310589
:100440004105510509F448C0B901882777FD809519
:10045000982F0F94B51620913608309137084091A7
:100460003808509139080F94F3189B01AC01609142
:10047000E70A7091E80A8091E90A9091EA0A0F94DC
:100480003A156093E70A7093E80A8093E90A90931B
:10049000EA0A10921208109213081092140810928F
:1004A00015088BED9AE06FED7AE043EE5AE027EE07
:1004B0003AE00F2EF0E0EF2EF0E0FF2EF0E80F2FE5
:1004C000FFE31F2FF02DEAE0CE2EEBE0DE2E0E94A0
:1004D00057F981E08093B3038091B303882349F0F7
:1004E00087EE9AE00E947431BC0180E096E20E949F
:1004F000067380910B0882FF10C00E947D388FEB3D
:100500009AE39093B2038093B10310921208109271
:10051000130810921408109215081F910F91FF9064
:10052000EF90DF90CF900895CF92DF92EF92FF92FD
:100530000F931F93209112083091130840911408D3
:1005400050911508211531054105510509F476C072
:10055000B901882777FD8095982F0F94B5162091C3
:1005600036083091370840913808509139080F9477
:10057000F3182091E30A3091E40A4091E50A509182
:10058000E60A0F943A156093E30A7093E40A8093A5
:10059000E50A9093E60A20E030E040E050E00F9456
:1005A0001316882364F480E090E0A0E0B0E080932C
:1005B000E30A9093E40AA093E50AB093E60A6091F7
:1005C000E30A7091E40A8091E50A9091E60A20E03E
:1005D00030E04AE753E40F942118181664F480E0E1
:1005E00090E0AAE7B3E48093E30A9093E40AA0932F
:1005F000E50AB093E60A10921208109213081092BE
:100600001408109215088BED9AE06FED7AE043EE36
:100610005AE027EE3AE00F2EF0E0EF2EF0E0FF2E4A
:10062000F0E80F2FF0E41F2FF02DFAE0CF2EFBE0C3
:10063000DF2E0E9457F981E08093B3038091B303CA
:10064000882349F083EE9AE00E947431BC0189E06E
:1006500096E20E94067380910B0882FF10C00E94F0
:100660007D388FEB9AE39093B2038093B10310929D
:1006700012081092130810921408109215081F9176
:100680000F91FF90EF90DF90CF900895CF92DF927F
:10069000EF92FF920F931F9320911208309113084D
:1006A0004091140850911508211531054105510557
:1006B00009F476C0B901882777FD8095982F0F94AB
:1006C000B51620913608309137084091380850917E
:1006D00039080F94F3182091DF0A3091E00A409115
:1006E000E10A5091E20A0F943A156093DF0A709381
:1006F000E00A8093E10A9093E20A20E030E040E0D3
:1007000050E00F941316882364F480E090E0A0E09A
:10071000B0E08093DF0A9093E00AA093E10AB093DF
:10072000E20A6091DF0A7091E00A8091E10A9091FB
:10073000E20A20E030E849E853E40F942118181643
:1007400064F480E090E8A9E8B3E48093DF0A909332
:10075000E00AA093E10AB093E20A10921208109204
:10076000130810921408109215088BED9AE06FEDA3
:100770007AE043EE5AE027EE3AE00F2EF0E0EF2E5B
:10078000F0E0FF2EF8E40F2FF2E41F2FF02DAAE087
:10079000CA2EABE0DA2E0E9457F981E08093B303B2
:1007A0008091B303882349F08FED9AE00E94743161
:1007B000BC018BE096E20E94067380910B0882FFD9
:1007C00010C00E947D388FEB9AE39093B203809320
:1007D000B10310921208109213081092140810928C
:1007E00015081F910F91FF90EF90DF90CF90089523
:1007F000CF92DF92EF92FF920F931F9320911208F6
:1008000030911308409114085091150821153105B5
:100810004105510509F476C0B901882777FD809517
:10082000982F0F94B51620913608309137084091D3
:100830003808509139080F94F3182091DB0A309151
:10084000DC0A4091DD0A5091DE0A0F943A1560935C
:10085000DB0A7093DC0A8093DD0A9093DE0A20E0C5
:1008600030E040E050E00F941316882364F480E0F9
:1008700090E0A0E0B0E08093DB0A9093DC0AA093C4
:10088000DD0AB093DE0A6091DB0A7091DC0A809188
:10089000DD0A9091DE0A20E030E045E953E40F9450
:1008A0002118181664F480E090E0A5E9B3E4809381
:1008B000DB0A9093DC0AA093DD0AB093DE0A109263
:1008C00012081092130810921408109215088BED5C
:1008D0009AE06FED7AE043EE5AE027EE3AE00F2E11
:1008E000F0E0EF2EF0E0FF2EF8E40F2FF2E41F2FE0
:1008F000F02DBAE0CB2EBBE0DB2E0E9457F981E051
:100900008093B3038091B303882349F08BED9AE081
:100910000E947431BC018DE096E20E9406738091C2
:100920000B0882FF10C00E947D388FEB9AE39093F2
:10093000B2038093B1031092120810921308109220
:100940001408109215081F910F91FF90EF90DF90FF
:10095000CF900895FF920F931F938C01262FFC01D7
:10096000F1AC04966F2D42AD0F94F40AF80EF80125
:10097000F1AE81E090E01F910F91FF9008950F93E9
:100980001F9381ED97E01092D2071092D10721E3D7
:1009900034E0FC01329322938F01109208081092E8
:1009A000090810920A0802966BEA73E00F94CB0DC7
:1009B00089E294E0F801918380831F910F9108955B
:1009C0006091320870913308809134089091350815
:1009D0000E94CBD46093EB037093EC038093ED0300
:1009E0009093EE030C94B2D360912E0870912F086F
:1009F00080913008909131080E94BFD46093E70342
:100A00007093E8038093E9039093EA030C94B2D3C4
:100A10001F93CF93DF93EC01162F8BAD882331F416
:100A200081E08BAFCE0104960F94620DCE01049647
:100A3000612F0F94830DDF91CF911F910895682F3F
:100A400070E06F7370707093CE076093CD078FEC7A
:100A500097E0DECFBC018091CC05882349F48EE875
:100A600093E044E150E00E94F62182E08093B303DA
:100A70000895F0DF81E08093CC0510921208109267
:100A80001308109214081092150881EA98E39093C5
:100A9000B2038093B1030895BC018091CC058823F3
:100AA00049F48EE893E044E150E00E94602282E045
:100AB0008093B3030895CF93DF93EC018BAD88232C
:100AC00031F481E08BAFCE0104960F94620DCE011C
:100AD00004960F94700DDF91CF910895EF92FF92DD
:100AE0000F938FEC97E06091CD0792DF8FEC97E04A
:100AF000E2DF83ED97E060EA72E10F94540A83ED40
:100B000097E061E00F949F0D83ED97E060E040E097
:100B10002091D3070091D4070F94ED0883ED97E05F
:100B200061E00F949F0D83ED97E00F94740D88237F
:100B300001F78FEC97E0BFDF83ED97E060E040E0E6
:100B400028E000E434E8E32E36E2F32E0F940A0C9A
:100B500083ED97E060EA72E10F94540A83ED97E029
:100B60006DE341E121E232E00F94CD0A83ED97E09D
:100B700060EA72E10F94540A83ED97E065E541E184
:100B800025E232E00F94CD0A83ED97E060EA72E14E
:100B90000F94540A83ED97E06FE34DE128E232E0D1
:100BA0000F94CD0A83ED97E06FED75E30F94540A2F
:100BB00083ED97E06FE349E223E332E00F94CD0A3F
:100BC00083ED97E06FED75E30F94540A83ED97E0A2
:100BD0006FE345E32FE332E00F94CD0A83ED97E016
:100BE0006FE34EE329E432E00F94CD0A83ED97E002
:100BF0000F94740D882309F09FCF68EB7BE080E0B1
:100C000090E00F94990E0F91FF90EF900895EF925E
:100C1000FF920F931F930E94953429B130E074E046
:100C2000369527957A95E1F741E050E0242735275E
:100C3000217030708091160890E02817390711F163
:100C400082E08093B30389B190E064E09695879544
:100C50006A95E1F7842795278170809316083EDF17
:100C600080911608882339F087E498E00E9473E8A1
:100C700086E796E206C087E498E00E948FE089E666
:100C800096E2E8DEE0901708F09018080091190845
:100C900010911A080F948B0EE616F706080719072D
:100CA00008F0B8C020918905222361F181E080938A
:100CB000B303332727FD3095432F532F809112081C
:100CC00090911308A0911408B0911508820F931FFA
:100CD000A41FB51F8093120890931308A0931408C3
:100CE000B0931508109289050F948B0E6856754CB9
:100CF0008F4F9F4F6093430870934408809345083B
:100D00009093460880910B0882FF0EC00F948B0EC3
:100D10006856754C8F4F9F4F6093430870934408FB
:100D20008093450890934608809142088F5F809396
:100D300042088FEC97E0BFDE1DE783ED97E060EAA5
:100D400072E10F94540A10930808109209088091D8
:100D5000420880FF04C083ED97E061E003C083EDAB
:100D600097E060E00F949F0D83ED97E06FE74FE30E
:100D70000F94880D83ED97E061E00F949F0DE09153
:100D8000B103F091B20319958091B303882331F038
:100D900083ED97E00F94740D882379F6E090430873
:100DA000F090440800914508109146080F948B0E6E
:100DB000E616F70608071907C0F48091B103909171
:100DC000B203815A984389F01092120810921308C6
:100DD000109214081092150881EA98E39093B203D8
:100DE0008093B10382E08093B3038091B30388239F
:100DF00019F081508093B3030F948B0E6C597F4F81
:100E00008F4F9F4F609317087093180880931908AD
:100E100090931A081F910F91FF90EF9008955EDE56
:100E20008CE460E00F9432108DE460E00F94321097
:100E30009FB7F894E5E0F1E08081806280839FBFF6
:100E40009FB7F894E5E0F1E08081806480839FBFE4
:100E50008EE460E00F943210729A81E560E00F94A6
:100E600032105C9A89B182958F70809581708093E1
:100E700016080E9495341092890508956091C60560
:100E80007091C705882777FD8095982F0F94B51628
:100E90000F9482167093F00C6093EF0C6091C8056C
:100EA0007091C905882777FD8095982F0F94B51606
:100EB0000F9482167093F20C6093F10C8091CA0526
:100EC0009091CB0590930D0B80930C0B1092120810
:100ED00010921308109214081092150881EA98E3F2
:100EE0009093B2038093B1030C949AD46091C0059F
:100EF0007091C105882777FD8095982F0F94B516BE
:100F00000F9482167093F00C6093EF0C6091C20501
:100F10007091C305882777FD8095982F0F94B5169B
:100F20000F9482167093F20C6093F10C8091C405BB
:100F30009091C50590930D0B80930C0B10921208A5
:100F400010921308109214081092150881EA98E381
:100F50009093B2038093B1030C949AD46091BA0534
:100F60007091BB05882777FD8095982F0F94B51653
:100F70000F9482167093F00C6093EF0C6091BC0597
:100F80007091BD05882777FD8095982F0F94B51631
:100F90000F9482167093F20C6093F10C8091BE0551
:100FA0009091BF0590930D0B80930C0B109212083B
:100FB00010921308109214081092150881EA98E311
:100FC0009093B2038093B1030C949AD46091B405CA
:100FD0007091B505882777FD8095982F0F94B516E9
:100FE0000F9482167093F00C6093EF0C6091B6052D
:100FF0007091B705882777FD8095982F0F94B516C7
:101000000F9482167093F20C6093F10C8091B805E6
:101010009091B90590930D0B80930C0B10921208D0
:1010200010921308109214081092150881EA98E3A0
:101030009093B2038093B1030C949AD46091AE055F
:101040007091AF05882777FD8095982F0F94B5167E
:101050000F9482167093F00C6093EF0C6091B005C2
:101060007091B105882777FD8095982F0F94B5165C
:101070000F9482167093F20C6093F10C8091B2057C
:101080009091B30590930D0B80930C0B1092120866
:1010900010921308109214081092150881EA98E330
:1010A0009093B2038093B1030C949AD46091A805F5
:1010B0007091A905882777FD8095982F0F94B51614
:1010C0000F9482167093F00C6093EF0C6091AA0558
:1010D0007091AB05882777FD8095982F0F94B516F2
:1010E0000F9482167093F20C6093F10C8091AC0512
:1010F0009091AD0590930D0B80930C0B10921208FC
:1011000010921308109214081092150881EA98E3BF
:101110009093B2038093B1030C949AD46091A2058A
:101120007091A305882777FD8095982F0F94B516A9
:101130000F9482167093F00C6093EF0C6091A405ED
:101140007091A505882777FD8095982F0F94B51687
:101150000F9482167093F20C6093F10C8091A605A7
:101160009091A70590930D0B80930C0B1092120891
:1011700010921308109214081092150881EA98E34F
:101180009093B2038093B1030C949AD460919C0520
:1011900070919D05882777FD8095982F0F94B5163F
:1011A0000F9482167093F00C6093EF0C60919E0583
:1011B00070919F05882777FD8095982F0F94B5161D
:1011C0000F9482167093F20C6093F10C8091A0053D
:1011D0009091A10590930D0B80930C0B1092120827
:1011E00010921308109214081092150881EA98E3DF
:1011F0009093B2038093B1030C949AD460919605B6
:1012000070919705882777FD8095982F0F94B516D4
:101210000F9482167093F00C6093EF0C6091980518
:1012200070919905882777FD8095982F0F94B516B2
:101230000F9482167093F20C6093F10C80919A05D2
:1012400090919B0590930D0B80930C0B10921208BC
:1012500010921308109214081092150881EA98E36E
:101260009093B2038093B1030C949AD4609190054B
:1012700070919105882777FD8095982F0F94B5166A
:101280000F9482167093F00C6093EF0C60919205AE
:1012900070919305882777FD8095982F0F94B51648
:1012A0000F9482167093F20C6093F10C8091940568
:1012B0009091950590930D0B80930C0B1092120852
:1012C00010921308109214081092150881EA98E3FE
:1012D0009093B2038093B1030C949AD460918A05E1
:1012E00070918B05882777FD8095982F0F94B51600
:1012F0000F9482167093F00C6093EF0C60918C0544
:1013000070918D05882777FD8095982F0F94B516DD
:101310000F9482167093F20C6093F10C80918E05FD
:1013200090918F0590930D0B80930C0B10921208E7
:1013300010921308109214081092150881EA98E38D
:101340009093B2038093B1030C949AD44F925F921E
:101350006F927F928F929F92AF92BF92CF92DF92C5
:10136000EF92FF920F931F93CF93DF933C014B01BA
:10137000C42E29018AE0481729F095E1491709F0A0
:10138000D2C070C09C9AA4989B9AA39880910401A3
:101390008460809304019FB7F89480910501846074
:1013A000809305019FBFA49A0F9438088AE590E0C6
:1013B0000F942E0888EF0E942D310F94380880E09A
:1013C0000E942D3180E80E942D310F94380880E072
:1013D0000E942D3180E10E942D310F9438088AE05F
:1013E00090E00F942E0880E30E942D3180EE0E9441
:1013F0002D310F94380800E0802F807780680E949C
:101400002D31802F8295807F0E942D310F943808D6
:1014100080E80E942D3180E00E942D310F94380821
:101420008AEF0E942D310F94380810E080E00E946E
:101430002D3180E00E942D310F9438081F5F10324B
:10144000A9F788EF0E942D310F9438080F5F003202
:1014500099F680E00E942D3180EC0E942D310F948E
:10146000380860C0DB011296ED91FC911397D28091
:1014700016810781A49A0F943808812F902F7C0140
:10148000A12CE2E0BE2EAE0CBF1C88EF0E942D31D5
:101490000F943808BFE1BD1588F08D2D80778068E6
:1014A0000E942D318D2D8295807F0E942D310F94C9
:1014B000380880E80E942D3180E012C01D2D1052A6
:1014C000812F807780680E942D31812F8295807FC7
:1014D0000E942D310F94380880E80E942D3180E859
:1014E0000E942D310F9438088AEF0E942D310F94FD
:1014F0003808E70110E08881807F0E942D318991B2
:101500008295807F0E942D311F5F1031A1F780E10D
:1015100090E0E80EF91E0F943808EA14FB0411F06D
:10152000D394B3CFA498C301B4014C2D92010F946E
:10153000860BDF91CF911F910F91FF90EF90DF907D
:10154000CF90BF90AF909F908F907F906F905F9063
:101550004F900895AF92BF92CF92DF92EF92FF9299
:101560000F931F938091120890911308A091140873
:10157000B091150881509048A040B04040F01092C2
:101580001208109213081092140810921508609116
:10159000120870911308809114089091150825E0A5
:1015A00030E040E050E00F940B1A79018A018091FD
:1015B0000C0890E0A0E0B0E0E816F9060A071B0767
:1015C00010F420930C0800910C0880910B0890E017
:1015D0009695879596958795FF24F394F82210E0C9
:1015E000F5E4AF2EB12CC12CD12CEE24E3940023D2
:1015F00089F58091B3038823C1F0809112089091FE
:101600001308A0911408B09115080597A105B1051C
:1016100028F4812F6BEB71E24BEF04C0812F6BEB51
:1016200071E240E22BEF0E940C35FF2009F47FC3EA
:101630008091120890911308A0911408B091150898
:101640000597A105B10508F072C30E947D3883EDAE
:1016500091E441C0013009F04BC08091B30388236D
:10166000F9F060911208709113088091140890911C
:10167000150825E030E040E050E00F940B1A2130CF
:1016800031054105510529F4812F6FEA71E24EE3DE
:1016900004C0812F6FEA71E240E22AEF0E940C350C
:1016A000FF2009F444C360911208709113088091DF
:1016B00014089091150825E030E040E050E00F94C8
:1016C0000B1A213031054105510509F030C30E9444
:1016D0007D3880E998E79093B2038093B10310922C
:1016E000120810921308109214081092150858C38B
:1016F000023009F03EC08091B3038823F9F0609175
:10170000120870911308809114089091150825E033
:1017100030E040E050E00F940B1A223031054105D3
:10172000510529F4812F6BEA71E24EE304C0812F49
:101730006BEA71E240E220E20E940C35FF2009F4DE
:10174000F6C260911208709113088091140890916C
:10175000150825E030E040E050E00F940B1A2230ED
:1017600031054105510509F0E2C20E947D38B6DD20
:1017700017C3033009F03EC08091B3038823F9F00A
:1017800060911208709113088091140890911508C7
:1017900025E030E040E050E00F940B1A2330310593
:1017A0004105510529F4812F66EA71E24EE304C038
:1017B000812F66EA71E240E220E20E940C35FF20B0
:1017C00009F4B5C260911208709113088091140851
:1017D0009091150825E030E040E050E00F940B1A9E
:1017E000233031054105510509F0A1C20E947D3821
:1017F0003DDDD6C2043009F03EC08091B30388239A
:10180000F9F060911208709113088091140890917A
:10181000150825E030E040E050E00F940B1A24302A
:1018200031054105510529F4812F62EA71E24EE349
:1018300004C0812F62EA71E240E220E20E940C358E
:10184000FF2009F474C2609112087091130880910E
:1018500014089091150825E030E040E050E00F9426
:101860000B1A243031054105510509F060C20E9470
:101870007D38C4DC95C2053009F03EC08091B303C9
:101880008823F9F060911208709113088091140870
:101890009091150825E030E040E050E00F940B1ADD
:1018A000253031054105510529F4812F6BE971E29D
:1018B0004EE304C0812F6BE971E240E220E20E9416
:1018C0000C35FF2009F433C260911208709113089F
:1018D000809114089091150825E030E040E050E038
:1018E0000F940B1A253031054105510509F01FC22F
:1018F0000E947D384BDC54C2063009F03EC0809116
:10190000B3038823F9F06091120870911308809155
:1019100014089091150825E030E040E050E00F9465
:101920000B1A263031054105510529F4812F65E94F
:1019300071E24EE304C0812F65E971E240E220E2EA
:101940000E940C35FF2009F4F2C1609112087091D9
:101950001308809114089091150825E030E040E0CC
:1019600050E00F940B1A263031054105510509F05E
:10197000DEC10E947D38D2DB13C2073009F03EC0C1
:101980008091B3038823F9F06091120870911308D5
:10199000809114089091150825E030E040E050E077
:1019A0000F940B1A273031054105510529F4812F79
:1019B0006BE871E24EE304C0812F6BE871E240E214
:1019C00020E20E940C35FF2009F4B1C16091120899
:1019D00070911308809114089091150825E030E06B
:1019E00040E050E00F940B1A2730310541055105B6
:1019F00009F09DC10E947D3859DBD2C1083009F041
:101A00003EC08091B3038823F9F060911208709171
:101A10001308809114089091150825E030E040E00B
:101A200050E00F940B1A283031054105510529F477
:101A3000812F64E871E24EE304C0812F64E871E213
:101A400040E220E20E940C35FF2009F470C1609151
:101A5000120870911308809114089091150825E0E0
:101A600030E040E050E00F940B1A2830310541057A
:101A7000510509F05CC10E947D38E0DA91C109305E
:101A800009F03EC08091B3038823F9F060911208F9
:101A900070911308809114089091150825E030E0AA
:101AA00040E050E00F940B1A2930310541055105F3
:101AB00029F4812F6BE771E24EE304C0812F6BE7BD
:101AC00071E240E220E20E940C35FF2009F42FC1B0
:101AD0006091120870911308809114089091150874
:101AE00025E030E040E050E00F940B1A293031053A
:101AF0004105510509F01BC10E947D3867DA50C1CC
:101B00000A3009F03EC08091B3038823F9F0609158
:101B1000120870911308809114089091150825E01F
:101B200030E040E050E00F940B1A2A3031054105B7
:101B3000510529F4812F63E771E24EE304C0812F40
:101B400063E771E240E220E20E940C35FF2009F4D5
:101B5000EEC0609112087091130880911408909162
:101B6000150825E030E040E050E00F940B1A2A30D1
:101B700031054105510509F0DAC00E947D38EED9E2
:101B80000FC10B3009F03EC08091B3038823F9F0F8
:101B900060911208709113088091140890911508B3
:101BA00025E030E040E050E00F940B1A2B30310577
:101BB0004105510529F4812F6AE671E24EE304C024
:101BC000812F6AE671E240E220E20E940C35FF209C
:101BD00009F4ADC060911208709113088091140847
:101BE0009091150825E030E040E050E00F940B1A8A
:101BF0002B3031054105510509F099C00E947D380F
:101C000075D9CEC00C3009F03EC08091B303882353
